 java

 Timestamp is dfa8d2c4 (reproducible build file hash)

 Preferred load address is 0000000180000000

 Start         Length     Name                   Class
 0001:00000000 0000ddb0H .text$mn                CODE
 0001:0000ddb0 00000036H .text$mn$00             CODE
 0001:0000dde6 00000092H .text$x                 CODE
 0002:00000000 00000a88H .idata$5                DATA
 0002:00000a88 00000038H .00cfg                  DATA
 0002:00000ac0 00000008H .CRT$XCA                DATA
 0002:00000ac8 00000008H .CRT$XCZ                DATA
 0002:00000ad0 00000008H .CRT$XIA                DATA
 0002:00000ad8 00000008H .CRT$XIZ                DATA
 0002:00000ae0 00000008H .CRT$XPA                DATA
 0002:00000ae8 00000008H .CRT$XPZ                DATA
 0002:00000af0 00000008H .CRT$XTA                DATA
 0002:00000af8 00000008H .CRT$XTZ                DATA
 0002:00000b00 00000000H .gehcont$y              DATA
 0002:00000b00 00000000H .gfids$y                DATA
 0002:00000b00 00001b80H .rdata                  DATA
 0002:00002680 00000000H .rdata$CastGuardVftablesA DATA
 0002:00002680 00000000H .rdata$CastGuardVftablesC DATA
 0002:00002680 00000080H .rdata$voltmd           DATA
 0002:00002700 000002b8H .rdata$zzzdbg           DATA
 0002:000029b8 00000008H .rtc$IAA                DATA
 0002:000029c0 00000008H .rtc$IZZ                DATA
 0002:000029c8 00000008H .rtc$TAA                DATA
 0002:000029d0 00000008H .rtc$TZZ                DATA
 0002:000029d8 00000a18H .xdata                  DATA
 0002:000033f0 00003cccH .edata                  DATA
 0002:000070bc 00000118H .idata$2                DATA
 0002:000071d4 00000014H .idata$3                DATA
 0002:000071e8 00000a88H .idata$4                DATA
 0002:00007c70 00001d0eH .idata$6                DATA
 0003:00000000 00000d10H .data                   DATA
 0003:00000d10 000007e8H .bss                    DATA
 0004:00000000 00000d20H .pdata                  DATA
 0005:00000000 00000060H .rsrc$01                DATA
 0005:00000060 00000320H .rsrc$02                DATA

  Address         Publics by Value              Rva+Base               Lib:Object

 0000:00000000       __AbsoluteZero             0000000000000000     <absolute>
 0000:00000000       ___safe_se_handler_count   0000000000000000     <absolute>
 0000:00000000       ___safe_se_handler_table   0000000000000000     <absolute>
 0000:00000000       __arm64x_extra_rfe_table   0000000000000000     <absolute>
 0000:00000000       __arm64x_extra_rfe_table_size 0000000000000000     <absolute>
 0000:00000000       __arm64x_native_entrypoint 0000000000000000     <absolute>
 0000:00000000       __arm64x_redirection_metadata 0000000000000000     <absolute>
 0000:00000000       __arm64x_redirection_metadata_count 0000000000000000     <absolute>
 0000:00000000       __dynamic_value_reloc_table 0000000000000000     <absolute>
 0000:00000000       __enclave_config           0000000000000000     <absolute>
 0000:00000000       __guard_check_icall_a64n_fptr 0000000000000000     <absolute>
 0000:00000000       __guard_eh_cont_count      0000000000000000     <absolute>
 0000:00000000       __guard_eh_cont_table      0000000000000000     <absolute>
 0000:00000000       __guard_fids_count         0000000000000000     <absolute>
 0000:00000000       __guard_fids_table         0000000000000000     <absolute>
 0000:00000000       __guard_iat_count          0000000000000000     <absolute>
 0000:00000000       __guard_iat_table          0000000000000000     <absolute>
 0000:00000000       __guard_longjmp_count      0000000000000000     <absolute>
 0000:00000000       __guard_longjmp_table      0000000000000000     <absolute>
 0000:00000000       __hybrid_auxiliary_delayload_iat 0000000000000000     <absolute>
 0000:00000000       __hybrid_auxiliary_delayload_iat_copy 0000000000000000     <absolute>
 0000:00000000       __hybrid_auxiliary_iat     0000000000000000     <absolute>
 0000:00000000       __hybrid_auxiliary_iat_copy 0000000000000000     <absolute>
 0000:00000000       __hybrid_code_map          0000000000000000     <absolute>
 0000:00000000       __hybrid_code_map_count    0000000000000000     <absolute>
 0000:00000000       __hybrid_image_info_bitfield 0000000000000000     <absolute>
 0000:00000000       __x64_code_ranges_to_entry_points 0000000000000000     <absolute>
 0000:00000000       __x64_code_ranges_to_entry_points_count 0000000000000000     <absolute>
 0000:00000100       __guard_flags              0000000000000100     <absolute>
 0000:00000000       __ImageBase                0000000180000000     <linker-defined>
 0001:00000000       Java_java_lang_reflect_Array_get 0000000180001000 f   Array.obj
 0001:0000000c       Java_java_lang_reflect_Array_getBoolean 000000018000100c f   Array.obj
 0001:00000020       Java_java_lang_reflect_Array_getByte 0000000180001020 f   Array.obj
 0001:00000034       Java_java_lang_reflect_Array_getChar 0000000180001034 f   Array.obj
 0001:00000048       Java_java_lang_reflect_Array_getDouble 0000000180001048 f   Array.obj
 0001:00000070       Java_java_lang_reflect_Array_getFloat 0000000180001070 f   Array.obj
 0001:00000098       Java_java_lang_reflect_Array_getInt 0000000180001098 f   Array.obj
 0001:000000ac       Java_java_lang_reflect_Array_getLength 00000001800010ac f   Array.obj
 0001:000000b4       Java_java_lang_reflect_Array_getLong 00000001800010b4 f   Array.obj
 0001:000000c8       Java_java_lang_reflect_Array_getShort 00000001800010c8 f   Array.obj
 0001:000000dc       Java_java_lang_reflect_Array_multiNewArray 00000001800010dc f   Array.obj
 0001:000000e8       Java_java_lang_reflect_Array_newArray 00000001800010e8 f   Array.obj
 0001:000000f4       Java_java_lang_reflect_Array_set 00000001800010f4 f   Array.obj
 0001:00000108       Java_java_lang_reflect_Array_setBoolean 0000000180001108 f   Array.obj
 0001:00000130       Java_java_lang_reflect_Array_setByte 0000000180001130 f   Array.obj
 0001:00000158       Java_java_lang_reflect_Array_setChar 0000000180001158 f   Array.obj
 0001:00000184       Java_java_lang_reflect_Array_setDouble 0000000180001184 f   Array.obj
 0001:000001a8       Java_java_lang_reflect_Array_setFloat 00000001800011a8 f   Array.obj
 0001:000001d4       Java_java_lang_reflect_Array_setInt 00000001800011d4 f   Array.obj
 0001:000001fc       Java_java_lang_reflect_Array_setLong 00000001800011fc f   Array.obj
 0001:00000220       Java_java_lang_reflect_Array_setShort 0000000180001220 f   Array.obj
 0001:0000024c       Java_jdk_internal_loader_BootLoader_getSystemPackageLocation 000000018000124c f   BootLoader.obj
 0001:00000254       Java_jdk_internal_loader_BootLoader_getSystemPackageNames 0000000180001254 f   BootLoader.obj
 0001:0000025c       Java_jdk_internal_loader_BootLoader_setBootLoaderUnnamedModule0 000000018000125c f   BootLoader.obj
 0001:00000264       Java_jdk_internal_misc_CDS_defineArchivedModules 0000000180001264 f   CDS.obj
 0001:00000270       Java_jdk_internal_misc_CDS_dumpClassList 0000000180001270 f   CDS.obj
 0001:00000278       Java_jdk_internal_misc_CDS_dumpDynamicArchive 0000000180001278 f   CDS.obj
 0001:00000280       Java_jdk_internal_misc_CDS_getCDSConfigStatus 0000000180001280 f   CDS.obj
 0001:00000288       Java_jdk_internal_misc_CDS_getRandomSeedForDumping 0000000180001288 f   CDS.obj
 0001:00000290       Java_jdk_internal_misc_CDS_initializeFromArchive 0000000180001290 f   CDS.obj
 0001:00000298       Java_jdk_internal_misc_CDS_logLambdaFormInvoker 0000000180001298 f   CDS.obj
 0001:000002a0       Java_jdk_internal_misc_CDS_needsClassInitBarrier0 00000001800012a0 f   CDS.obj
 0001:000002a8       Java_java_lang_Class_forName0 00000001800012a8 f   Class.obj
 0001:00000404       Java_java_lang_Class_getPrimitiveClass 0000000180001404 f   Class.obj
 0001:00000480       Java_java_lang_Class_isAssignableFrom 0000000180001480 f   Class.obj
 0001:000004ac       Java_java_lang_Class_isInstance 00000001800014ac f   Class.obj
 0001:000004c8       Java_java_lang_Class_registerNatives 00000001800014c8 f   Class.obj
 0001:000004f0       Java_java_lang_ClassLoader_defineClass0 00000001800014f0 f   ClassLoader.obj
 0001:00000680       Java_java_lang_ClassLoader_defineClass1 0000000180001680 f   ClassLoader.obj
 0001:00000830       Java_java_lang_ClassLoader_defineClass2 0000000180001830 f   ClassLoader.obj
 0001:00000994       Java_java_lang_ClassLoader_findBootstrapClass 0000000180001994 f   ClassLoader.obj
 0001:00000a44       Java_java_lang_ClassLoader_findLoadedClass0 0000000180001a44 f   ClassLoader.obj
 0001:00000a54       Java_java_lang_ClassLoader_registerNatives 0000000180001a54 f   ClassLoader.obj
 0001:00000b10       Java_java_io_Console_istty 0000000180001b10 f   Console_md.obj
 0001:00000b64       Java_jdk_internal_reflect_ConstantPool_getClassAt0 0000000180001b64 f   ConstantPool.obj
 0001:00000b6c       Java_jdk_internal_reflect_ConstantPool_getClassAtIfLoaded0 0000000180001b6c f   ConstantPool.obj
 0001:00000b74       Java_jdk_internal_reflect_ConstantPool_getClassRefIndexAt0 0000000180001b74 f   ConstantPool.obj
 0001:00000b7c       Java_jdk_internal_reflect_ConstantPool_getDoubleAt0 0000000180001b7c f   ConstantPool.obj
 0001:00000b84       Java_jdk_internal_reflect_ConstantPool_getFieldAt0 0000000180001b84 f   ConstantPool.obj
 0001:00000b8c       Java_jdk_internal_reflect_ConstantPool_getFieldAtIfLoaded0 0000000180001b8c f   ConstantPool.obj
 0001:00000b94       Java_jdk_internal_reflect_ConstantPool_getFloatAt0 0000000180001b94 f   ConstantPool.obj
 0001:00000b9c       Java_jdk_internal_reflect_ConstantPool_getIntAt0 0000000180001b9c f   ConstantPool.obj
 0001:00000ba4       Java_jdk_internal_reflect_ConstantPool_getLongAt0 0000000180001ba4 f   ConstantPool.obj
 0001:00000bac       Java_jdk_internal_reflect_ConstantPool_getMemberRefInfoAt0 0000000180001bac f   ConstantPool.obj
 0001:00000bb4       Java_jdk_internal_reflect_ConstantPool_getMethodAt0 0000000180001bb4 f   ConstantPool.obj
 0001:00000bbc       Java_jdk_internal_reflect_ConstantPool_getMethodAtIfLoaded0 0000000180001bbc f   ConstantPool.obj
 0001:00000bc4       Java_jdk_internal_reflect_ConstantPool_getNameAndTypeRefIndexAt0 0000000180001bc4 f   ConstantPool.obj
 0001:00000bcc       Java_jdk_internal_reflect_ConstantPool_getNameAndTypeRefInfoAt0 0000000180001bcc f   ConstantPool.obj
 0001:00000bd4       Java_jdk_internal_reflect_ConstantPool_getSize0 0000000180001bd4 f   ConstantPool.obj
 0001:00000bdc       Java_jdk_internal_reflect_ConstantPool_getStringAt0 0000000180001bdc f   ConstantPool.obj
 0001:00000be4       Java_jdk_internal_reflect_ConstantPool_getTagAt0 0000000180001be4 f   ConstantPool.obj
 0001:00000bec       Java_jdk_internal_reflect_ConstantPool_getUTF8At0 0000000180001bec f   ConstantPool.obj
 0001:00000bf4       Java_jdk_internal_vm_Continuation_registerNatives 0000000180001bf4 f   Continuation.obj
 0001:00000bfc       Java_jdk_internal_vm_ContinuationSupport_isSupported0 0000000180001bfc f   ContinuationSupport.obj
 0001:00000c04       Java_java_lang_Double_doubleToRawLongBits 0000000180001c04 f   Double.obj
 0001:00000c10       Java_java_lang_Double_longBitsToDouble 0000000180001c10 f   Double.obj
 0001:00000c1c       Java_java_lang_reflect_Executable_getParameters0 0000000180001c1c f   Executable.obj
 0001:00000c24       Java_java_lang_reflect_Executable_getTypeAnnotationBytes0 0000000180001c24 f   Executable.obj
 0001:00000c2c       Java_java_lang_reflect_Field_getTypeAnnotationBytes0 0000000180001c2c f   Field.obj
 0001:00000c34       Java_java_io_FileCleanable_cleanupClose0 0000000180001c34 f   FileDescriptor_md.obj
 0001:00000c64       Java_java_io_FileDescriptor_close0 0000000180001c64 f   FileDescriptor_md.obj
 0001:00000c6c       Java_java_io_FileDescriptor_getAppend 0000000180001c6c f   FileDescriptor_md.obj
 0001:00000c70       Java_java_io_FileDescriptor_getHandle 0000000180001c70 f   FileDescriptor_md.obj
 0001:00000ca0       Java_java_io_FileDescriptor_initIDs 0000000180001ca0 f   FileDescriptor_md.obj
 0001:00000d2c       Java_java_io_FileDescriptor_sync0 0000000180001d2c f   FileDescriptor_md.obj
 0001:00000d70       Java_java_io_FileInputStream_available0 0000000180001d70 f   FileInputStream.obj
 0001:00000ddc       Java_java_io_FileInputStream_initIDs 0000000180001ddc f   FileInputStream.obj
 0001:00000e04       Java_java_io_FileInputStream_isRegularFile0 0000000180001e04 f   FileInputStream.obj
 0001:00000e2c       Java_java_io_FileInputStream_length0 0000000180001e2c f   FileInputStream.obj
 0001:00000e90       Java_java_io_FileInputStream_open0 0000000180001e90 f   FileInputStream.obj
 0001:00000eac       Java_java_io_FileInputStream_position0 0000000180001eac f   FileInputStream.obj
 0001:00000f14       Java_java_io_FileInputStream_read0 0000000180001f14 f   FileInputStream.obj
 0001:00000f20       Java_java_io_FileInputStream_readBytes 0000000180001f20 f   FileInputStream.obj
 0001:00000f44       Java_java_io_FileInputStream_skip0 0000000180001f44 f   FileInputStream.obj
 0001:00000ff0       Java_java_io_FileOutputStream_initIDs 0000000180001ff0 f   FileOutputStream.obj
 0001:00001018       Java_java_io_FileOutputStream_open0 0000000180002018 f   FileOutputStream.obj
 0001:00001040       Java_java_io_FileOutputStream_write 0000000180002040 f   FileOutputStream.obj
 0001:0000105c       Java_java_io_FileOutputStream_writeBytes 000000018000205c f   FileOutputStream.obj
 0001:00001088       Java_java_lang_ref_Finalizer_isFinalizationEnabled 0000000180002088 f   Finalizer.obj
 0001:00001090       Java_java_lang_ref_Finalizer_reportComplete 0000000180002090 f   Finalizer.obj
 0001:00001098       Java_java_lang_Float_floatToRawIntBits 0000000180002098 f   Float.obj
 0001:000010a4       Java_java_lang_Float_intBitsToFloat 00000001800020a4 f   Float.obj
 0001:000010b0       Java_jdk_internal_vm_ForeignLinkerSupport_isSupported0 00000001800020b0 f   ForeignLinkerSupport.obj
 0001:000010b8       EnumCalendarInfoProc       00000001800020b8 f   HostLocaleProviderAdapter_md.obj
 0001:000010f4       Java_sun_util_locale_provider_HostLocaleProviderAdapterImpl_getAmPmStrings 00000001800020f4 f   HostLocaleProviderAdapter_md.obj
 0001:00001138       Java_sun_util_locale_provider_HostLocaleProviderAdapterImpl_getCalendarDataValue 0000000180002138 f   HostLocaleProviderAdapter_md.obj
 0001:000011c8       Java_sun_util_locale_provider_HostLocaleProviderAdapterImpl_getCalendarDisplayStrings 00000001800021c8 f   HostLocaleProviderAdapter_md.obj
 0001:00001364       Java_sun_util_locale_provider_HostLocaleProviderAdapterImpl_getCalendarID 0000000180002364 f   HostLocaleProviderAdapter_md.obj
 0001:000013cc       Java_sun_util_locale_provider_HostLocaleProviderAdapterImpl_getCurrencySymbol 00000001800023cc f   HostLocaleProviderAdapter_md.obj
 0001:00001490       Java_sun_util_locale_provider_HostLocaleProviderAdapterImpl_getDateTimePattern 0000000180002490 f   HostLocaleProviderAdapter_md.obj
 0001:0000159c       Java_sun_util_locale_provider_HostLocaleProviderAdapterImpl_getDecimalSeparator 000000018000259c f   HostLocaleProviderAdapter_md.obj
 0001:00001648       Java_sun_util_locale_provider_HostLocaleProviderAdapterImpl_getDefaultLocale 0000000180002648 f   HostLocaleProviderAdapter_md.obj
 0001:000016bc       Java_sun_util_locale_provider_HostLocaleProviderAdapterImpl_getDisplayString 00000001800026bc f   HostLocaleProviderAdapter_md.obj
 0001:000017ac       Java_sun_util_locale_provider_HostLocaleProviderAdapterImpl_getEras 00000001800027ac f   HostLocaleProviderAdapter_md.obj
 0001:000017cc       Java_sun_util_locale_provider_HostLocaleProviderAdapterImpl_getGroupingSeparator 00000001800027cc f   HostLocaleProviderAdapter_md.obj
 0001:00001878       Java_sun_util_locale_provider_HostLocaleProviderAdapterImpl_getInfinity 0000000180002878 f   HostLocaleProviderAdapter_md.obj
 0001:0000193c       Java_sun_util_locale_provider_HostLocaleProviderAdapterImpl_getInternationalCurrencySymbol 000000018000293c f   HostLocaleProviderAdapter_md.obj
 0001:00001a00       Java_sun_util_locale_provider_HostLocaleProviderAdapterImpl_getMinusSign 0000000180002a00 f   HostLocaleProviderAdapter_md.obj
 0001:00001aac       Java_sun_util_locale_provider_HostLocaleProviderAdapterImpl_getMonetaryDecimalSeparator 0000000180002aac f   HostLocaleProviderAdapter_md.obj
 0001:00001b58       Java_sun_util_locale_provider_HostLocaleProviderAdapterImpl_getMonths 0000000180002b58 f   HostLocaleProviderAdapter_md.obj
 0001:00001ba0       Java_sun_util_locale_provider_HostLocaleProviderAdapterImpl_getNaN 0000000180002ba0 f   HostLocaleProviderAdapter_md.obj
 0001:00001c64       Java_sun_util_locale_provider_HostLocaleProviderAdapterImpl_getNumberPattern 0000000180002c64 f   HostLocaleProviderAdapter_md.obj
 0001:00001d0c       Java_sun_util_locale_provider_HostLocaleProviderAdapterImpl_getPerMill 0000000180002d0c f   HostLocaleProviderAdapter_md.obj
 0001:00001db8       Java_sun_util_locale_provider_HostLocaleProviderAdapterImpl_getPercent 0000000180002db8 f   HostLocaleProviderAdapter_md.obj
 0001:00001e64       Java_sun_util_locale_provider_HostLocaleProviderAdapterImpl_getShortMonths 0000000180002e64 f   HostLocaleProviderAdapter_md.obj
 0001:00001eac       Java_sun_util_locale_provider_HostLocaleProviderAdapterImpl_getShortWeekdays 0000000180002eac f   HostLocaleProviderAdapter_md.obj
 0001:00001ef4       Java_sun_util_locale_provider_HostLocaleProviderAdapterImpl_getWeekdays 0000000180002ef4 f   HostLocaleProviderAdapter_md.obj
 0001:00001f3c       Java_sun_util_locale_provider_HostLocaleProviderAdapterImpl_getZeroDigit 0000000180002f3c f   HostLocaleProviderAdapter_md.obj
 0001:00001fe8       Java_sun_util_locale_provider_HostLocaleProviderAdapterImpl_initialize 0000000180002fe8 f   HostLocaleProviderAdapter_md.obj
 0001:0000209c       Java_sun_util_locale_provider_HostLocaleProviderAdapterImpl_isNativeDigit 000000018000309c f   HostLocaleProviderAdapter_md.obj
 0001:00002120       enumCalendarInfoWrapper    0000000180003120 f   HostLocaleProviderAdapter_md.obj
 0001:000021a0       getCalendarID              00000001800031a0 f   HostLocaleProviderAdapter_md.obj
 0001:00002210       getCalendarInfoWrapper     0000000180003210 f   HostLocaleProviderAdapter_md.obj
 0001:000022a0       getErasImpl                00000001800032a0 f   HostLocaleProviderAdapter_md.obj
 0001:00002528       getFixPart                 0000000180003528 f   HostLocaleProviderAdapter_md.obj
 0001:000025ec       getLocaleInfoWrapper       00000001800035ec f   HostLocaleProviderAdapter_md.obj
 0001:0000265c       getNumberPart              000000018000365c f   HostLocaleProviderAdapter_md.obj
 0001:0000281c       getNumberPattern           000000018000381c f   HostLocaleProviderAdapter_md.obj
 0001:000029cc       replaceCalendarArrayElems  00000001800039cc f   HostLocaleProviderAdapter_md.obj
 0001:00002b5c       Java_jdk_internal_io_JdkConsoleImpl_echo 0000000180003b5c f   JdkConsoleImpl_md.obj
 0001:00002c00       Java_java_lang_invoke_LambdaProxyClassArchive_addToArchive 0000000180003c00 f   LambdaProxyClassArchive.obj
 0001:00002c4c       Java_java_lang_invoke_LambdaProxyClassArchive_findFromArchive 0000000180003c4c f   LambdaProxyClassArchive.obj
 0001:00002c8c       Java_java_lang_Module_addExports0 0000000180003c8c f   Module.obj
 0001:00002ca0       Java_java_lang_Module_addExportsToAll0 0000000180003ca0 f   Module.obj
 0001:00002cac       Java_java_lang_Module_addExportsToAllUnnamed0 0000000180003cac f   Module.obj
 0001:00002cb8       Java_java_lang_Module_addReads0 0000000180003cb8 f   Module.obj
 0001:00002cc4       Java_java_lang_Module_defineModule0 0000000180003cc4 f   Module.obj
 0001:00002cf4       Java_jdk_internal_reflect_DirectConstructorHandleAccessor_00024NativeAccessor_newInstance0 0000000180003cf4 f   NativeAccessors.obj
 0001:00002d00       Java_jdk_internal_reflect_DirectMethodHandleAccessor_00024NativeAccessor_invoke0 0000000180003d00 f   NativeAccessors.obj
 0001:00002d14       Java_jdk_internal_loader_NativeLibraries_findBuiltinLib 0000000180003d14 f   NativeLibraries.obj
 0001:00002e6c       Java_jdk_internal_loader_NativeLibraries_load 0000000180003e6c f   NativeLibraries.obj
 0001:00003098       Java_jdk_internal_loader_NativeLibraries_unload 0000000180004098 f   NativeLibraries.obj
 0001:00003150       Java_jdk_internal_loader_NativeLibrary_findEntry0 0000000180004150 f   NativeLibraries.obj
 0001:0000333c       Java_java_lang_NullPointerException_getExtendedNPEMessage 000000018000433c f   NullPointerException.obj
 0001:00003344       Java_java_lang_Object_getClass 0000000180004344 f   Object.obj
 0001:00003368       Java_java_io_ObjectStreamClass_hasStaticInitializer 0000000180004368 f   ObjectStreamClass.obj
 0001:0000346c       Java_java_io_ObjectStreamClass_initNative 000000018000446c f   ObjectStreamClass.obj
 0001:000034a4       Java_java_lang_ref_PhantomReference_clear0 00000001800044a4 f   PhantomReference.obj
 0001:000034a4       Java_java_lang_ref_Reference_clear0 00000001800044a4 f   Reference.obj
 0001:000034ac       Java_java_lang_ref_PhantomReference_refersTo0 00000001800044ac f   PhantomReference.obj
 0001:000034b4       Java_jdk_internal_misc_PreviewFeatures_isPreviewEnabled 00000001800044b4 f   PreviewFeatures.obj
 0001:000034bc       Java_java_lang_ProcessEnvironment_environmentBlock 00000001800044bc f   ProcessEnvironment_md.obj
 0001:00003538       Java_java_lang_ProcessHandleImpl_00024Info_info0 0000000180004538 f   ProcessHandleImpl_win.obj
 0001:000035a8       Java_java_lang_ProcessHandleImpl_00024Info_initIDs 00000001800045a8 f   ProcessHandleImpl_win.obj
 0001:000036b8       Java_java_lang_ProcessHandleImpl_destroy0 00000001800046b8 f   ProcessHandleImpl_win.obj
 0001:00003724       Java_java_lang_ProcessHandleImpl_getCurrentPid0 0000000180004724 f   ProcessHandleImpl_win.obj
 0001:00003738       Java_java_lang_ProcessHandleImpl_getProcessPids0 0000000180004738 f   ProcessHandleImpl_win.obj
 0001:00003a2c       Java_java_lang_ProcessHandleImpl_initNative 0000000180004a2c f   ProcessHandleImpl_win.obj
 0001:00003a2c       _guard_check_icall_nop     0000000180004a2c f   MSVCRT:guard_support.obj
 0001:00003a30       Java_java_lang_ProcessHandleImpl_isAlive0 0000000180004a30 f   ProcessHandleImpl_win.obj
 0001:00003a90       Java_java_lang_ProcessHandleImpl_parent0 0000000180004a90 f   ProcessHandleImpl_win.obj
 0001:00003bac       Java_java_lang_ProcessHandleImpl_waitForProcessExit0 0000000180004bac f   ProcessHandleImpl_win.obj
 0001:00004090       Java_java_lang_ProcessImpl_closeHandle 0000000180005090 f   ProcessImpl_md.obj
 0001:0000409c       Java_java_lang_ProcessImpl_create 000000018000509c f   ProcessImpl_md.obj
 0001:000042a4       Java_java_lang_ProcessImpl_getExitCodeProcess 00000001800052a4 f   ProcessImpl_md.obj
 0001:000042d8       Java_java_lang_ProcessImpl_getProcessId0 00000001800052d8 f   ProcessImpl_md.obj
 0001:000042e4       Java_java_lang_ProcessImpl_getStillActive 00000001800052e4 f   ProcessImpl_md.obj
 0001:000042ec       Java_java_lang_ProcessImpl_isProcessAlive 00000001800052ec f   ProcessImpl_md.obj
 0001:00004308       Java_java_lang_ProcessImpl_openForAtomicAppend 0000000180005308 f   ProcessImpl_md.obj
 0001:00004394       Java_java_lang_ProcessImpl_terminateProcess 0000000180005394 f   ProcessImpl_md.obj
 0001:000043a4       Java_java_lang_ProcessImpl_waitForInterruptibly 00000001800053a4 f   ProcessImpl_md.obj
 0001:000043ec       Java_java_lang_ProcessImpl_waitForTimeoutInterruptibly 00000001800053ec f   ProcessImpl_md.obj
 0001:00004440       __local_stdio_printf_options 0000000180005440 f i ProcessImpl_md.obj
 0001:000044f0       os_error_message           00000001800054f0 f   ProcessImpl_md.obj
 0001:000048bc       swprintf                   00000001800058bc f i ProcessImpl_md.obj
 0001:00004a38       Java_java_io_RandomAccessFile_getFilePointer 0000000180005a38 f   RandomAccessFile.obj
 0001:00004aa0       Java_java_io_RandomAccessFile_initIDs 0000000180005aa0 f   RandomAccessFile.obj
 0001:00004ac8       Java_java_io_RandomAccessFile_length0 0000000180005ac8 f   RandomAccessFile.obj
 0001:00004b2c       Java_java_io_RandomAccessFile_open0 0000000180005b2c f   RandomAccessFile.obj
 0001:00004b84       Java_java_io_RandomAccessFile_read0 0000000180005b84 f   RandomAccessFile.obj
 0001:00004b90       Java_java_io_RandomAccessFile_readBytes0 0000000180005b90 f   RandomAccessFile.obj
 0001:00004bb4       Java_java_io_RandomAccessFile_seek0 0000000180005bb4 f   RandomAccessFile.obj
 0001:00004c24       Java_java_io_RandomAccessFile_setLength0 0000000180005c24 f   RandomAccessFile.obj
 0001:00004cd0       Java_java_io_RandomAccessFile_write0 0000000180005cd0 f   RandomAccessFile.obj
 0001:00004cf0       Java_java_io_RandomAccessFile_writeBytes0 0000000180005cf0 f   RandomAccessFile.obj
 0001:00004d18       Java_jdk_internal_loader_RawNativeLibraries_load0 0000000180005d18 f   RawNativeLibraries.obj
 0001:00004db4       Java_jdk_internal_loader_RawNativeLibraries_unload0 0000000180005db4 f   RawNativeLibraries.obj
 0001:00004e78       Java_java_lang_ref_Reference_getAndClearReferencePendingList 0000000180005e78 f   Reference.obj
 0001:00004e80       Java_java_lang_ref_Reference_hasReferencePendingList 0000000180005e80 f   Reference.obj
 0001:00004e88       Java_java_lang_ref_Reference_refersTo0 0000000180005e88 f   Reference.obj
 0001:00004e90       Java_java_lang_ref_Reference_waitForReferencePendingList 0000000180005e90 f   Reference.obj
 0001:00004e98       Java_jdk_internal_reflect_Reflection_areNestMates 0000000180005e98 f   Reflection.obj
 0001:00004ea4       Java_jdk_internal_reflect_Reflection_getCallerClass 0000000180005ea4 f   Reflection.obj
 0001:00004eac       Java_jdk_internal_reflect_Reflection_getClassAccessFlags 0000000180005eac f   Reflection.obj
 0001:00004eb4       Java_java_lang_Runtime_availableProcessors 0000000180005eb4 f   Runtime.obj
 0001:00004ebc       Java_java_lang_Runtime_freeMemory 0000000180005ebc f   Runtime.obj
 0001:00004ec4       Java_java_lang_Runtime_gc  0000000180005ec4 f   Runtime.obj
 0001:00004ecc       Java_java_lang_Runtime_maxMemory 0000000180005ecc f   Runtime.obj
 0001:00004ed4       Java_java_lang_Runtime_totalMemory 0000000180005ed4 f   Runtime.obj
 0001:00004edc       Java_java_lang_Shutdown_beforeHalt 0000000180005edc f   Shutdown.obj
 0001:00004ee4       Java_java_lang_Shutdown_halt0 0000000180005ee4 f   Shutdown.obj
 0001:00004eec       Java_jdk_internal_misc_Signal_findSignal0 0000000180005eec f   Signal.obj
 0001:00004f68       Java_jdk_internal_misc_Signal_handle0 0000000180005f68 f   Signal.obj
 0001:00004f74       Java_jdk_internal_misc_Signal_raise0 0000000180005f74 f   Signal.obj
 0001:00004f7c       Java_java_lang_StackFrameInfo_expandStackFrameInfo 0000000180005f7c f   StackFrameInfo.obj
 0001:00004f84       Java_java_lang_StackStreamFactory_00024AbstractStackWalker_callStackWalk 0000000180005f84 f   StackStreamFactory.obj
 0001:00004f8c       Java_java_lang_StackStreamFactory_00024AbstractStackWalker_fetchStackFrames 0000000180005f8c f   StackStreamFactory.obj
 0001:00004f94       Java_java_lang_StackStreamFactory_00024AbstractStackWalker_setContinuation 0000000180005f94 f   StackStreamFactory.obj
 0001:00004f9c       Java_java_lang_StackStreamFactory_checkStackWalkModes 0000000180005f9c f   StackStreamFactory.obj
 0001:00004f9c       __acrt_initialize          0000000180005f9c f   MSVCRT:ucrt_stubs.obj
 0001:00004f9c       __acrt_thread_attach       0000000180005f9c f   MSVCRT:ucrt_stubs.obj
 0001:00004f9c       __acrt_thread_detach       0000000180005f9c f   MSVCRT:ucrt_stubs.obj
 0001:00004f9c       __acrt_uninitialize        0000000180005f9c f   MSVCRT:ucrt_stubs.obj
 0001:00004f9c       __acrt_uninitialize_critical 0000000180005f9c f   MSVCRT:ucrt_stubs.obj
 0001:00004f9c       __scrt_stub_for_acrt_initialize 0000000180005f9c f   MSVCRT:ucrt_stubs.obj
 0001:00004f9c       __scrt_stub_for_acrt_thread_attach 0000000180005f9c f   MSVCRT:ucrt_stubs.obj
 0001:00004f9c       __scrt_stub_for_acrt_thread_detach 0000000180005f9c f   MSVCRT:ucrt_stubs.obj
 0001:00004f9c       __scrt_stub_for_acrt_uninitialize 0000000180005f9c f   MSVCRT:ucrt_stubs.obj
 0001:00004f9c       __scrt_stub_for_acrt_uninitialize_critical 0000000180005f9c f   MSVCRT:ucrt_stubs.obj
 0001:00004f9c       __vcrt_initialize          0000000180005f9c f   MSVCRT:ucrt_stubs.obj
 0001:00004f9c       __vcrt_thread_attach       0000000180005f9c f   MSVCRT:ucrt_stubs.obj
 0001:00004f9c       __vcrt_thread_detach       0000000180005f9c f   MSVCRT:ucrt_stubs.obj
 0001:00004f9c       __vcrt_uninitialize        0000000180005f9c f   MSVCRT:ucrt_stubs.obj
 0001:00004f9c       __vcrt_uninitialize_critical 0000000180005f9c f   MSVCRT:ucrt_stubs.obj
 0001:00004f9c       handleIsRegularFile        0000000180005f9c f   io_util_md.obj
 0001:00004fa0       Java_java_lang_StackTraceElement_initStackTraceElement 0000000180005fa0 f   StackTraceElement.obj
 0001:00004fac       Java_java_lang_StackTraceElement_initStackTraceElements 0000000180005fac f   StackTraceElement.obj
 0001:00004fc0       Java_java_lang_String_intern 0000000180005fc0 f   String.obj
 0001:00004fc8       Java_java_lang_System_identityHashCode 0000000180005fc8 f   System.obj
 0001:00004fd0       Java_java_lang_System_mapLibraryName 0000000180005fd0 f   System.obj
 0001:00005110       Java_java_lang_System_registerNatives 0000000180006110 f   System.obj
 0001:00005128       Java_java_lang_System_setErr0 0000000180006128 f   System.obj
 0001:00005184       Java_java_lang_System_setIn0 0000000180006184 f   System.obj
 0001:000051e0       Java_java_lang_System_setOut0 00000001800061e0 f   System.obj
 0001:0000523c       Java_jdk_internal_util_SystemProps_00024Raw_platformProperties 000000018000623c f   System.obj
 0001:00005d10       Java_jdk_internal_util_SystemProps_00024Raw_vmProperties 0000000180006d10 f   System.obj
 0001:00005d18       Java_java_lang_Thread_clearInterruptEvent 0000000180006d18 f   Thread.obj
 0001:00005d30       Java_java_lang_Thread_registerNatives 0000000180006d30 f   Thread.obj
 0001:00005d48       Java_jdk_internal_vm_ThreadSnapshot_create 0000000180006d48 f   ThreadSnapshot.obj
 0001:00005d50       Java_java_lang_Throwable_fillInStackTrace 0000000180006d50 f   Throwable.obj
 0001:00005d68       Java_java_util_TimeZone_getSystemGMTOffsetID 0000000180006d68 f   TimeZone.obj
 0001:00005db4       Java_java_util_TimeZone_getSystemTimeZoneID 0000000180006db4 f   TimeZone.obj
 0001:00005ec0       findJavaTZ_md              0000000180006ec0 f   TimeZone_md.obj
 0001:00005f4c       getGMTOffsetID             0000000180006f4c f   TimeZone_md.obj
 0001:000068bc       snprintf                   00000001800078bc f i TimeZone_md.obj
 0001:00006914       Java_jdk_internal_misc_VM_getRuntimeArguments 0000000180007914 f   VM.obj
 0001:0000691c       Java_jdk_internal_misc_VM_initialize 000000018000791c f   VM.obj
 0001:00006934       Java_jdk_internal_misc_VM_latestUserDefinedLoader0 0000000180007934 f   VM.obj
 0001:0000693c       Java_jdk_internal_vm_VMSupport_getVMTemporaryDirectory 000000018000793c f   VMSupport.obj
 0001:00006944       Java_jdk_internal_vm_VMSupport_initAgentProperties 0000000180007944 f   VMSupport.obj
 0001:0000694c       Java_jdk_internal_misc_VM_getegid 000000018000794c f   VM_md.obj
 0001:0000694c       Java_jdk_internal_misc_VM_geteuid 000000018000794c f   VM_md.obj
 0001:0000694c       Java_jdk_internal_misc_VM_getgid 000000018000794c f   VM_md.obj
 0001:0000694c       Java_jdk_internal_misc_VM_getuid 000000018000794c f   VM_md.obj
 0001:00006954       Java_java_lang_VirtualThread_registerNatives 0000000180007954 f   VirtualThread.obj
 0001:0000696c       Java_sun_io_Win32ErrorMode_setErrorMode 000000018000796c f   Win32ErrorMode.obj
 0001:00006980       Java_sun_security_provider_NativeSeedGenerator_nativeGenerateSeed 0000000180007980 f   WinCAPISeedGenerator.obj
 0001:00006a60       Java_java_io_WinNTFileSystem_canonicalize0 0000000180007a60 f   WinNTFileSystem_md.obj
 0001:00006bd4       Java_java_io_WinNTFileSystem_canonicalizeWithPrefix0 0000000180007bd4 f   WinNTFileSystem_md.obj
 0001:00006d90       Java_java_io_WinNTFileSystem_checkAccess0 0000000180007d90 f   WinNTFileSystem_md.obj
 0001:00006e0c       Java_java_io_WinNTFileSystem_createDirectory0 0000000180007e0c f   WinNTFileSystem_md.obj
 0001:00006e54       Java_java_io_WinNTFileSystem_createFileExclusively0 0000000180007e54 f   WinNTFileSystem_md.obj
 0001:00006f28       Java_java_io_WinNTFileSystem_delete0 0000000180007f28 f   WinNTFileSystem_md.obj
 0001:00006f74       Java_java_io_WinNTFileSystem_getBooleanAttributes0 0000000180007f74 f   WinNTFileSystem_md.obj
 0001:00006fdc       Java_java_io_WinNTFileSystem_getDriveDirectory 0000000180007fdc f   WinNTFileSystem_md.obj
 0001:00007064       Java_java_io_WinNTFileSystem_getFinalPath0 0000000180008064 f   WinNTFileSystem_md.obj
 0001:0000713c       Java_java_io_WinNTFileSystem_getLastModifiedTime0 000000018000813c f   WinNTFileSystem_md.obj
 0001:000071f4       Java_java_io_WinNTFileSystem_getLength0 00000001800081f4 f   WinNTFileSystem_md.obj
 0001:0000736c       Java_java_io_WinNTFileSystem_getNameMax0 000000018000836c f   WinNTFileSystem_md.obj
 0001:00007434       Java_java_io_WinNTFileSystem_getSpace0 0000000180008434 f   WinNTFileSystem_md.obj
 0001:000074f8       Java_java_io_WinNTFileSystem_initIDs 00000001800084f8 f   WinNTFileSystem_md.obj
 0001:00007540       Java_java_io_WinNTFileSystem_list0 0000000180008540 f   WinNTFileSystem_md.obj
 0001:00007884       Java_java_io_WinNTFileSystem_listRoots0 0000000180008884 f   WinNTFileSystem_md.obj
 0001:0000788c       Java_java_io_WinNTFileSystem_rename0 000000018000888c f   WinNTFileSystem_md.obj
 0001:00007920       Java_java_io_WinNTFileSystem_setLastModifiedTime0 0000000180008920 f   WinNTFileSystem_md.obj
 0001:000079ec       Java_java_io_WinNTFileSystem_setPermission0 00000001800089ec f   WinNTFileSystem_md.obj
 0001:00007acc       Java_java_io_WinNTFileSystem_setReadOnly0 0000000180008acc f   WinNTFileSystem_md.obj
 0001:00007bf8       getFinalAttributes         0000000180008bf8 f   WinNTFileSystem_md.obj
 0001:00007cc8       getFinalAttributesIfReparsePoint 0000000180008cc8 f   WinNTFileSystem_md.obj
 0001:0000818c       JDK_Canonicalize           000000018000918c f   canonicalize_md.obj
 0001:00008298       getPrefixed                0000000180009298 f   canonicalize_md.obj
 0001:00008330       lastErrorReportable        0000000180009330 f   canonicalize_md.obj
 0001:0000837c       wcanonicalize              000000018000937c f   canonicalize_md.obj
 0001:000086a0       wcanonicalizeWithPrefix    00000001800096a0 f   canonicalize_md.obj
 0001:00008850       fixClassname               0000000180009850 f   check_classname.obj
 0001:00008b44       verifyClassname            0000000180009b44 f   check_classname.obj
 0001:00008bc8       verifyFixClassname         0000000180009bc8 f   check_classname.obj
 0001:00008c3c       JNI_OnLoad                 0000000180009c3c f   check_version.obj
 0001:00008c44       readBytes                  0000000180009c44 f   io_util.obj
 0001:00008db4       readSingle                 0000000180009db4 f   io_util.obj
 0001:00008e14       throwFileNotFoundException 0000000180009e14 f   io_util.obj
 0001:00008e84       writeBytes                 0000000180009e84 f   io_util.obj
 0001:00009010       writeSingle                000000018000a010 f   io_util.obj
 0001:00009084       currentDir                 000000018000a084 f   io_util_md.obj
 0001:000090ec       currentDirLength           000000018000a0ec f   io_util_md.obj
 0001:00009198       fileDescriptorClose        000000018000a198 f   io_util_md.obj
 0001:00009230       fileOpen                   000000018000a230 f   io_util_md.obj
 0001:000092e0       fileToNTPath               000000018000a2e0 f   io_util_md.obj
 0001:0000930c       getFD                      000000018000a30c f   io_util_md.obj
 0001:0000934c       handleAppend               000000018000a34c f   io_util_md.obj
 0001:00009394       handleAvailable            000000018000a394 f   io_util_md.obj
 0001:00009478       handleGetLength            000000018000a478 f   io_util_md.obj
 0001:0000949c       handleLseek                000000018000a49c f   io_util_md.obj
 0001:000094e4       handleRead                 000000018000a4e4 f   io_util_md.obj
 0001:00009528       handleSetLength            000000018000a528 f   io_util_md.obj
 0001:00009684       handleSync                 000000018000a684 f   io_util_md.obj
 0001:000096a8       handleWrite                000000018000a6a8 f   io_util_md.obj
 0001:000096e0       pathToNTPath               000000018000a6e0 f   io_util_md.obj
 0001:00009840       prefixAbpath               000000018000a840 f   io_util_md.obj
 0001:000098e8       winFileHandleOpen          000000018000a8e8 f   io_util_md.obj
 0001:000099dc       GetJavaProperties          000000018000a9dc f   java_props_md.obj
 0001:0000a0c8       GetStringPlatform          000000018000b0c8 f   java_props_md.obj
 0001:0000a2f8       __local_stdio_scanf_options 000000018000b2f8 f i java_props_md.obj
 0001:0000a3a4       getEncodingFromLangID      000000018000b3a4 f   java_props_md.obj
 0001:0000a5c0       getHomeFromShell32         000000018000b5c0 f   java_props_md.obj
 0001:0000a618       getJavaIDFromLangID        000000018000b618 f   java_props_md.obj
 0001:0000a71c       sscanf                     000000018000b71c f i java_props_md.obj
 0001:0000a768       JDK_LoadSystemLibrary      000000018000b768 f   jdk_util_md.obj
 0001:0000a838       jio_fprintf                000000018000b838 f   jio.obj
 0001:0000a85c       jio_snprintf               000000018000b85c f   jio.obj
 0001:0000a87c       GetStringPlatformChars     000000018000b87c f   jni_util.obj
 0001:0000a87c       JNU_GetStringPlatformChars 000000018000b87c f   jni_util.obj
 0001:0000a884       GetStringPlatformCharsStrict 000000018000b884 f   jni_util.obj
 0001:0000a884       JNU_GetStringPlatformCharsStrict 000000018000b884 f   jni_util.obj
 0001:0000a88c       InitializeEncoding         000000018000b88c f   jni_util.obj
 0001:0000ab5c       JNU_CallMethodByName       000000018000bb5c f   jni_util.obj
 0001:0000ab80       JNU_CallMethodByNameV      000000018000bb80 f   jni_util.obj
 0001:0000adc8       JNU_CallStaticMethodByName 000000018000bdc8 f   jni_util.obj
 0001:0000afbc       JNU_ClassString            000000018000bfbc f   jni_util.obj
 0001:0000b03c       JNU_CopyObjectArray        000000018000c03c f   jni_util.obj
 0001:0000b0dc       JNU_GetEnv                 000000018000c0dc f   jni_util.obj
 0001:0000b0f8       JNU_GetFieldByName         000000018000c0f8 f   jni_util.obj
 0001:0000b2cc       JNU_GetStaticFieldByName   000000018000c2cc f   jni_util.obj
 0001:0000b498       JNU_IsInstanceOfByName     000000018000c498 f   jni_util.obj
 0001:0000b520       JNU_NewObjectByName        000000018000c520 f   jni_util.obj
 0001:0000b5b8       JNU_NewStringPlatform      000000018000c5b8 f   jni_util.obj
 0001:0000b668       JNU_ReleaseStringPlatformChars 000000018000c668 f   jni_util.obj
 0001:0000b674       JNU_SetFieldByName         000000018000c674 f   jni_util.obj
 0001:0000b830       JNU_ThrowArrayIndexOutOfBoundsException 000000018000c830 f   jni_util.obj
 0001:0000b840       JNU_ThrowByName            000000018000c840 f   jni_util.obj
 0001:0000b878       JNU_ThrowByNameWithLastError 000000018000c878 f   jni_util.obj
 0001:0000b8f0       JNU_ThrowByNameWithMessageAndLastError 000000018000c8f0 f   jni_util.obj
 0001:0000ba84       JNU_ThrowClassNotFoundException 000000018000ca84 f   jni_util.obj
 0001:0000ba94       JNU_ThrowIOException       000000018000ca94 f   jni_util.obj
 0001:0000baa4       JNU_ThrowIOExceptionWithLastError 000000018000caa4 f   jni_util.obj
 0001:0000bab4       JNU_ThrowIOExceptionWithMessageAndLastError 000000018000cab4 f   jni_util.obj
 0001:0000bac4       JNU_ThrowIllegalArgumentException 000000018000cac4 f   jni_util.obj
 0001:0000bad4       JNU_ThrowInternalError     000000018000cad4 f   jni_util.obj
 0001:0000bae4       JNU_ThrowNullPointerException 000000018000cae4 f   jni_util.obj
 0001:0000baf4       JNU_ThrowOutOfMemoryError  000000018000caf4 f   jni_util.obj
 0001:0000bb04       JNU_ToString               000000018000cb04 f   jni_util.obj
 0001:0000c874       getErrorString             000000018000d874 f   jni_util_md.obj
 0001:0000c898       getLastErrorString         000000018000d898 f   jni_util_md.obj
 0001:0000c980       getProcessHandle           000000018000d980 f   jni_util_md.obj
 0001:0000c989       JVM_GetArrayLength         000000018000d989 f   jvm:jvm.dll
 0001:0000c98f       JVM_GetArrayElement        000000018000d98f f   jvm:jvm.dll
 0001:0000c995       JVM_GetPrimitiveArrayElement 000000018000d995 f   jvm:jvm.dll
 0001:0000c99b       JVM_SetArrayElement        000000018000d99b f   jvm:jvm.dll
 0001:0000c9a1       JVM_SetPrimitiveArrayElement 000000018000d9a1 f   jvm:jvm.dll
 0001:0000c9a7       JVM_NewArray               000000018000d9a7 f   jvm:jvm.dll
 0001:0000c9ad       JVM_NewMultiArray          000000018000d9ad f   jvm:jvm.dll
 0001:0000c9b3       JVM_GetSystemPackage       000000018000d9b3 f   jvm:jvm.dll
 0001:0000c9b9       JVM_GetSystemPackages      000000018000d9b9 f   jvm:jvm.dll
 0001:0000c9bf       JVM_SetBootLoaderUnnamedModule 000000018000d9bf f   jvm:jvm.dll
 0001:0000c9c5       JVM_InitializeFromArchive  000000018000d9c5 f   jvm:jvm.dll
 0001:0000c9cb       JVM_GetCDSConfigStatus     000000018000d9cb f   jvm:jvm.dll
 0001:0000c9d1       JVM_GetRandomSeedForDumping 000000018000d9d1 f   jvm:jvm.dll
 0001:0000c9d7       JVM_LogLambdaFormInvoker   000000018000d9d7 f   jvm:jvm.dll
 0001:0000c9dd       JVM_DumpClassListToFile    000000018000d9dd f   jvm:jvm.dll
 0001:0000c9e3       JVM_DumpDynamicArchive     000000018000d9e3 f   jvm:jvm.dll
 0001:0000c9e9       JVM_NeedsClassInitBarrierForCDS 000000018000d9e9 f   jvm:jvm.dll
 0001:0000c9ef       JVM_DefineArchivedModules  000000018000d9ef f   jvm:jvm.dll
 0001:0000c9f5       JVM_InitClassName          000000018000d9f5 f   jvm:jvm.dll
 0001:0000c9fb       JVM_GetClassInterfaces     000000018000d9fb f   jvm:jvm.dll
 0001:0000ca01       JVM_IsHiddenClass          000000018000da01 f   jvm:jvm.dll
 0001:0000ca07       JVM_GetDeclaredClasses     000000018000da07 f   jvm:jvm.dll
 0001:0000ca0d       JVM_GetDeclaringClass      000000018000da0d f   jvm:jvm.dll
 0001:0000ca13       JVM_GetSimpleBinaryName    000000018000da13 f   jvm:jvm.dll
 0001:0000ca19       JVM_GetClassSignature      000000018000da19 f   jvm:jvm.dll
 0001:0000ca1f       JVM_GetClassAnnotations    000000018000da1f f   jvm:jvm.dll
 0001:0000ca25       JVM_GetClassTypeAnnotations 000000018000da25 f   jvm:jvm.dll
 0001:0000ca2b       JVM_GetClassDeclaredMethods 000000018000da2b f   jvm:jvm.dll
 0001:0000ca31       JVM_GetClassDeclaredFields 000000018000da31 f   jvm:jvm.dll
 0001:0000ca37       JVM_GetClassDeclaredConstructors 000000018000da37 f   jvm:jvm.dll
 0001:0000ca3d       JVM_GetClassAccessFlags    000000018000da3d f   jvm:jvm.dll
 0001:0000ca43       JVM_GetNestHost            000000018000da43 f   jvm:jvm.dll
 0001:0000ca49       JVM_GetNestMembers         000000018000da49 f   jvm:jvm.dll
 0001:0000ca4f       JVM_IsRecord               000000018000da4f f   jvm:jvm.dll
 0001:0000ca55       JVM_GetRecordComponents    000000018000da55 f   jvm:jvm.dll
 0001:0000ca5b       JVM_GetPermittedSubclasses 000000018000da5b f   jvm:jvm.dll
 0001:0000ca61       JVM_GetClassConstantPool   000000018000da61 f   jvm:jvm.dll
 0001:0000ca67       JVM_DesiredAssertionStatus 000000018000da67 f   jvm:jvm.dll
 0001:0000ca6d       JVM_GetEnclosingMethodInfo 000000018000da6d f   jvm:jvm.dll
 0001:0000ca73       JVM_GetClassFileVersion    000000018000da73 f   jvm:jvm.dll
 0001:0000ca79       JVM_FindPrimitiveClass     000000018000da79 f   jvm:jvm.dll
 0001:0000ca7f       JVM_FindClassFromCaller    000000018000da7f f   jvm:jvm.dll
 0001:0000ca85       JVM_AssertionStatusDirectives 000000018000da85 f   jvm:jvm.dll
 0001:0000ca8b       JVM_FindClassFromBootLoader 000000018000da8b f   jvm:jvm.dll
 0001:0000ca91       JVM_FindLoadedClass        000000018000da91 f   jvm:jvm.dll
 0001:0000ca97       JVM_DefineClassWithSource  000000018000da97 f   jvm:jvm.dll
 0001:0000ca9d       JVM_LookupDefineClass      000000018000da9d f   jvm:jvm.dll
 0001:0000caa3       JVM_ConstantPoolGetSize    000000018000daa3 f   jvm:jvm.dll
 0001:0000caa9       JVM_ConstantPoolGetClassAt 000000018000daa9 f   jvm:jvm.dll
 0001:0000caaf       JVM_ConstantPoolGetClassAtIfLoaded 000000018000daaf f   jvm:jvm.dll
 0001:0000cab5       JVM_ConstantPoolGetClassRefIndexAt 000000018000dab5 f   jvm:jvm.dll
 0001:0000cabb       JVM_ConstantPoolGetMethodAt 000000018000dabb f   jvm:jvm.dll
 0001:0000cac1       JVM_ConstantPoolGetMethodAtIfLoaded 000000018000dac1 f   jvm:jvm.dll
 0001:0000cac7       JVM_ConstantPoolGetFieldAt 000000018000dac7 f   jvm:jvm.dll
 0001:0000cacd       JVM_ConstantPoolGetFieldAtIfLoaded 000000018000dacd f   jvm:jvm.dll
 0001:0000cad3       JVM_ConstantPoolGetMemberRefInfoAt 000000018000dad3 f   jvm:jvm.dll
 0001:0000cad9       JVM_ConstantPoolGetNameAndTypeRefIndexAt 000000018000dad9 f   jvm:jvm.dll
 0001:0000cadf       JVM_ConstantPoolGetNameAndTypeRefInfoAt 000000018000dadf f   jvm:jvm.dll
 0001:0000cae5       JVM_ConstantPoolGetIntAt   000000018000dae5 f   jvm:jvm.dll
 0001:0000caeb       JVM_ConstantPoolGetLongAt  000000018000daeb f   jvm:jvm.dll
 0001:0000caf1       JVM_ConstantPoolGetFloatAt 000000018000daf1 f   jvm:jvm.dll
 0001:0000caf7       JVM_ConstantPoolGetDoubleAt 000000018000daf7 f   jvm:jvm.dll
 0001:0000cafd       JVM_ConstantPoolGetStringAt 000000018000dafd f   jvm:jvm.dll
 0001:0000cb03       JVM_ConstantPoolGetUTF8At  000000018000db03 f   jvm:jvm.dll
 0001:0000cb09       JVM_ConstantPoolGetTagAt   000000018000db09 f   jvm:jvm.dll
 0001:0000cb0f       JVM_RegisterContinuationMethods 000000018000db0f f   jvm:jvm.dll
 0001:0000cb15       JVM_IsContinuationsSupported 000000018000db15 f   jvm:jvm.dll
 0001:0000cb1b       JVM_GetMethodTypeAnnotations 000000018000db1b f   jvm:jvm.dll
 0001:0000cb21       JVM_GetMethodParameters    000000018000db21 f   jvm:jvm.dll
 0001:0000cb27       JVM_GetFieldTypeAnnotations 000000018000db27 f   jvm:jvm.dll
 0001:0000cb2d       JVM_ReportFinalizationComplete 000000018000db2d f   jvm:jvm.dll
 0001:0000cb33       JVM_IsFinalizationEnabled  000000018000db33 f   jvm:jvm.dll
 0001:0000cb39       JVM_IsForeignLinkerSupported 000000018000db39 f   jvm:jvm.dll
 0001:0000cb3f       JVM_RegisterLambdaProxyClassForArchiving 000000018000db3f f   jvm:jvm.dll
 0001:0000cb45       JVM_LookupLambdaProxyClassFromArchive 000000018000db45 f   jvm:jvm.dll
 0001:0000cb4b       JVM_DefineModule           000000018000db4b f   jvm:jvm.dll
 0001:0000cb51       JVM_AddModuleExports       000000018000db51 f   jvm:jvm.dll
 0001:0000cb57       JVM_AddModuleExportsToAllUnnamed 000000018000db57 f   jvm:jvm.dll
 0001:0000cb5d       JVM_AddModuleExportsToAll  000000018000db5d f   jvm:jvm.dll
 0001:0000cb63       JVM_AddReadsModule         000000018000db63 f   jvm:jvm.dll
 0001:0000cb69       JVM_InvokeMethod           000000018000db69 f   jvm:jvm.dll
 0001:0000cb6f       JVM_NewInstanceFromConstructor 000000018000db6f f   jvm:jvm.dll
 0001:0000cb75       JVM_LoadLibrary            000000018000db75 f   jvm:jvm.dll
 0001:0000cb7b       JVM_UnloadLibrary          000000018000db7b f   jvm:jvm.dll
 0001:0000cb81       JVM_FindLibraryEntry       000000018000db81 f   jvm:jvm.dll
 0001:0000cb87       JVM_IsSupportedJNIVersion  000000018000db87 f   jvm:jvm.dll
 0001:0000cb8d       JVM_GetExtendedNPEMessage  000000018000db8d f   jvm:jvm.dll
 0001:0000cb93       JVM_ReferenceClear         000000018000db93 f   jvm:jvm.dll
 0001:0000cb99       JVM_PhantomReferenceRefersTo 000000018000db99 f   jvm:jvm.dll
 0001:0000cb9f       JVM_IsPreviewEnabled       000000018000db9f f   jvm:jvm.dll
 0001:0000cba5       JVM_GetThreadInterruptEvent 000000018000dba5 f   jvm:jvm.dll
 0001:0000cbab       JVM_GetAndClearReferencePendingList 000000018000dbab f   jvm:jvm.dll
 0001:0000cbb1       JVM_HasReferencePendingList 000000018000dbb1 f   jvm:jvm.dll
 0001:0000cbb7       JVM_WaitForReferencePendingList 000000018000dbb7 f   jvm:jvm.dll
 0001:0000cbbd       JVM_ReferenceRefersTo      000000018000dbbd f   jvm:jvm.dll
 0001:0000cbc3       JVM_GetCallerClass         000000018000dbc3 f   jvm:jvm.dll
 0001:0000cbc9       JVM_AreNestMates           000000018000dbc9 f   jvm:jvm.dll
 0001:0000cbcf       JVM_GC                     000000018000dbcf f   jvm:jvm.dll
 0001:0000cbd5       JVM_TotalMemory            000000018000dbd5 f   jvm:jvm.dll
 0001:0000cbdb       JVM_FreeMemory             000000018000dbdb f   jvm:jvm.dll
 0001:0000cbe1       JVM_MaxMemory              000000018000dbe1 f   jvm:jvm.dll
 0001:0000cbe7       JVM_ActiveProcessorCount   000000018000dbe7 f   jvm:jvm.dll
 0001:0000cbed       JVM_BeforeHalt             000000018000dbed f   jvm:jvm.dll
 0001:0000cbf3       JVM_Halt                   000000018000dbf3 f   jvm:jvm.dll
 0001:0000cbf9       JVM_RegisterSignal         000000018000dbf9 f   jvm:jvm.dll
 0001:0000cbff       JVM_RaiseSignal            000000018000dbff f   jvm:jvm.dll
 0001:0000cc05       JVM_FindSignal             000000018000dc05 f   jvm:jvm.dll
 0001:0000cc0b       JVM_ExpandStackFrameInfo   000000018000dc0b f   jvm:jvm.dll
 0001:0000cc11       JVM_CallStackWalk          000000018000dc11 f   jvm:jvm.dll
 0001:0000cc17       JVM_MoreStackWalk          000000018000dc17 f   jvm:jvm.dll
 0001:0000cc1d       JVM_SetStackWalkContinuation 000000018000dc1d f   jvm:jvm.dll
 0001:0000cc23       JVM_InitStackTraceElementArray 000000018000dc23 f   jvm:jvm.dll
 0001:0000cc29       JVM_InitStackTraceElement  000000018000dc29 f   jvm:jvm.dll
 0001:0000cc2f       JVM_InternString           000000018000dc2f f   jvm:jvm.dll
 0001:0000cc35       JVM_CurrentTimeMillis      000000018000dc35 f   jvm:jvm.dll
 0001:0000cc3b       JVM_NanoTime               000000018000dc3b f   jvm:jvm.dll
 0001:0000cc41       JVM_ArrayCopy              000000018000dc41 f   jvm:jvm.dll
 0001:0000cc47       JVM_IHashCode              000000018000dc47 f   jvm:jvm.dll
 0001:0000cc4d       JVM_GetProperties          000000018000dc4d f   jvm:jvm.dll
 0001:0000cc53       JVM_StartThread            000000018000dc53 f   jvm:jvm.dll
 0001:0000cc59       JVM_SetThreadPriority      000000018000dc59 f   jvm:jvm.dll
 0001:0000cc5f       JVM_Yield                  000000018000dc5f f   jvm:jvm.dll
 0001:0000cc65       JVM_SleepNanos             000000018000dc65 f   jvm:jvm.dll
 0001:0000cc6b       JVM_CurrentCarrierThread   000000018000dc6b f   jvm:jvm.dll
 0001:0000cc71       JVM_CurrentThread          000000018000dc71 f   jvm:jvm.dll
 0001:0000cc77       JVM_SetCurrentThread       000000018000dc77 f   jvm:jvm.dll
 0001:0000cc7d       JVM_Interrupt              000000018000dc7d f   jvm:jvm.dll
 0001:0000cc83       JVM_HoldsLock              000000018000dc83 f   jvm:jvm.dll
 0001:0000cc89       JVM_GetStackTrace          000000018000dc89 f   jvm:jvm.dll
 0001:0000cc8f       JVM_GetAllThreads          000000018000dc8f f   jvm:jvm.dll
 0001:0000cc95       JVM_SetNativeThreadName    000000018000dc95 f   jvm:jvm.dll
 0001:0000cc9b       JVM_DumpThreads            000000018000dc9b f   jvm:jvm.dll
 0001:0000cca1       JVM_ScopedValueCache       000000018000dca1 f   jvm:jvm.dll
 0001:0000cca7       JVM_SetScopedValueCache    000000018000dca7 f   jvm:jvm.dll
 0001:0000ccad       JVM_FindScopedValueBindings 000000018000dcad f   jvm:jvm.dll
 0001:0000ccb3       JVM_GetNextThreadIdOffset  000000018000dcb3 f   jvm:jvm.dll
 0001:0000ccb9       JVM_EnsureMaterializedForStackWalk_func 000000018000dcb9 f   jvm:jvm.dll
 0001:0000ccbf       JVM_CreateThreadSnapshot   000000018000dcbf f   jvm:jvm.dll
 0001:0000ccc5       JVM_FillInStackTrace       000000018000dcc5 f   jvm:jvm.dll
 0001:0000cccb       JVM_GetNanoTimeAdjustment  000000018000dccb f   jvm:jvm.dll
 0001:0000ccd1       JVM_GetVmArguments         000000018000dcd1 f   jvm:jvm.dll
 0001:0000ccd7       JVM_LatestUserDefinedLoader 000000018000dcd7 f   jvm:jvm.dll
 0001:0000ccdd       JVM_InitAgentProperties    000000018000dcdd f   jvm:jvm.dll
 0001:0000cce3       JVM_GetTemporaryDirectory  000000018000dce3 f   jvm:jvm.dll
 0001:0000cce9       JVM_VirtualThreadStart     000000018000dce9 f   jvm:jvm.dll
 0001:0000ccef       JVM_VirtualThreadEnd       000000018000dcef f   jvm:jvm.dll
 0001:0000ccf5       JVM_VirtualThreadMount     000000018000dcf5 f   jvm:jvm.dll
 0001:0000ccfb       JVM_VirtualThreadUnmount   000000018000dcfb f   jvm:jvm.dll
 0001:0000cd01       JVM_VirtualThreadDisableSuspend 000000018000dd01 f   jvm:jvm.dll
 0001:0000cd07       JVM_VirtualThreadPinnedEvent 000000018000dd07 f   jvm:jvm.dll
 0001:0000cd0d       JVM_TakeVirtualThreadListToUnblock 000000018000dd0d f   jvm:jvm.dll
 0001:0000cd13       jio_vsnprintf              000000018000dd13 f   jvm:jvm.dll
 0001:0000cd19       jio_vfprintf               000000018000dd19 f   jvm:jvm.dll
 0001:0000cd1f       ConvertSidToStringSidW     000000018000dd1f f   advapi32:ADVAPI32.dll
 0001:0000cd25       SHGetKnownFolderPath       000000018000dd25 f   shell32:SHELL32.dll
 0001:0000cd2b       GetFileVersionInfoSizeW    000000018000dd2b f   version:VERSION.dll
 0001:0000cd31       GetFileVersionInfoW        000000018000dd31 f   version:VERSION.dll
 0001:0000cd37       VerQueryValueW             000000018000dd37 f   version:VERSION.dll
 0001:0000cd40       __GSHandlerCheck           000000018000dd40 f   MSVCRT:gshandler.obj
 0001:0000cd60       __GSHandlerCheckCommon     000000018000dd60 f   MSVCRT:gshandler.obj
 0001:0000cdd0       __security_check_cookie    000000018000ddd0 f   MSVCRT:amdsecgs.obj
 0001:0000cdf0       __raise_securityfailure    000000018000ddf0 f   MSVCRT:gs_report.obj
 0001:0000ce24       __report_gsfailure         000000018000de24 f   MSVCRT:gs_report.obj
 0001:0000cef8       __report_rangecheckfailure 000000018000def8 f   MSVCRT:gs_report.obj
 0001:0000cf0c       __report_securityfailure   000000018000df0c f   MSVCRT:gs_report.obj
 0001:0000d0a0       __chkstk                   000000018000e0a0 f   MSVCRT:chkstk.obj
 0001:0000d0a0       _alloca_probe              000000018000e0a0 f   MSVCRT:chkstk.obj
 0001:0000d400       _DllMainCRTStartup         000000018000e400 f   MSVCRT:dll_dllmain.obj
 0001:0000d440       __security_init_cookie     000000018000e440 f   MSVCRT:gs_support.obj
 0001:0000d4ec       DllMain                    000000018000e4ec f   MSVCRT:dll_dllmain_stub.obj
 0001:0000d510       ?__scrt_initialize_type_info@@YAXXZ 000000018000e510 f   MSVCRT:tncleanup.obj
 0001:0000d520       ?__scrt_uninitialize_type_info@@YAXXZ 000000018000e520 f   MSVCRT:tncleanup.obj
 0001:0000d52c       __scrt_initialize_default_local_stdio_options 000000018000e52c f   MSVCRT:default_local_stdio_options.obj
 0001:0000d548       __scrt_acquire_startup_lock 000000018000e548 f   MSVCRT:utility.obj
 0001:0000d584       __scrt_dllmain_after_initialize_c 000000018000e584 f   MSVCRT:utility.obj
 0001:0000d5b8       __scrt_dllmain_before_initialize_c 000000018000e5b8 f   MSVCRT:utility.obj
 0001:0000d5d0       __scrt_dllmain_crt_thread_attach 000000018000e5d0 f   MSVCRT:utility.obj
 0001:0000d5f8       __scrt_dllmain_crt_thread_detach 000000018000e5f8 f   MSVCRT:utility.obj
 0001:0000d610       __scrt_dllmain_exception_filter 000000018000e610 f   MSVCRT:utility.obj
 0001:0000d670       __scrt_dllmain_uninitialize_c 000000018000e670 f   MSVCRT:utility.obj
 0001:0000d6a0       __scrt_dllmain_uninitialize_critical 000000018000e6a0 f   MSVCRT:utility.obj
 0001:0000d6b4       __scrt_initialize_crt      000000018000e6b4 f   MSVCRT:utility.obj
 0001:0000d6f0       __scrt_initialize_onexit_tables 000000018000e6f0 f   MSVCRT:utility.obj
 0001:0000d77c       __scrt_is_nonwritable_in_current_image 000000018000e77c f   MSVCRT:utility.obj
 0001:0000d814       __scrt_release_startup_lock 000000018000e814 f   MSVCRT:utility.obj
 0001:0000d838       __scrt_uninitialize_crt    000000018000e838 f   MSVCRT:utility.obj
 0001:0000d864       __scrt_get_dyn_tls_init_callback 000000018000e864 f   MSVCRT:dyn_tls_init.obj
 0001:0000d86c       __crt_debugger_hook        000000018000e86c f   MSVCRT:utility_desktop.obj
 0001:0000d874       __scrt_fastfail            000000018000e874 f   MSVCRT:utility_desktop.obj
 0001:0000d9bc       _RTC_Initialize            000000018000e9bc f   MSVCRT:initsect.obj
 0001:0000d9f8       _RTC_Terminate             000000018000e9f8 f   MSVCRT:initsect.obj
 0001:0000da34       __isa_available_init       000000018000ea34 f   MSVCRT:cpu_disp.obj
 0001:0000dd00       _get_startup_argv_mode     000000018000ed00 f   MSVCRT:argv_mode.obj
 0001:0000dd08       __scrt_is_ucrt_dll_in_use  000000018000ed08 f   MSVCRT:ucrt_detection.obj
 0001:0000dd20       CreateToolhelp32Snapshot   000000018000ed20 f   kernel32:KERNEL32.dll
 0001:0000dd26       Process32First             000000018000ed26 f   kernel32:KERNEL32.dll
 0001:0000dd2c       Process32Next              000000018000ed2c f   kernel32:KERNEL32.dll
 0001:0000dd32       memcpy                     000000018000ed32 f   vcruntime:VCRUNTIME140.dll
 0001:0000dd38       memset                     000000018000ed38 f   vcruntime:VCRUNTIME140.dll
 0001:0000dd3e       memcmp                     000000018000ed3e f   vcruntime:VCRUNTIME140.dll
 0001:0000dd44       memmove                    000000018000ed44 f   vcruntime:VCRUNTIME140.dll
 0001:0000dd4a       wcsrchr                    000000018000ed4a f   vcruntime:VCRUNTIME140.dll
 0001:0000dd50       wcschr                     000000018000ed50 f   vcruntime:VCRUNTIME140.dll
 0001:0000dd56       __C_specific_handler       000000018000ed56 f   vcruntime:VCRUNTIME140.dll
 0001:0000dd5c       __std_type_info_destroy_list 000000018000ed5c f   vcruntime:VCRUNTIME140.dll
 0001:0000dd62       strcat                     000000018000ed62 f   ucrt:api-ms-win-crt-string-l1-1-0.dll
 0001:0000dd68       strcpy                     000000018000ed68 f   ucrt:api-ms-win-crt-string-l1-1-0.dll
 0001:0000dd6e       strlen                     000000018000ed6e f   ucrt:api-ms-win-crt-string-l1-1-0.dll
 0001:0000dd74       strcmp                     000000018000ed74 f   ucrt:api-ms-win-crt-string-l1-1-0.dll
 0001:0000dd7a       _initterm                  000000018000ed7a f   ucrt:api-ms-win-crt-runtime-l1-1-0.dll
 0001:0000dd80       _initterm_e                000000018000ed80 f   ucrt:api-ms-win-crt-runtime-l1-1-0.dll
 0001:0000dd86       _seh_filter_dll            000000018000ed86 f   ucrt:api-ms-win-crt-runtime-l1-1-0.dll
 0001:0000dd8c       _configure_narrow_argv     000000018000ed8c f   ucrt:api-ms-win-crt-runtime-l1-1-0.dll
 0001:0000dd92       _initialize_narrow_environment 000000018000ed92 f   ucrt:api-ms-win-crt-runtime-l1-1-0.dll
 0001:0000dd98       _initialize_onexit_table   000000018000ed98 f   ucrt:api-ms-win-crt-runtime-l1-1-0.dll
 0001:0000dd9e       _execute_onexit_table      000000018000ed9e f   ucrt:api-ms-win-crt-runtime-l1-1-0.dll
 0001:0000dda4       _cexit                     000000018000eda4 f   ucrt:api-ms-win-crt-runtime-l1-1-0.dll
 0001:0000ddac       __scrt_stub_for_is_c_termination_complete 000000018000edac f   MSVCRT:ucrt_stubs.obj
 0001:0000ddac       _is_c_termination_complete 000000018000edac f   MSVCRT:ucrt_stubs.obj
 0001:0000ddc0       _guard_dispatch_icall_nop  000000018000edc0 f   MSVCRT:guard_dispatch.obj
 0001:0000dde0       _guard_xfg_dispatch_icall_nop 000000018000ede0 f   MSVCRT:guard_xfg_dispatch.obj
 0002:00000000       __imp_OpenProcessToken     000000018000f000     advapi32:ADVAPI32.dll
 0002:00000008       __imp_GetTokenInformation  000000018000f008     advapi32:ADVAPI32.dll
 0002:00000010       __imp_LookupAccountSidW    000000018000f010     advapi32:ADVAPI32.dll
 0002:00000018       __imp_ConvertSidToStringSidW 000000018000f018     advapi32:ADVAPI32.dll
 0002:00000020       __imp_RegCloseKey          000000018000f020     advapi32:ADVAPI32.dll
 0002:00000028       __imp_RegEnumKeyExA        000000018000f028     advapi32:ADVAPI32.dll
 0002:00000030       __imp_RegOpenKeyExA        000000018000f030     advapi32:ADVAPI32.dll
 0002:00000038       __imp_RegOpenKeyExW        000000018000f038     advapi32:ADVAPI32.dll
 0002:00000040       __imp_RegQueryInfoKeyA     000000018000f040     advapi32:ADVAPI32.dll
 0002:00000048       __imp_RegQueryValueExA     000000018000f048     advapi32:ADVAPI32.dll
 0002:00000050       __imp_RegQueryValueExW     000000018000f050     advapi32:ADVAPI32.dll
 0002:00000058       __imp_CryptAcquireContextA 000000018000f058     advapi32:ADVAPI32.dll
 0002:00000060       __imp_CryptReleaseContext  000000018000f060     advapi32:ADVAPI32.dll
 0002:00000068       __imp_CryptGenRandom       000000018000f068     advapi32:ADVAPI32.dll
 0002:00000070       __imp_GetUserNameW         000000018000f070     advapi32:ADVAPI32.dll
 0002:00000078       \177ADVAPI32_NULL_THUNK_DATA 000000018000f078     advapi32:ADVAPI32.dll
 0002:00000080       __imp_GetStdHandle         000000018000f080     kernel32:KERNEL32.dll
 0002:00000088       __imp_GetFileType          000000018000f088     kernel32:KERNEL32.dll
 0002:00000090       __imp_CloseHandle          000000018000f090     kernel32:KERNEL32.dll
 0002:00000098       __imp_GetModuleHandleA     000000018000f098     kernel32:KERNEL32.dll
 0002:000000a0       __imp_IsDebuggerPresent    000000018000f0a0     kernel32:KERNEL32.dll
 0002:000000a8       __imp_InitializeSListHead  000000018000f0a8     kernel32:KERNEL32.dll
 0002:000000b0       __imp_DisableThreadLibraryCalls 000000018000f0b0     kernel32:KERNEL32.dll
 0002:000000b8       __imp_GetSystemTimeAsFileTime 000000018000f0b8     kernel32:KERNEL32.dll
 0002:000000c0       __imp_GetCurrentThreadId   000000018000f0c0     kernel32:KERNEL32.dll
 0002:000000c8       __imp_QueryPerformanceCounter 000000018000f0c8     kernel32:KERNEL32.dll
 0002:000000d0       __imp_GetCurrentProcess    000000018000f0d0     kernel32:KERNEL32.dll
 0002:000000d8       __imp_SetUnhandledExceptionFilter 000000018000f0d8     kernel32:KERNEL32.dll
 0002:000000e0       __imp_UnhandledExceptionFilter 000000018000f0e0     kernel32:KERNEL32.dll
 0002:000000e8       __imp_RtlVirtualUnwind     000000018000f0e8     kernel32:KERNEL32.dll
 0002:000000f0       __imp_RtlLookupFunctionEntry 000000018000f0f0     kernel32:KERNEL32.dll
 0002:000000f8       __imp_RtlCaptureContext    000000018000f0f8     kernel32:KERNEL32.dll
 0002:00000100       __imp_LoadLibraryA         000000018000f100     kernel32:KERNEL32.dll
 0002:00000108       __imp_GetSystemDirectoryA  000000018000f108     kernel32:KERNEL32.dll
 0002:00000110       __imp_GetConsoleOutputCP   000000018000f110     kernel32:KERNEL32.dll
 0002:00000118       __imp_GetConsoleCP         000000018000f118     kernel32:KERNEL32.dll
 0002:00000120       __imp_GetACP               000000018000f120     kernel32:KERNEL32.dll
 0002:00000128       __imp_IsValidCodePage      000000018000f128     kernel32:KERNEL32.dll
 0002:00000130       __imp_GetNativeSystemInfo  000000018000f130     kernel32:KERNEL32.dll
 0002:00000138       __imp_GetVersionExA        000000018000f138     kernel32:KERNEL32.dll
 0002:00000140       __imp_GetWindowsDirectoryA 000000018000f140     kernel32:KERNEL32.dll
 0002:00000148       __imp_GetSystemDirectoryW  000000018000f148     kernel32:KERNEL32.dll
 0002:00000150       __imp_GetSystemInfo        000000018000f150     kernel32:KERNEL32.dll
 0002:00000158       __imp_IsProcessorFeaturePresent 000000018000f158     kernel32:KERNEL32.dll
 0002:00000160       __imp_GetTempPathW         000000018000f160     kernel32:KERNEL32.dll
 0002:00000168       __imp_GetCurrentDirectoryW 000000018000f168     kernel32:KERNEL32.dll
 0002:00000170       __imp_PeekConsoleInputA    000000018000f170     kernel32:KERNEL32.dll
 0002:00000178       __imp_GetNumberOfConsoleInputEvents 000000018000f178     kernel32:KERNEL32.dll
 0002:00000180       __imp_PeekNamedPipe        000000018000f180     kernel32:KERNEL32.dll
 0002:00000188       __imp_WriteFile            000000018000f188     kernel32:KERNEL32.dll
 0002:00000190       __imp_SetFilePointerEx     000000018000f190     kernel32:KERNEL32.dll
 0002:00000198       __imp_SetFileInformationByHandle 000000018000f198     kernel32:KERNEL32.dll
 0002:000001a0       __imp_ReadFile             000000018000f1a0     kernel32:KERNEL32.dll
 0002:000001a8       __imp_GetFileSizeEx        000000018000f1a8     kernel32:KERNEL32.dll
 0002:000001b0       __imp_GetDriveTypeW        000000018000f1b0     kernel32:KERNEL32.dll
 0002:000001b8       __imp_FlushFileBuffers     000000018000f1b8     kernel32:KERNEL32.dll
 0002:000001c0       __imp_DeviceIoControl      000000018000f1c0     kernel32:KERNEL32.dll
 0002:000001c8       __imp_SetLastError         000000018000f1c8     kernel32:KERNEL32.dll
 0002:000001d0       __imp_SetFileTime          000000018000f1d0     kernel32:KERNEL32.dll
 0002:000001d8       __imp_SetFileAttributesW   000000018000f1d8     kernel32:KERNEL32.dll
 0002:000001e0       __imp_RemoveDirectoryW     000000018000f1e0     kernel32:KERNEL32.dll
 0002:000001e8       __imp_GetVolumePathNameW   000000018000f1e8     kernel32:KERNEL32.dll
 0002:000001f0       __imp_GetVolumeInformationW 000000018000f1f0     kernel32:KERNEL32.dll
 0002:000001f8       __imp_GetLogicalDrives     000000018000f1f8     kernel32:KERNEL32.dll
 0002:00000200       __imp_GetFullPathNameW     000000018000f200     kernel32:KERNEL32.dll
 0002:00000208       __imp_GetFileTime          000000018000f208     kernel32:KERNEL32.dll
 0002:00000210       __imp_GetFinalPathNameByHandleW 000000018000f210     kernel32:KERNEL32.dll
 0002:00000218       __imp_GetFileInformationByHandle 000000018000f218     kernel32:KERNEL32.dll
 0002:00000220       __imp_GetFileAttributesExW 000000018000f220     kernel32:KERNEL32.dll
 0002:00000228       __imp_GetFileAttributesW   000000018000f228     kernel32:KERNEL32.dll
 0002:00000230       __imp_GetDiskFreeSpaceExW  000000018000f230     kernel32:KERNEL32.dll
 0002:00000238       __imp_FindNextFileW        000000018000f238     kernel32:KERNEL32.dll
 0002:00000240       __imp_FindFirstFileW       000000018000f240     kernel32:KERNEL32.dll
 0002:00000248       __imp_FindClose            000000018000f248     kernel32:KERNEL32.dll
 0002:00000250       __imp_DeleteFileW          000000018000f250     kernel32:KERNEL32.dll
 0002:00000258       __imp_CreateDirectoryW     000000018000f258     kernel32:KERNEL32.dll
 0002:00000260       __imp_SetErrorMode         000000018000f260     kernel32:KERNEL32.dll
 0002:00000268       __imp_GetUserGeoID         000000018000f268     kernel32:KERNEL32.dll
 0002:00000270       __imp_GetGeoInfoA          000000018000f270     kernel32:KERNEL32.dll
 0002:00000278       __imp_GetLocaleInfoA       000000018000f278     kernel32:KERNEL32.dll
 0002:00000280       __imp_MultiByteToWideChar  000000018000f280     kernel32:KERNEL32.dll
 0002:00000288       __imp_GetDynamicTimeZoneInformation 000000018000f288     kernel32:KERNEL32.dll
 0002:00000290       __imp_GetTimeZoneInformation 000000018000f290     kernel32:KERNEL32.dll
 0002:00000298       __imp_ResetEvent           000000018000f298     kernel32:KERNEL32.dll
 0002:000002a0       __imp_GetConsoleWindow     000000018000f2a0     kernel32:KERNEL32.dll
 0002:000002a8       __imp_WideCharToMultiByte  000000018000f2a8     kernel32:KERNEL32.dll
 0002:000002b0       __imp_FormatMessageW       000000018000f2b0     kernel32:KERNEL32.dll
 0002:000002b8       __imp_GetProcessId         000000018000f2b8     kernel32:KERNEL32.dll
 0002:000002c0       __imp_CreateProcessW       000000018000f2c0     kernel32:KERNEL32.dll
 0002:000002c8       __imp_WaitForMultipleObjects 000000018000f2c8     kernel32:KERNEL32.dll
 0002:000002d0       __imp_CreatePipe           000000018000f2d0     kernel32:KERNEL32.dll
 0002:000002d8       __imp_SetHandleInformation 000000018000f2d8     kernel32:KERNEL32.dll
 0002:000002e0       __imp_GetHandleInformation 000000018000f2e0     kernel32:KERNEL32.dll
 0002:000002e8       __imp_CreateFileW          000000018000f2e8     kernel32:KERNEL32.dll
 0002:000002f0       __imp_Process32Next        000000018000f2f0     kernel32:KERNEL32.dll
 0002:000002f8       __imp_Process32First       000000018000f2f8     kernel32:KERNEL32.dll
 0002:00000300       __imp_CreateToolhelp32Snapshot 000000018000f300     kernel32:KERNEL32.dll
 0002:00000308       __imp_QueryFullProcessImageNameW 000000018000f308     kernel32:KERNEL32.dll
 0002:00000310       __imp_LocalFree            000000018000f310     kernel32:KERNEL32.dll
 0002:00000318       __imp_OpenProcess          000000018000f318     kernel32:KERNEL32.dll
 0002:00000320       __imp_GetExitCodeProcess   000000018000f320     kernel32:KERNEL32.dll
 0002:00000328       __imp_TerminateProcess     000000018000f328     kernel32:KERNEL32.dll
 0002:00000330       __imp_GetCurrentProcessId  000000018000f330     kernel32:KERNEL32.dll
 0002:00000338       __imp_GetProcessTimes      000000018000f338     kernel32:KERNEL32.dll
 0002:00000340       __imp_WaitForSingleObject  000000018000f340     kernel32:KERNEL32.dll
 0002:00000348       __imp_GetLastError         000000018000f348     kernel32:KERNEL32.dll
 0002:00000350       __imp_FreeEnvironmentStringsW 000000018000f350     kernel32:KERNEL32.dll
 0002:00000358       __imp_GetEnvironmentStringsW 000000018000f358     kernel32:KERNEL32.dll
 0002:00000360       __imp_SetConsoleMode       000000018000f360     kernel32:KERNEL32.dll
 0002:00000368       __imp_GetConsoleMode       000000018000f368     kernel32:KERNEL32.dll
 0002:00000370       __imp_GetUserDefaultLCID   000000018000f370     kernel32:KERNEL32.dll
 0002:00000378       __imp_GetUserDefaultUILanguage 000000018000f378     kernel32:KERNEL32.dll
 0002:00000380       __imp_GetProcAddress       000000018000f380     kernel32:KERNEL32.dll
 0002:00000388       \177KERNEL32_NULL_THUNK_DATA 000000018000f388     kernel32:KERNEL32.dll
 0002:00000390       __imp_SHGetKnownFolderPath 000000018000f390     shell32:SHELL32.dll
 0002:00000398       \177SHELL32_NULL_THUNK_DATA 000000018000f398     shell32:SHELL32.dll
 0002:000003a0       __imp___std_type_info_destroy_list 000000018000f3a0     vcruntime:VCRUNTIME140.dll
 0002:000003a8       __imp_memcpy               000000018000f3a8     vcruntime:VCRUNTIME140.dll
 0002:000003b0       __imp_memcmp               000000018000f3b0     vcruntime:VCRUNTIME140.dll
 0002:000003b8       __imp_memset               000000018000f3b8     vcruntime:VCRUNTIME140.dll
 0002:000003c0       __imp_wcschr               000000018000f3c0     vcruntime:VCRUNTIME140.dll
 0002:000003c8       __imp_memmove              000000018000f3c8     vcruntime:VCRUNTIME140.dll
 0002:000003d0       __imp_wcsrchr              000000018000f3d0     vcruntime:VCRUNTIME140.dll
 0002:000003d8       __imp___C_specific_handler 000000018000f3d8     vcruntime:VCRUNTIME140.dll
 0002:000003e0       \177VCRUNTIME140_NULL_THUNK_DATA 000000018000f3e0     vcruntime:VCRUNTIME140.dll
 0002:000003e8       __imp_VerQueryValueW       000000018000f3e8     version:VERSION.dll
 0002:000003f0       __imp_GetFileVersionInfoW  000000018000f3f0     version:VERSION.dll
 0002:000003f8       __imp_GetFileVersionInfoSizeW 000000018000f3f8     version:VERSION.dll
 0002:00000400       \177VERSION_NULL_THUNK_DATA 000000018000f400     version:VERSION.dll
 0002:00000408       __imp_wcstombs             000000018000f408     ucrt:api-ms-win-crt-convert-l1-1-0.dll
 0002:00000410       __imp__itoa_s              000000018000f410     ucrt:api-ms-win-crt-convert-l1-1-0.dll
 0002:00000418       __imp_atoi                 000000018000f418     ucrt:api-ms-win-crt-convert-l1-1-0.dll
 0002:00000420       \177api-ms-win-crt-convert-l1-1-0_NULL_THUNK_DATA 000000018000f420     ucrt:api-ms-win-crt-convert-l1-1-0.dll
 0002:00000428       __imp__wgetcwd             000000018000f428     ucrt:api-ms-win-crt-environment-l1-1-0.dll
 0002:00000430       __imp__wgetdcwd            000000018000f430     ucrt:api-ms-win-crt-environment-l1-1-0.dll
 0002:00000438       __imp__wgetenv             000000018000f438     ucrt:api-ms-win-crt-environment-l1-1-0.dll
 0002:00000440       \177api-ms-win-crt-environment-l1-1-0_NULL_THUNK_DATA 000000018000f440     ucrt:api-ms-win-crt-environment-l1-1-0.dll
 0002:00000448       __imp__wrename             000000018000f448     ucrt:api-ms-win-crt-filesystem-l1-1-0.dll
 0002:00000450       __imp__wfullpath           000000018000f450     ucrt:api-ms-win-crt-filesystem-l1-1-0.dll
 0002:00000458       \177api-ms-win-crt-filesystem-l1-1-0_NULL_THUNK_DATA 000000018000f458     ucrt:api-ms-win-crt-filesystem-l1-1-0.dll
 0002:00000460       __imp_malloc               000000018000f460     ucrt:api-ms-win-crt-heap-l1-1-0.dll
 0002:00000468       __imp_realloc              000000018000f468     ucrt:api-ms-win-crt-heap-l1-1-0.dll
 0002:00000470       __imp_free                 000000018000f470     ucrt:api-ms-win-crt-heap-l1-1-0.dll
 0002:00000478       \177api-ms-win-crt-heap-l1-1-0_NULL_THUNK_DATA 000000018000f478     ucrt:api-ms-win-crt-heap-l1-1-0.dll
 0002:00000480       __imp__initialize_onexit_table 000000018000f480     ucrt:api-ms-win-crt-runtime-l1-1-0.dll
 0002:00000488       __imp__initialize_narrow_environment 000000018000f488     ucrt:api-ms-win-crt-runtime-l1-1-0.dll
 0002:00000490       __imp__seh_filter_dll      000000018000f490     ucrt:api-ms-win-crt-runtime-l1-1-0.dll
 0002:00000498       __imp__initterm_e          000000018000f498     ucrt:api-ms-win-crt-runtime-l1-1-0.dll
 0002:000004a0       __imp__initterm            000000018000f4a0     ucrt:api-ms-win-crt-runtime-l1-1-0.dll
 0002:000004a8       __imp_strerror_s           000000018000f4a8     ucrt:api-ms-win-crt-runtime-l1-1-0.dll
 0002:000004b0       __imp__cexit               000000018000f4b0     ucrt:api-ms-win-crt-runtime-l1-1-0.dll
 0002:000004b8       __imp__errno               000000018000f4b8     ucrt:api-ms-win-crt-runtime-l1-1-0.dll
 0002:000004c0       __imp__execute_onexit_table 000000018000f4c0     ucrt:api-ms-win-crt-runtime-l1-1-0.dll
 0002:000004c8       __imp__configure_narrow_argv 000000018000f4c8     ucrt:api-ms-win-crt-runtime-l1-1-0.dll
 0002:000004d0       \177api-ms-win-crt-runtime-l1-1-0_NULL_THUNK_DATA 000000018000f4d0     ucrt:api-ms-win-crt-runtime-l1-1-0.dll
 0002:000004d8       __imp___acrt_iob_func      000000018000f4d8     ucrt:api-ms-win-crt-stdio-l1-1-0.dll
 0002:000004e0       __imp___stdio_common_vswprintf 000000018000f4e0     ucrt:api-ms-win-crt-stdio-l1-1-0.dll
 0002:000004e8       __imp_fopen_s              000000018000f4e8     ucrt:api-ms-win-crt-stdio-l1-1-0.dll
 0002:000004f0       __imp_fopen                000000018000f4f0     ucrt:api-ms-win-crt-stdio-l1-1-0.dll
 0002:000004f8       __imp___stdio_common_vsscanf 000000018000f4f8     ucrt:api-ms-win-crt-stdio-l1-1-0.dll
 0002:00000500       __imp___stdio_common_vsprintf 000000018000f500     ucrt:api-ms-win-crt-stdio-l1-1-0.dll
 0002:00000508       __imp_fgets                000000018000f508     ucrt:api-ms-win-crt-stdio-l1-1-0.dll
 0002:00000510       __imp_fclose               000000018000f510     ucrt:api-ms-win-crt-stdio-l1-1-0.dll
 0002:00000518       \177api-ms-win-crt-stdio-l1-1-0_NULL_THUNK_DATA 000000018000f518     ucrt:api-ms-win-crt-stdio-l1-1-0.dll
 0002:00000520       __imp_iswctype             000000018000f520     ucrt:api-ms-win-crt-string-l1-1-0.dll
 0002:00000528       __imp__wcsupr              000000018000f528     ucrt:api-ms-win-crt-string-l1-1-0.dll
 0002:00000530       __imp__strdup              000000018000f530     ucrt:api-ms-win-crt-string-l1-1-0.dll
 0002:00000538       __imp_strcmp               000000018000f538     ucrt:api-ms-win-crt-string-l1-1-0.dll
 0002:00000540       __imp_towupper             000000018000f540     ucrt:api-ms-win-crt-string-l1-1-0.dll
 0002:00000548       __imp_wcscat               000000018000f548     ucrt:api-ms-win-crt-string-l1-1-0.dll
 0002:00000550       __imp_strlen               000000018000f550     ucrt:api-ms-win-crt-string-l1-1-0.dll
 0002:00000558       __imp_strcpy               000000018000f558     ucrt:api-ms-win-crt-string-l1-1-0.dll
 0002:00000560       __imp_strcat               000000018000f560     ucrt:api-ms-win-crt-string-l1-1-0.dll
 0002:00000568       __imp_wcslen               000000018000f568     ucrt:api-ms-win-crt-string-l1-1-0.dll
 0002:00000570       __imp_wcscpy               000000018000f570     ucrt:api-ms-win-crt-string-l1-1-0.dll
 0002:00000578       __imp_wcscmp               000000018000f578     ucrt:api-ms-win-crt-string-l1-1-0.dll
 0002:00000580       __imp__wcsdup              000000018000f580     ucrt:api-ms-win-crt-string-l1-1-0.dll
 0002:00000588       __imp_wcscat_s             000000018000f588     ucrt:api-ms-win-crt-string-l1-1-0.dll
 0002:00000590       __imp_wcsncat              000000018000f590     ucrt:api-ms-win-crt-string-l1-1-0.dll
 0002:00000598       __imp_wcsncmp              000000018000f598     ucrt:api-ms-win-crt-string-l1-1-0.dll
 0002:000005a0       \177api-ms-win-crt-string-l1-1-0_NULL_THUNK_DATA 000000018000f5a0     ucrt:api-ms-win-crt-string-l1-1-0.dll
 0002:000005a8       __imp_JVM_ExpandStackFrameInfo 000000018000f5a8     jvm:jvm.dll
 0002:000005b0       __imp_JVM_FindSignal       000000018000f5b0     jvm:jvm.dll
 0002:000005b8       __imp_JVM_RaiseSignal      000000018000f5b8     jvm:jvm.dll
 0002:000005c0       __imp_JVM_RegisterSignal   000000018000f5c0     jvm:jvm.dll
 0002:000005c8       __imp_JVM_Halt             000000018000f5c8     jvm:jvm.dll
 0002:000005d0       __imp_JVM_BeforeHalt       000000018000f5d0     jvm:jvm.dll
 0002:000005d8       __imp_JVM_ActiveProcessorCount 000000018000f5d8     jvm:jvm.dll
 0002:000005e0       __imp_JVM_MaxMemory        000000018000f5e0     jvm:jvm.dll
 0002:000005e8       __imp_JVM_FreeMemory       000000018000f5e8     jvm:jvm.dll
 0002:000005f0       __imp_JVM_TotalMemory      000000018000f5f0     jvm:jvm.dll
 0002:000005f8       __imp_JVM_GC               000000018000f5f8     jvm:jvm.dll
 0002:00000600       __imp_JVM_AreNestMates     000000018000f600     jvm:jvm.dll
 0002:00000608       __imp_JVM_GetCallerClass   000000018000f608     jvm:jvm.dll
 0002:00000610       __imp_JVM_ReferenceRefersTo 000000018000f610     jvm:jvm.dll
 0002:00000618       __imp_JVM_WaitForReferencePendingList 000000018000f618     jvm:jvm.dll
 0002:00000620       __imp_JVM_HasReferencePendingList 000000018000f620     jvm:jvm.dll
 0002:00000628       __imp_JVM_GetAndClearReferencePendingList 000000018000f628     jvm:jvm.dll
 0002:00000630       __imp_JVM_GetThreadInterruptEvent 000000018000f630     jvm:jvm.dll
 0002:00000638       __imp_JVM_IsPreviewEnabled 000000018000f638     jvm:jvm.dll
 0002:00000640       __imp_JVM_PhantomReferenceRefersTo 000000018000f640     jvm:jvm.dll
 0002:00000648       __imp_JVM_ReferenceClear   000000018000f648     jvm:jvm.dll
 0002:00000650       __imp_JVM_GetExtendedNPEMessage 000000018000f650     jvm:jvm.dll
 0002:00000658       __imp_JVM_IsSupportedJNIVersion 000000018000f658     jvm:jvm.dll
 0002:00000660       __imp_JVM_FindLibraryEntry 000000018000f660     jvm:jvm.dll
 0002:00000668       __imp_JVM_UnloadLibrary    000000018000f668     jvm:jvm.dll
 0002:00000670       __imp_JVM_LoadLibrary      000000018000f670     jvm:jvm.dll
 0002:00000678       __imp_JVM_NewInstanceFromConstructor 000000018000f678     jvm:jvm.dll
 0002:00000680       __imp_JVM_InvokeMethod     000000018000f680     jvm:jvm.dll
 0002:00000688       __imp_JVM_AddReadsModule   000000018000f688     jvm:jvm.dll
 0002:00000690       __imp_JVM_AddModuleExportsToAll 000000018000f690     jvm:jvm.dll
 0002:00000698       __imp_JVM_AddModuleExportsToAllUnnamed 000000018000f698     jvm:jvm.dll
 0002:000006a0       __imp_JVM_AddModuleExports 000000018000f6a0     jvm:jvm.dll
 0002:000006a8       __imp_JVM_DefineModule     000000018000f6a8     jvm:jvm.dll
 0002:000006b0       __imp_JVM_LookupLambdaProxyClassFromArchive 000000018000f6b0     jvm:jvm.dll
 0002:000006b8       __imp_JVM_RegisterLambdaProxyClassForArchiving 000000018000f6b8     jvm:jvm.dll
 0002:000006c0       __imp_JVM_IsForeignLinkerSupported 000000018000f6c0     jvm:jvm.dll
 0002:000006c8       __imp_JVM_IsFinalizationEnabled 000000018000f6c8     jvm:jvm.dll
 0002:000006d0       __imp_JVM_ReportFinalizationComplete 000000018000f6d0     jvm:jvm.dll
 0002:000006d8       __imp_JVM_GetFieldTypeAnnotations 000000018000f6d8     jvm:jvm.dll
 0002:000006e0       __imp_JVM_GetMethodParameters 000000018000f6e0     jvm:jvm.dll
 0002:000006e8       __imp_JVM_GetMethodTypeAnnotations 000000018000f6e8     jvm:jvm.dll
 0002:000006f0       __imp_JVM_IsContinuationsSupported 000000018000f6f0     jvm:jvm.dll
 0002:000006f8       __imp_JVM_RegisterContinuationMethods 000000018000f6f8     jvm:jvm.dll
 0002:00000700       __imp_JVM_ConstantPoolGetTagAt 000000018000f700     jvm:jvm.dll
 0002:00000708       __imp_JVM_ConstantPoolGetUTF8At 000000018000f708     jvm:jvm.dll
 0002:00000710       __imp_JVM_ConstantPoolGetStringAt 000000018000f710     jvm:jvm.dll
 0002:00000718       __imp_JVM_ConstantPoolGetDoubleAt 000000018000f718     jvm:jvm.dll
 0002:00000720       __imp_JVM_ConstantPoolGetFloatAt 000000018000f720     jvm:jvm.dll
 0002:00000728       __imp_JVM_ConstantPoolGetLongAt 000000018000f728     jvm:jvm.dll
 0002:00000730       __imp_JVM_ConstantPoolGetIntAt 000000018000f730     jvm:jvm.dll
 0002:00000738       __imp_JVM_ConstantPoolGetNameAndTypeRefInfoAt 000000018000f738     jvm:jvm.dll
 0002:00000740       __imp_JVM_CallStackWalk    000000018000f740     jvm:jvm.dll
 0002:00000748       __imp_JVM_ConstantPoolGetMemberRefInfoAt 000000018000f748     jvm:jvm.dll
 0002:00000750       __imp_JVM_ConstantPoolGetFieldAtIfLoaded 000000018000f750     jvm:jvm.dll
 0002:00000758       __imp_JVM_ConstantPoolGetFieldAt 000000018000f758     jvm:jvm.dll
 0002:00000760       __imp_JVM_ConstantPoolGetMethodAtIfLoaded 000000018000f760     jvm:jvm.dll
 0002:00000768       __imp_JVM_ConstantPoolGetMethodAt 000000018000f768     jvm:jvm.dll
 0002:00000770       __imp_JVM_ConstantPoolGetClassRefIndexAt 000000018000f770     jvm:jvm.dll
 0002:00000778       __imp_JVM_ConstantPoolGetClassAtIfLoaded 000000018000f778     jvm:jvm.dll
 0002:00000780       __imp_JVM_ConstantPoolGetClassAt 000000018000f780     jvm:jvm.dll
 0002:00000788       __imp_JVM_ConstantPoolGetSize 000000018000f788     jvm:jvm.dll
 0002:00000790       __imp_JVM_LookupDefineClass 000000018000f790     jvm:jvm.dll
 0002:00000798       __imp_JVM_DefineClassWithSource 000000018000f798     jvm:jvm.dll
 0002:000007a0       __imp_JVM_FindLoadedClass  000000018000f7a0     jvm:jvm.dll
 0002:000007a8       __imp_JVM_FindClassFromBootLoader 000000018000f7a8     jvm:jvm.dll
 0002:000007b0       __imp_JVM_AssertionStatusDirectives 000000018000f7b0     jvm:jvm.dll
 0002:000007b8       __imp_JVM_FindClassFromCaller 000000018000f7b8     jvm:jvm.dll
 0002:000007c0       __imp_JVM_FindPrimitiveClass 000000018000f7c0     jvm:jvm.dll
 0002:000007c8       __imp_JVM_GetClassFileVersion 000000018000f7c8     jvm:jvm.dll
 0002:000007d0       __imp_JVM_GetEnclosingMethodInfo 000000018000f7d0     jvm:jvm.dll
 0002:000007d8       __imp_JVM_DesiredAssertionStatus 000000018000f7d8     jvm:jvm.dll
 0002:000007e0       __imp_JVM_GetClassConstantPool 000000018000f7e0     jvm:jvm.dll
 0002:000007e8       __imp_JVM_GetPermittedSubclasses 000000018000f7e8     jvm:jvm.dll
 0002:000007f0       __imp_JVM_GetRecordComponents 000000018000f7f0     jvm:jvm.dll
 0002:000007f8       __imp_JVM_IsRecord         000000018000f7f8     jvm:jvm.dll
 0002:00000800       __imp_JVM_GetNestMembers   000000018000f800     jvm:jvm.dll
 0002:00000808       __imp_JVM_GetNestHost      000000018000f808     jvm:jvm.dll
 0002:00000810       __imp_JVM_GetClassAccessFlags 000000018000f810     jvm:jvm.dll
 0002:00000818       __imp_JVM_GetClassDeclaredConstructors 000000018000f818     jvm:jvm.dll
 0002:00000820       __imp_JVM_GetClassDeclaredFields 000000018000f820     jvm:jvm.dll
 0002:00000828       __imp_JVM_GetClassDeclaredMethods 000000018000f828     jvm:jvm.dll
 0002:00000830       __imp_JVM_GetClassTypeAnnotations 000000018000f830     jvm:jvm.dll
 0002:00000838       __imp_JVM_GetClassAnnotations 000000018000f838     jvm:jvm.dll
 0002:00000840       __imp_JVM_GetClassSignature 000000018000f840     jvm:jvm.dll
 0002:00000848       __imp_JVM_GetSimpleBinaryName 000000018000f848     jvm:jvm.dll
 0002:00000850       __imp_JVM_GetDeclaringClass 000000018000f850     jvm:jvm.dll
 0002:00000858       __imp_JVM_GetDeclaredClasses 000000018000f858     jvm:jvm.dll
 0002:00000860       __imp_JVM_IsHiddenClass    000000018000f860     jvm:jvm.dll
 0002:00000868       __imp_JVM_GetClassInterfaces 000000018000f868     jvm:jvm.dll
 0002:00000870       __imp_JVM_InitClassName    000000018000f870     jvm:jvm.dll
 0002:00000878       __imp_JVM_DefineArchivedModules 000000018000f878     jvm:jvm.dll
 0002:00000880       __imp_JVM_NeedsClassInitBarrierForCDS 000000018000f880     jvm:jvm.dll
 0002:00000888       __imp_JVM_DumpDynamicArchive 000000018000f888     jvm:jvm.dll
 0002:00000890       __imp_JVM_DumpClassListToFile 000000018000f890     jvm:jvm.dll
 0002:00000898       __imp_JVM_LogLambdaFormInvoker 000000018000f898     jvm:jvm.dll
 0002:000008a0       __imp_JVM_GetRandomSeedForDumping 000000018000f8a0     jvm:jvm.dll
 0002:000008a8       __imp_JVM_GetCDSConfigStatus 000000018000f8a8     jvm:jvm.dll
 0002:000008b0       __imp_JVM_InitializeFromArchive 000000018000f8b0     jvm:jvm.dll
 0002:000008b8       __imp_JVM_SetBootLoaderUnnamedModule 000000018000f8b8     jvm:jvm.dll
 0002:000008c0       __imp_JVM_GetSystemPackages 000000018000f8c0     jvm:jvm.dll
 0002:000008c8       __imp_JVM_MoreStackWalk    000000018000f8c8     jvm:jvm.dll
 0002:000008d0       __imp_JVM_SetStackWalkContinuation 000000018000f8d0     jvm:jvm.dll
 0002:000008d8       __imp_JVM_InitStackTraceElementArray 000000018000f8d8     jvm:jvm.dll
 0002:000008e0       __imp_JVM_InitStackTraceElement 000000018000f8e0     jvm:jvm.dll
 0002:000008e8       __imp_JVM_InternString     000000018000f8e8     jvm:jvm.dll
 0002:000008f0       __imp_JVM_CurrentTimeMillis 000000018000f8f0     jvm:jvm.dll
 0002:000008f8       __imp_JVM_NanoTime         000000018000f8f8     jvm:jvm.dll
 0002:00000900       __imp_JVM_ArrayCopy        000000018000f900     jvm:jvm.dll
 0002:00000908       __imp_JVM_IHashCode        000000018000f908     jvm:jvm.dll
 0002:00000910       __imp_JVM_GetProperties    000000018000f910     jvm:jvm.dll
 0002:00000918       __imp_JVM_StartThread      000000018000f918     jvm:jvm.dll
 0002:00000920       __imp_JVM_SetThreadPriority 000000018000f920     jvm:jvm.dll
 0002:00000928       __imp_JVM_Yield            000000018000f928     jvm:jvm.dll
 0002:00000930       __imp_JVM_SleepNanos       000000018000f930     jvm:jvm.dll
 0002:00000938       __imp_JVM_CurrentCarrierThread 000000018000f938     jvm:jvm.dll
 0002:00000940       __imp_JVM_CurrentThread    000000018000f940     jvm:jvm.dll
 0002:00000948       __imp_JVM_GetArrayElement  000000018000f948     jvm:jvm.dll
 0002:00000950       __imp_JVM_SetCurrentThread 000000018000f950     jvm:jvm.dll
 0002:00000958       __imp_JVM_Interrupt        000000018000f958     jvm:jvm.dll
 0002:00000960       __imp_JVM_GetSystemPackage 000000018000f960     jvm:jvm.dll
 0002:00000968       __imp_JVM_HoldsLock        000000018000f968     jvm:jvm.dll
 0002:00000970       __imp_JVM_GetStackTrace    000000018000f970     jvm:jvm.dll
 0002:00000978       __imp_JVM_GetAllThreads    000000018000f978     jvm:jvm.dll
 0002:00000980       __imp_JVM_SetNativeThreadName 000000018000f980     jvm:jvm.dll
 0002:00000988       __imp_JVM_DumpThreads      000000018000f988     jvm:jvm.dll
 0002:00000990       __imp_JVM_ScopedValueCache 000000018000f990     jvm:jvm.dll
 0002:00000998       __imp_JVM_SetScopedValueCache 000000018000f998     jvm:jvm.dll
 0002:000009a0       __imp_JVM_FindScopedValueBindings 000000018000f9a0     jvm:jvm.dll
 0002:000009a8       __imp_JVM_NewMultiArray    000000018000f9a8     jvm:jvm.dll
 0002:000009b0       __imp_JVM_NewArray         000000018000f9b0     jvm:jvm.dll
 0002:000009b8       __imp_JVM_GetNextThreadIdOffset 000000018000f9b8     jvm:jvm.dll
 0002:000009c0       __imp_JVM_EnsureMaterializedForStackWalk_func 000000018000f9c0     jvm:jvm.dll
 0002:000009c8       __imp_JVM_CreateThreadSnapshot 000000018000f9c8     jvm:jvm.dll
 0002:000009d0       __imp_JVM_SetPrimitiveArrayElement 000000018000f9d0     jvm:jvm.dll
 0002:000009d8       __imp_JVM_SetArrayElement  000000018000f9d8     jvm:jvm.dll
 0002:000009e0       __imp_JVM_GetPrimitiveArrayElement 000000018000f9e0     jvm:jvm.dll
 0002:000009e8       __imp_JVM_FillInStackTrace 000000018000f9e8     jvm:jvm.dll
 0002:000009f0       __imp_JVM_GetNanoTimeAdjustment 000000018000f9f0     jvm:jvm.dll
 0002:000009f8       __imp_JVM_GetVmArguments   000000018000f9f8     jvm:jvm.dll
 0002:00000a00       __imp_jio_vfprintf         000000018000fa00     jvm:jvm.dll
 0002:00000a08       __imp_jio_vsnprintf        000000018000fa08     jvm:jvm.dll
 0002:00000a10       __imp_JVM_TakeVirtualThreadListToUnblock 000000018000fa10     jvm:jvm.dll
 0002:00000a18       __imp_JVM_VirtualThreadPinnedEvent 000000018000fa18     jvm:jvm.dll
 0002:00000a20       __imp_JVM_VirtualThreadDisableSuspend 000000018000fa20     jvm:jvm.dll
 0002:00000a28       __imp_JVM_VirtualThreadUnmount 000000018000fa28     jvm:jvm.dll
 0002:00000a30       __imp_JVM_VirtualThreadMount 000000018000fa30     jvm:jvm.dll
 0002:00000a38       __imp_JVM_VirtualThreadEnd 000000018000fa38     jvm:jvm.dll
 0002:00000a40       __imp_JVM_VirtualThreadStart 000000018000fa40     jvm:jvm.dll
 0002:00000a48       __imp_JVM_GetTemporaryDirectory 000000018000fa48     jvm:jvm.dll
 0002:00000a50       __imp_JVM_InitAgentProperties 000000018000fa50     jvm:jvm.dll
 0002:00000a58       __imp_JVM_ConstantPoolGetNameAndTypeRefIndexAt 000000018000fa58     jvm:jvm.dll
 0002:00000a60       __imp_JVM_LatestUserDefinedLoader 000000018000fa60     jvm:jvm.dll
 0002:00000a68       __imp_JVM_GetArrayLength   000000018000fa68     jvm:jvm.dll
 0002:00000a70       \177jvm_NULL_THUNK_DATA    000000018000fa70     jvm:jvm.dll
 0002:00000a78       __imp_CoTaskMemFree        000000018000fa78     ole32:ole32.dll
 0002:00000a80       \177ole32_NULL_THUNK_DATA  000000018000fa80     ole32:ole32.dll
 0002:00000a88       __guard_check_icall_fptr   000000018000fa88     MSVCRT:guard_support.obj
 0002:00000a90       __guard_xfg_check_icall_fptr 000000018000fa90     MSVCRT:guard_support.obj
 0002:00000a98       __guard_dispatch_icall_fptr 000000018000fa98     MSVCRT:guard_support.obj
 0002:00000aa0       __guard_xfg_dispatch_icall_fptr 000000018000faa0     MSVCRT:guard_support.obj
 0002:00000aa8       __guard_xfg_table_dispatch_icall_fptr 000000018000faa8     MSVCRT:guard_support.obj
 0002:00000ab0       __castguard_check_failure_os_handled_fptr 000000018000fab0     MSVCRT:guard_support.obj
 0002:00000ab8       __guard_memcpy_fptr        000000018000fab8     vcruntime:softmemtag.obj
 0002:00000ac0       __xc_a                     000000018000fac0     MSVCRT:initializers.obj
 0002:00000ac8       __xc_z                     000000018000fac8     MSVCRT:initializers.obj
 0002:00000ad0       __xi_a                     000000018000fad0     MSVCRT:initializers.obj
 0002:00000ad8       __xi_z                     000000018000fad8     MSVCRT:initializers.obj
 0002:00000ae0       __xp_a                     000000018000fae0     MSVCRT:initializers.obj
 0002:00000ae8       __xp_z                     000000018000fae8     MSVCRT:initializers.obj
 0002:00000af0       __xt_a                     000000018000faf0     MSVCRT:initializers.obj
 0002:00000af8       __xt_z                     000000018000faf8     MSVCRT:initializers.obj
 0002:00000b00       ??_C@_0O@LMKLDNGH@initClassName@ 000000018000fb00     Class.obj
 0002:00000b10       ??_C@_0BF@FOHFOJOB@?$CI?$CJLjava?1lang?1String?$DL@ 000000018000fb10     Class.obj
 0002:00000b28       ??_C@_0O@BCDKKCAE@getSuperclass@ 000000018000fb28     Class.obj
 0002:00000b38       ??_C@_0BE@IIFEGCLG@?$CI?$CJLjava?1lang?1Class?$DL@ 000000018000fb38     Class.obj
 0002:00000b50       ??_C@_0P@FLDOEJHK@getInterfaces0@ 000000018000fb50     Class.obj
 0002:00000b60       ??_C@_0BF@BNKCIMJP@?$CI?$CJ?$FLLjava?1lang?1Class?$DL@ 000000018000fb60     Class.obj
 0002:00000b78       ??_C@_08POGCNBGK@isHidden@ 000000018000fb78     Class.obj
 0002:00000b84       ??_C@_03MMPFGPID@?$CI?$CJZ@ 000000018000fb84     Class.obj
 0002:00000b88       ??_C@_0BD@BEKBHNDA@getDeclaredFields0@ 000000018000fb88     Class.obj
 0002:00000ba0       ??_C@_0BO@KFNILMGC@?$CIZ?$CJ?$FLLjava?1lang?1reflect?1Field?$DL@ 000000018000fba0     Class.obj
 0002:00000bc0       ??_C@_0BE@LOILJEHC@getDeclaredMethods0@ 000000018000fbc0     Class.obj
 0002:00000bd8       ??_C@_0BP@IIIKNIKA@?$CIZ?$CJ?$FLLjava?1lang?1reflect?1Method?$DL@ 000000018000fbd8     Class.obj
 0002:00000bf8       ??_C@_0BJ@KLPKFLFA@getDeclaredConstructors0@ 000000018000fbf8     Class.obj
 0002:00000c18       ??_C@_0CE@FDMOFPI@?$CIZ?$CJ?$FLLjava?1lang?1reflect?1Construc@ 000000018000fc18     Class.obj
 0002:00000c40       ??_C@_0BE@CIFNAIBM@getDeclaredClasses0@ 000000018000fc40     Class.obj
 0002:00000c58       ??_C@_0BD@NHPDOJGF@getDeclaringClass0@ 000000018000fc58     Class.obj
 0002:00000c70       ??_C@_0BF@ODCBBOMF@getSimpleBinaryName0@ 000000018000fc70     Class.obj
 0002:00000c88       ??_C@_0BF@KFMFPKNK@getGenericSignature0@ 000000018000fc88     Class.obj
 0002:00000ca0       ??_C@_0BC@CDJDGCDH@getRawAnnotations@ 000000018000fca0     Class.obj
 0002:00000cb4       ??_C@_04LHPAGAEF@?$CI?$CJ?$FLB@ 000000018000fcb4     Class.obj
 0002:00000cc0       ??_C@_0BA@DLHKEBGM@getConstantPool@ 000000018000fcc0     Class.obj
 0002:00000cd0       ??_C@_0CG@OKGFDDJA@?$CI?$CJLjdk?1internal?1reflect?1Constan@ 000000018000fcd0     Class.obj
 0002:00000cf8       ??_C@_0BI@EOEBGMEG@desiredAssertionStatus0@ 000000018000fcf8     Class.obj
 0002:00000d10       ??_C@_0BF@CBMAAKJJ@?$CILjava?1lang?1Class?$DL?$CJZ@ 000000018000fd10     Class.obj
 0002:00000d28       ??_C@_0BE@OLDEPMPN@getEnclosingMethod0@ 000000018000fd28     Class.obj
 0002:00000d40       ??_C@_0BG@PFDHKCPA@?$CI?$CJ?$FLLjava?1lang?1Object?$DL@ 000000018000fd40     Class.obj
 0002:00000d58       ??_C@_0BG@CNILIFMJ@getRawTypeAnnotations@ 000000018000fd58     Class.obj
 0002:00000d70       ??_C@_0N@NMCDFPDB@getNestHost0@ 000000018000fd70     Class.obj
 0002:00000d80       ??_C@_0BA@DLOACIFG@getNestMembers0@ 000000018000fd80     Class.obj
 0002:00000d90       ??_C@_0BF@GFGGJCDB@getRecordComponents0@ 000000018000fd90     Class.obj
 0002:00000da8       ??_C@_0CH@JOFOJHIB@?$CI?$CJ?$FLLjava?1lang?1reflect?1RecordCom@ 000000018000fda8     Class.obj
 0002:00000dd0       ??_C@_09PCIIHAKK@isRecord0@ 000000018000fdd0     Class.obj
 0002:00000de0       ??_C@_0BI@GAOMCNP@getPermittedSubclasses0@ 000000018000fde0     Class.obj
 0002:00000df8       ??_C@_0BF@EBBECJAJ@getClassFileVersion0@ 000000018000fdf8     Class.obj
 0002:00000e10       ??_C@_03KNBKCOBB@?$CI?$CJI@ 000000018000fe10     Class.obj
 0002:00000e18       ??_C@_0BI@PIENPELF@getClassAccessFlagsRaw0@ 000000018000fe18     Class.obj
 0002:00000e30       ??_C@_0BD@EELMJMNJ@retrieveDirectives@ 000000018000fe30     ClassLoader.obj
 0002:00000e48       ??_C@_0CI@FCANAINE@?$CI?$CJLjava?1lang?1AssertionStatusDir@ 000000018000fe48     ClassLoader.obj
 0002:00000e70       ??_C@_01JPJNBJEM@I@        000000018000fe70     FileDescriptor_md.obj
 0002:00000e74       ??_C@_02ENHFDPNM@fd@       000000018000fe74     FileDescriptor_md.obj
 0002:00000e78       ??_C@_01LELAEKIP@J@        000000018000fe78     FileDescriptor_md.obj
 0002:00000e7c       ??_C@_06NCGDPKCC@handle@   000000018000fe7c     FileDescriptor_md.obj
 0002:00000e84       ??_C@_01POHCFINO@Z@        000000018000fe84     FileDescriptor_md.obj
 0002:00000e88       ??_C@_06PCICMFGG@append@   000000018000fe88     FileDescriptor_md.obj
 0002:00000e90       ??_C@_0M@IALGLCNJ@sync?5failed@ 000000018000fe90     FileDescriptor_md.obj
 0002:00000ea0       ??_C@_0BM@MBMINGIL@java?1io?1SyncFailedException@ 000000018000fea0     FileDescriptor_md.obj
 0002:00000ec0       ??_C@_0N@NOKLILHD@close?5failed@ 000000018000fec0     FileDescriptor_md.obj
 0002:00000ed0       ??_C@_0BJ@BDFOFHPL@Ljava?1io?1FileDescriptor?$DL@ 000000018000fed0     FileInputStream.obj
 0002:00000ef0       ??_C@_0O@KLFONINF@Stream?5Closed@ 000000018000fef0     FileInputStream.obj
 0002:00000f00       ??_C@_0BB@CEBOPAFI@GetLength?5failed@ 000000018000ff00     FileInputStream.obj
 0002:00000f18       ??_C@_0M@HPFDGGMC@Seek?5failed@ 000000018000ff18     FileInputStream.obj
 0002:00000f28       ??_C@_0L@FCLNKJKA@Seek?5error@ 000000018000ff28     FileInputStream.obj
 0002:00000f34       ??_C@_11LOCGONAA@@         000000018000ff34     HostLocaleProviderAdapter_md.obj
 0002:00000f38       ??_C@_13BMLCKOLB@?$PP?$KE@ 000000018000ff38     HostLocaleProviderAdapter_md.obj
 0002:00000f3c       ??_C@_15GMICKCJK@?$PP?$KE?$AA?5@ 000000018000ff3c     HostLocaleProviderAdapter_md.obj
 0002:00000f44       ??_C@_13EJFHHPOP@?$AA?$CF@ 000000018000ff44     HostLocaleProviderAdapter_md.obj
 0002:00000f48       ??_C@_15LJGOGFOH@?$AA?$CF?$AA?5@ 000000018000ff48     HostLocaleProviderAdapter_md.obj
 0002:00000f50       ??_C@_13LLDNKHDC@?$AA?$CI@ 000000018000ff50     HostLocaleProviderAdapter_md.obj
 0002:00000f54       ??_C@_13IMODFHAA@?$AA?9@   000000018000ff54     HostLocaleProviderAdapter_md.obj
 0002:00000f58       ??_C@_15FFDNOHIK@?$AA?9?$AA?5@ 000000018000ff58     HostLocaleProviderAdapter_md.obj
 0002:00000f60       ??_C@_15GHMLFHFF@?$AA?$CI?$PP?$KE@ 000000018000ff60     HostLocaleProviderAdapter_md.obj
 0002:00000f68       ??_C@_15DHAGMGOG@?$AA?9?$PP?$KE@ 000000018000ff68     HostLocaleProviderAdapter_md.obj
 0002:00000f70       ??_C@_15JOOIHKEH@?$PP?$KE?$AA?9@ 000000018000ff70     HostLocaleProviderAdapter_md.obj
 0002:00000f78       ??_C@_17NKBBKLNH@?$AA?9?$PP?$KE?$AA?5@ 000000018000ff78     HostLocaleProviderAdapter_md.obj
 0002:00000f80       ??_C@_17OBCOLLDF@?$PP?$KE?$AA?5?$AA?9@ 000000018000ff80     HostLocaleProviderAdapter_md.obj
 0002:00000f88       ??_C@_17JCPBKFLD@?$AA?$CI?$PP?$KE?$AA?5@ 000000018000ff88     HostLocaleProviderAdapter_md.obj
 0002:00000f90       ??_C@_15GCODBHLI@?$AA?9?$AA?$CF@ 000000018000ff90     HostLocaleProviderAdapter_md.obj
 0002:00000f98       ??_C@_15ELAELNDK@?$AA?$CF?$AA?9@ 000000018000ff98     HostLocaleProviderAdapter_md.obj
 0002:00000fa0       ??_C@_17PPNGMKK@?$AA?9?$AA?$CF?$AA?5@ 000000018000ffa0     HostLocaleProviderAdapter_md.obj
 0002:00000fa8       ??_C@_17HOLPDOHB@?$AA?$CF?$AA?5?$AA?9@ 000000018000ffa8     HostLocaleProviderAdapter_md.obj
 0002:00000fb0       ??_C@_15ILJINFDI@?$AA?5?$PP?$KE@ 000000018000ffb0     HostLocaleProviderAdapter_md.obj
 0002:00000fb8       ??_C@_15NOHNAEGG@?$AA?5?$AA?$CF@ 000000018000ffb8     HostLocaleProviderAdapter_md.obj
 0002:00000fc0       ??_C@_13DIBMAFH@?$AA?$CJ@  000000018000ffc0     HostLocaleProviderAdapter_md.obj
 0002:00000fc4       ??_C@_13HOIJIPNN@?$AA?5@   000000018000ffc4     HostLocaleProviderAdapter_md.obj
 0002:00000fc8       ??_C@_15BLMJCMIJ@?$AA?5?$AA?9@ 000000018000ffc8     HostLocaleProviderAdapter_md.obj
 0002:00000fd0       ??_C@_15BBIKONBA@?$PP?$KE?$AA?$CJ@ 000000018000ffd0     HostLocaleProviderAdapter_md.obj
 0002:00000fd8       ??_C@_17LDHOGGNL@?$AA?5?$PP?$KE?$AA?9@ 000000018000ffd8     HostLocaleProviderAdapter_md.obj
 0002:00000fe0       ??_C@_17DNALNMHF@?$AA?9?$AA?5?$PP?$KE@ 000000018000ffe0     HostLocaleProviderAdapter_md.obj
 0002:00000fe8       ??_C@_17DMBMPBIM@?$AA?5?$PP?$KE?$AA?$CJ@ 000000018000ffe8     HostLocaleProviderAdapter_md.obj
 0002:00000ff0       ??_C@_17GGJCKBKG@?$AA?5?$AA?$CF?$AA?9@ 000000018000fff0     HostLocaleProviderAdapter_md.obj
 0002:00000ff8       ??_C@_17GIOOANCL@?$AA?9?$AA?5?$AA?$CF@ 000000018000fff8     HostLocaleProviderAdapter_md.obj
 0002:00001000       ??_C@_0BA@ONOKGCMP@GetLocaleInfoEx@ 0000000180010000     HostLocaleProviderAdapter_md.obj
 0002:00001010       ??_C@_0N@MDJJJHMB@kernel32?4dll@ 0000000180010010     HostLocaleProviderAdapter_md.obj
 0002:00001020       ??_C@_0BC@NJJJJEJP@GetCalendarInfoEx@ 0000000180010020     HostLocaleProviderAdapter_md.obj
 0002:00001038       ??_C@_0BF@IALNPCBG@EnumCalendarInfoExEx@ 0000000180010038     HostLocaleProviderAdapter_md.obj
 0002:00001050       ??_C@_0BI@FKAGBMCL@memory?5allocation?5error@ 0000000180010050     HostLocaleProviderAdapter_md.obj
 0002:00001068       ??_C@_0BB@FLFAIHG@java?1lang?1String@ 0000000180010068     HostLocaleProviderAdapter_md.obj
 0002:00001080       ??_C@_17PINHLBBM@?$AAu?$AAn?$AAd@ 0000000180010080     HostLocaleProviderAdapter_md.obj
 0002:00001088       ??_C@_15MNPNEAIF@?$AAe?$AAn@ 0000000180010088     HostLocaleProviderAdapter_md.obj
 0002:00001090       ??_C@_13PJJBFPED@?$AA?$DL@ 0000000180010090     HostLocaleProviderAdapter_md.obj
 0002:00001094       ??_C@_13DEFPDAGF@?$AA?0@   0000000180010094     HostLocaleProviderAdapter_md.obj
 0002:00001098       ??_C@_0BG@NEFMNKJA@GetConsoleMode?5failed@ 0000000180010098     JdkConsoleImpl_md.obj
 0002:000010b0       ??_C@_0BG@CBAKADNB@SetConsoleMode?5failed@ 00000001800100b0     JdkConsoleImpl_md.obj
 0002:000010c8       ??_C@_0DG@ILJBJODK@jdk?1internal?1loader?1NativeLibra@ 00000001800100c8     NativeLibraries.obj
 0002:00001100       ??_C@_0L@FFGJFOPI@jniVersion@ 0000000180010100     NativeLibraries.obj
 0002:00001110       ??_C@_0L@OIKEFKEO@JNI_OnLoad@ 0000000180010110     NativeLibraries.obj
 0002:00001120       ??_C@_0N@LLELHEHJ@JNI_OnUnload@ 0000000180010120     NativeLibraries.obj
 0002:00001130       ??_C@_01IDAFKMJL@_@        0000000180010130     NativeLibraries.obj
 0002:00001138       ??_C@_0CO@NLJCNFHA@unsupported?5JNI?5version?50x?$CF08X?5@ 0000000180010138     NativeLibraries.obj
 0002:00001168       ??_C@_0BP@JABHMODJ@java?1lang?1UnsatisfiedLinkError@ 0000000180010168     NativeLibraries.obj
 0002:00001187       ??_C@_00CNPNBAHC@@         0000000180010187     NativeLibraries.obj
 0002:00001188       ??_C@_04HLONOPDM@?4dll@    0000000180010188     NativeLibraries.obj
 0002:00001190       ??_C@_0CB@CKDHIJCP@NULL?5filename?5for?5native?5librar@ 0000000180010190     NativeLibraries.obj
 0002:000011b8       ??_C@_0BM@LKJNLDJK@java?1lang?1NoSuchMethodError@ 00000001800101b8     ObjectStreamClass.obj
 0002:000011d4       ??_C@_03GAEACAIP@?$CI?$CJV@ 00000001800101d4     ObjectStreamClass.obj
 0002:000011d8       ??_C@_08JOGLKNJI@?$DMclinit?$DO@ 00000001800101d8     ObjectStreamClass.obj
 0002:000011e8       ??_C@_0BN@PKAKOFME@GetEnvironmentStrings?5failed@ 00000001800101e8     ProcessEnvironment_md.obj
 0002:00001208       ??_C@_0BD@JFADHEFE@Ljava?1lang?1String?$DL@ 0000000180010208     ProcessHandleImpl_win.obj
 0002:00001220       ??_C@_07KMMNMMFF@command@  0000000180010220     ProcessHandleImpl_win.obj
 0002:00001228       ??_C@_0M@EELMKCHN@commandLine@ 0000000180010228     ProcessHandleImpl_win.obj
 0002:00001238       ??_C@_0BE@KHJCLGPN@?$FLLjava?1lang?1String?$DL@ 0000000180010238     ProcessHandleImpl_win.obj
 0002:00001250       ??_C@_09PBNAMLIK@arguments@ 0000000180010250     ProcessHandleImpl_win.obj
 0002:00001260       ??_C@_09MJNIPNBH@totalTime@ 0000000180010260     ProcessHandleImpl_win.obj
 0002:00001270       ??_C@_09IIHJADCI@startTime@ 0000000180010270     ProcessHandleImpl_win.obj
 0002:0000127c       ??_C@_04CCHAHKJA@user@     000000018001027c     ProcessHandleImpl_win.obj
 0002:00001288       ??_C@_0BD@OOONFEIA@GetExitCodeProcess@ 0000000180010288     ProcessHandleImpl_win.obj
 0002:000012a0       ??_C@_0BL@IONOAEOO@java?1lang?1RuntimeException@ 00000001800102a0     ProcessHandleImpl_win.obj
 0002:000012c0       ??_C@_0BF@GLIJPGCJ@WaitForSingleObjects@ 00000001800102c0     ProcessHandleImpl_win.obj
 0002:000012d8       ??_C@_0BH@DJKIHHBP@snapshot?5not?5available@ 00000001800102d8     ProcessHandleImpl_win.obj
 0002:000012f0       ??_C@_0BG@LPMGLOAP@array?5sizes?5not?5equal@ 00000001800102f0     ProcessHandleImpl_win.obj
 0002:00001308       ??_C@_0BE@JIDLIKOL@GetTokenInformation@ 0000000180010308     ProcessHandleImpl_win.obj
 0002:0000131c       ??_C@_13FPGAJAPJ@?$AA?2@   000000018001031c     ProcessHandleImpl_win.obj
 0002:00001320       ??_C@_1CA@BNEMBNGE@?$AA?$CF?$AAs?$AA?5?$AAe?$AAr?$AAr?$AAo?$AAr?$AA?$DN?$AA?$CF?$AAd?$AA?0?$AA?5?$AA?$CF?$AAs@ 0000000180010320     ProcessImpl_md.obj
 0002:00001340       ??_C@_1CI@OBOFAJOJ@?$AA?$CF?$AAs?$AA?5?$AAf?$AAa?$AAi?$AAl?$AAe?$AAd?$AA?0?$AA?5?$AAe?$AAr?$AAr?$AAo@ 0000000180010340     ProcessImpl_md.obj
 0002:00001368       ??_C@_0CM@EAKDBECK@Secondary?5error?5while?5OS?5messag@ 0000000180010368     ProcessImpl_md.obj
 0002:00001398       ??_C@_1BG@HKMEIOD@?$AAC?$AAr?$AAe?$AAa?$AAt?$AAe?$AAP?$AAi?$AAp?$AAe@ 0000000180010398     ProcessImpl_md.obj
 0002:000013b0       ??_C@_1BM@MMIOBBBF@?$AAC?$AAr?$AAe?$AAa?$AAt?$AAe?$AAP?$AAr?$AAo?$AAc?$AAe?$AAs?$AAs@ 00000001800103b0     ProcessImpl_md.obj
 0002:000013d0       ??_C@_1CG@LCLEBLIK@?$AAG?$AAe?$AAt?$AAE?$AAx?$AAi?$AAt?$AAC?$AAo?$AAd?$AAe?$AAP?$AAr?$AAo?$AAc@ 00000001800103d0     ProcessImpl_md.obj
 0002:000013f8       ??_C@_1CO@PLEHGDKC@?$AAW?$AAa?$AAi?$AAt?$AAF?$AAo?$AAr?$AAM?$AAu?$AAl?$AAt?$AAi?$AAp?$AAl?$AAe@ 00000001800103f8     ProcessImpl_md.obj
 0002:00001428       ??_C@_0M@GPOOGHPH@CreateFileW@ 0000000180010428     ProcessImpl_md.obj
 0002:00001440       __xmm@ffffffffffffffffffffffffffffffff 0000000180010440     ProcessImpl_md.obj
 0002:00001450       ??_C@_0BF@HDGNMJHD@Negative?5seek?5offset@ 0000000180010450     RandomAccessFile.obj
 0002:00001468       ??_C@_0BB@GOOEHMBA@setLength?5failed@ 0000000180010468     RandomAccessFile.obj
 0002:00001480       ??_C@_0DM@NBEIFEIG@jdk?1internal?1loader?1RawNativeLi@ 0000000180010480     RawNativeLibraries.obj
 0002:000014bc       ??_C@_04MEMAJGDJ@name@     00000001800104bc     Signal.obj
 0002:000014c8       ??_C@_0BC@JMDLHMGP@currentTimeMillis@ 00000001800104c8     System.obj
 0002:000014dc       ??_C@_03IGDHHNNC@?$CI?$CJJ@ 00000001800104dc     System.obj
 0002:000014e0       ??_C@_08GAAFINGG@nanoTime@ 00000001800104e0     System.obj
 0002:000014f0       ??_C@_09EEHNOAG@arraycopy@ 00000001800104f0     System.obj
 0002:00001500       ??_C@_0CL@DPOGMIND@?$CILjava?1lang?1Object?$DLILjava?1lang?1@ 0000000180010500     System.obj
 0002:0000152c       ??_C@_02JLHCEMDI@64@       000000018001052c     System.obj
 0002:00001530       ??_C@_0BG@GPDHLGHH@Ljava?1io?1InputStream?$DL@ 0000000180010530     System.obj
 0002:00001548       ??_C@_02LMMGJAGL@in@       0000000180010548     System.obj
 0002:00001550       ??_C@_0BG@FPECDKGJ@Ljava?1io?1PrintStream?$DL@ 0000000180010550     System.obj
 0002:00001568       ??_C@_03KEJHNBPP@out@      0000000180010568     System.obj
 0002:0000156c       ??_C@_03JIDPIAJI@err@      000000018001056c     System.obj
 0002:00001570       ??_C@_0O@OLOAHEKB@name?5too?5long@ 0000000180010570     System.obj
 0002:00001580       ??_C@_06MGHKGFHF@start0@   0000000180010580     Thread.obj
 0002:00001588       ??_C@_0N@GOFHJCMI@setPriority0@ 0000000180010588     Thread.obj
 0002:00001598       ??_C@_04PFANPMCN@?$CII?$CJV@ 0000000180010598     Thread.obj
 0002:000015a0       ??_C@_06IECCAOGC@yield0@   00000001800105a0     Thread.obj
 0002:000015a8       ??_C@_0M@BLHAOIHM@sleepNanos0@ 00000001800105a8     Thread.obj
 0002:000015b4       ??_C@_04OHLIFDMD@?$CIJ?$CJV@ 00000001800105b4     Thread.obj
 0002:000015c0       ??_C@_0BF@DBEINPFJ@currentCarrierThread@ 00000001800105c0     Thread.obj
 0002:000015d8       ??_C@_0BF@GLBLFFEM@?$CI?$CJLjava?1lang?1Thread?$DL@ 00000001800105d8     Thread.obj
 0002:000015f0       ??_C@_0O@GIDKOGNF@currentThread@ 00000001800105f0     Thread.obj
 0002:00001600       ??_C@_0BB@EFBMGMNO@setCurrentThread@ 0000000180010600     Thread.obj
 0002:00001618       ??_C@_0BG@FDENPHAO@?$CILjava?1lang?1Thread?$DL?$CJV@ 0000000180010618     Thread.obj
 0002:00001630       ??_C@_0L@KOCFLKPP@interrupt0@ 0000000180010630     Thread.obj
 0002:00001640       ??_C@_09BKEKKKBN@holdsLock@ 0000000180010640     Thread.obj
 0002:00001650       ??_C@_0BG@DHOOFEJE@?$CILjava?1lang?1Object?$DL?$CJZ@ 0000000180010650     Thread.obj
 0002:00001668       ??_C@_0L@MBENOCKD@getThreads@ 0000000180010668     Thread.obj
 0002:00001678       ??_C@_0BG@CJDMDLMO@?$CI?$CJ?$FLLjava?1lang?1Thread?$DL@ 0000000180010678     Thread.obj
 0002:00001690       ??_C@_0M@ECOKKOKF@dumpThreads@ 0000000180010690     Thread.obj
 0002:000016a0       ??_C@_0DF@ELFIABCA@?$CI?$FLLjava?1lang?1Thread?$DL?$CJ?$FL?$FLLjava?1la@ 00000001800106a0     Thread.obj
 0002:000016d8       ??_C@_0P@NNJPNOLO@getStackTrace0@ 00000001800106d8     Thread.obj
 0002:000016e8       ??_C@_0BF@LHBAMMHC@?$CI?$CJLjava?1lang?1Object?$DL@ 00000001800106e8     Thread.obj
 0002:00001700       ??_C@_0O@LPHHHNKJ@setNativeName@ 0000000180010700     Thread.obj
 0002:00001710       ??_C@_0BG@IKDDPPGD@?$CILjava?1lang?1String?$DL?$CJV@ 0000000180010710     Thread.obj
 0002:00001728       ??_C@_0BB@KGOCCEEG@scopedValueCache@ 0000000180010728     Thread.obj
 0002:00001740       ??_C@_0BE@LJNGDOLG@setScopedValueCache@ 0000000180010740     Thread.obj
 0002:00001758       ??_C@_0BH@JBNAJHIH@?$CI?$FLLjava?1lang?1Object?$DL?$CJV@ 0000000180010758     Thread.obj
 0002:00001770       ??_C@_0BG@PEOLFGEL@getNextThreadIdOffset@ 0000000180010770     Thread.obj
 0002:00001788       ??_C@_0BI@PEHKONLP@findScopedValueBindings@ 0000000180010788     Thread.obj
 0002:000017a0       ??_C@_0BP@DGPDEBNH@ensureMaterializedForStackWalk@ 00000001800107a0     Thread.obj
 0002:000017c0       ??_C@_0BG@JLFLBLJI@?$CILjava?1lang?1Object?$DL?$CJV@ 00000001800107c0     Thread.obj
 0002:000017d8       ??_C@_1BK@BOBBLECB@?$AAS?$AAt?$AAa?$AAn?$AAd?$AAa?$AAr?$AAd?$AAN?$AAa?$AAm?$AAe@ 00000001800107d8     TimeZone_md.obj
 0002:000017f8       ??_C@_0N@PEHDGIGO@StandardName@ 00000001800107f8     TimeZone_md.obj
 0002:00001808       ??_C@_17GFIDPLDA@?$AAS?$AAt?$AAd@ 0000000180010808     TimeZone_md.obj
 0002:00001810       ??_C@_03FFGKOOIA@Std@      0000000180010810     TimeZone_md.obj
 0002:00001818       ??_C@_0P@EKMDNJBA@GMT?$CFc?$CF02d?3?$CF02d@ 0000000180010818     TimeZone_md.obj
 0002:00001828       ??_C@_03HOONMGKE@GMT@      0000000180010828     TimeZone_md.obj
 0002:00001830       ??_C@_0DF@OCPBGDJE@System?2CurrentControlSet?2Contro@ 0000000180010830     TimeZone_md.obj
 0002:00001868       ??_C@_0BM@HEGPJGEC@DynamicDaylightTimeDisabled@ 0000000180010868     TimeZone_md.obj
 0002:00001888       ??_C@_0BA@GCKJIEGO@TimeZoneKeyName@ 0000000180010888     TimeZone_md.obj
 0002:00001898       ??_C@_0DI@LLEGOPFO@SOFTWARE?2Microsoft?2Windows?5NT?2C@ 0000000180010898     TimeZone_md.obj
 0002:000018d0       ??_C@_0DF@JEJGGGGH@SOFTWARE?2Microsoft?2Windows?2Curr@ 00000001800108d0     TimeZone_md.obj
 0002:00001908       ??_C@_03NKEEOHDM@TZI@      0000000180010908     TimeZone_md.obj
 0002:00001910       ??_C@_0BA@PBEHAGHA@?2lib?2tzmappings@ 0000000180010910     TimeZone_md.obj
 0002:00001920       ??_C@_02BMJICGCB@rt@       0000000180010920     TimeZone_md.obj
 0002:00001928       ??_C@_0BA@PMGFJNJD@can?8t?5open?5?$CFs?4?6@ 0000000180010928     TimeZone_md.obj
 0002:00001938       ??_C@_0BG@MJJAMJBB@premature?5end?5of?5line@ 0000000180010938     TimeZone_md.obj
 0002:00001950       ??_C@_0BN@NFCIANLB@illegal?5null?5character?5found@ 0000000180010950     TimeZone_md.obj
 0002:00001970       ??_C@_0CE@OJDILIEN@illegal?5non?9newline?5character?5f@ 0000000180010970     TimeZone_md.obj
 0002:00001994       ??_C@_03MMKGDKGA@001@      0000000180010994     TimeZone_md.obj
 0002:00001998       ??_C@_0DO@EINJANBE@Illegal?5format?5in?5tzmappings?5fi@ 0000000180010998     TimeZone_md.obj
 0002:000019d8       ??_C@_0P@DOCHMBNE@ActiveTimeBias@ 00000001800109d8     TimeZone_md.obj
 0002:000019e8       ??_C@_0BG@FPHJJCID@getNanoTimeAdjustment@ 00000001800109e8     VM.obj
 0002:00001a00       ??_C@_04BMPAOJO@?$CIJ?$CJJ@ 0000000180010a00     VM.obj
 0002:00001a08       ??_C@_0BB@EHHINCMA@notifyJvmtiStart@ 0000000180010a08     VirtualThread.obj
 0002:00001a20       ??_C@_0P@MCKODF@notifyJvmtiEnd@ 0000000180010a20     VirtualThread.obj
 0002:00001a30       ??_C@_0BB@KDNDINGE@notifyJvmtiMount@ 0000000180010a30     VirtualThread.obj
 0002:00001a44       ??_C@_04LHKBAEFM@?$CIZ?$CJV@ 0000000180010a44     VirtualThread.obj
 0002:00001a50       ??_C@_0BD@PIPCEHDM@notifyJvmtiUnmount@ 0000000180010a50     VirtualThread.obj
 0002:00001a68       ??_C@_0BK@FFACNDGC@notifyJvmtiDisableSuspend@ 0000000180010a68     VirtualThread.obj
 0002:00001a88       ??_C@_0BA@LBKNIIHF@postPinnedEvent@ 0000000180010a88     VirtualThread.obj
 0002:00001a98       ??_C@_0BP@PKGADD@takeVirtualThreadListToUnblock@ 0000000180010a98     VirtualThread.obj
 0002:00001ab8       ??_C@_0BM@OGAFEGPF@?$CI?$CJLjava?1lang?1VirtualThread?$DL@ 0000000180010ab8     VirtualThread.obj
 0002:00001ad4       ??_C@_04JCEIFDIJ@J2SE@     0000000180010ad4     WinCAPISeedGenerator.obj
 0002:00001ae0       ??_C@_0N@IOFABHFH@java?1io?1File@ 0000000180010ae0     WinNTFileSystem_md.obj
 0002:00001af0       ??_C@_04LNEJFJGI@path@     0000000180010af0     WinNTFileSystem_md.obj
 0002:00001af8       ??_C@_0CA@NIIGFDJD@native?5memory?5allocation?5failed@ 0000000180010af8     WinNTFileSystem_md.obj
 0002:00001b18       ??_C@_0N@NMICNPLE@Bad?5pathname@ 0000000180010b18     WinNTFileSystem_md.obj
 0002:00001b28       ??_C@_17LIAKHCCP@?$AAC?$AAO?$AAN@ 0000000180010b28     WinNTFileSystem_md.obj
 0002:00001b30       ??_C@_17PFHGFFKC@?$AAP?$AAR?$AAN@ 0000000180010b30     WinNTFileSystem_md.obj
 0002:00001b38       ??_C@_17CNBAFMOM@?$AAA?$AAU?$AAX@ 0000000180010b38     WinNTFileSystem_md.obj
 0002:00001b40       ??_C@_17CLELIOII@?$AAN?$AAU?$AAL@ 0000000180010b40     WinNTFileSystem_md.obj
 0002:00001b48       ??_C@_17KKLPNNMB@?$AAC?$AAO?$AAM@ 0000000180010b48     WinNTFileSystem_md.obj
 0002:00001b50       ??_C@_17KMAOGHDG@?$AAL?$AAP?$AAT@ 0000000180010b50     WinNTFileSystem_md.obj
 0002:00001b58       ??_C@_0BE@LONNMHBH@Could?5not?5open?5file@ 0000000180010b58     WinNTFileSystem_md.obj
 0002:00001b6c       ??_C@_13BBDEGPLJ@?$AA?$CK@ 0000000180010b6c     WinNTFileSystem_md.obj
 0002:00001b70       ??_C@_15PKPONJIK@?$AA?2?$AA?$CK@ 0000000180010b70     WinNTFileSystem_md.obj
 0002:00001b78       ??_C@_13JOFGPIOO@?$AA?4@   0000000180010b78     WinNTFileSystem_md.obj
 0002:00001b7c       ??_C@_15DDHGOCBH@?$AA?4?$AA?4@ 0000000180010b7c     WinNTFileSystem_md.obj
 0002:00001b88       ??_C@_0CH@PNOGCBMH@Could?5not?5get?5maximum?5component@ 0000000180010b88     WinNTFileSystem_md.obj
 0002:00001bb0       ??_C@_19BKJMDJK@?$AA?2?$AA?2?$AA?4?$AA?2@ 0000000180010bb0     canonicalize_md.obj
 0002:00001bc0       ??_C@_1BC@FBJNHMLC@?$AA?2?$AA?2?$AA?$DP?$AA?2?$AAU?$AAN?$AAC?$AA?$AA@ 0000000180010bc0     canonicalize_md.obj
 0002:00001bd8       ??_C@_1M@DJNCMBIG@?$AA?2?$AA?2?$AA?$DP?$AA?2?$AA?$AA@ 0000000180010bd8     canonicalize_md.obj
 0002:00001be8       ??_C@_0L@BHPPDFMA@Read?5error@ 0000000180010be8     io_util.obj
 0002:00001bf8       ??_C@_0CE@JOEPHHFN@java?1lang?1IndexOutOfBoundsExcep@ 0000000180010bf8     io_util.obj
 0002:00001c20       ??_C@_0M@PJBDJJDJ@Write?5error@ 0000000180010c20     io_util.obj
 0002:00001c30       ??_C@_0CI@HEGLGDKJ@?$CILjava?1lang?1String?$DLLjava?1lang?1S@ 0000000180010c30     io_util.obj
 0002:00001c58       ??_C@_0BO@FDOOLAPO@java?1io?1FileNotFoundException@ 0000000180010c58     io_util.obj
 0002:00001c78       ??_C@_05EGJIMALK@UTF?98@   0000000180010c78     java_props_md.obj
 0002:00001c80       ??_C@_03LIOLIPAH@GBK@      0000000180010c80     java_props_md.obj
 0002:00001c88       ??_C@_07DNCGDNOG@GB18030@  0000000180010c88     java_props_md.obj
 0002:00001c90       ??_C@_05PCINFEFG@MS950@    0000000180010c90     java_props_md.obj
 0002:00001c98       ??_C@_0P@JHCFFHNK@MS950_HKSCS_XP@ 0000000180010c98     java_props_md.obj
 0002:00001ca8       ??_C@_0BH@NKFNLGAB@?2FONTS?2SimSun18030?4ttc@ 0000000180010ca8     java_props_md.obj
 0002:00001cc0       ??_C@_01KDCPPGHE@r@        0000000180010cc0     java_props_md.obj
 0002:00001cc4       ??_C@_04BOOCJOME@ms?$CFd@  0000000180010cc4     java_props_md.obj
 0002:00001ccc       ??_C@_04LDGHIPEL@cp?$CFd@  0000000180010ccc     java_props_md.obj
 0002:00001cd4       ??_C@_01JOAMLHOP@?9@       0000000180010cd4     java_props_md.obj
 0002:00001cd8       ??_C@_05MDLPDLNO@amd64@    0000000180010cd8     java_props_md.obj
 0002:00001ce0       ??_C@_0DO@DIFICBBG@pentium_pro?$CLmmx?5pentium_pro?5pen@ 0000000180010ce0     java_props_md.obj
 0002:00001d20       ??_C@_0CC@BIODACBF@pentium_pro?5pentium?5i486?5i386?5i@ 0000000180010d20     java_props_md.obj
 0002:00001d48       ??_C@_0CC@PPFBHJAM@pentium?$CLmmx?5pentium?5i486?5i386?5i@ 0000000180010d48     java_props_md.obj
 0002:00001d70       ??_C@_0BG@CMPGKFGL@pentium?5i486?5i386?5i86@ 0000000180010d70     java_props_md.obj
 0002:00001d88       ??_C@_0O@MAAOGNKJ@i486?5i386?5i86@ 0000000180010d88     java_props_md.obj
 0002:00001d98       ??_C@_08IPFADFGF@i386?5i86@ 0000000180010d98     java_props_md.obj
 0002:00001da8       ??_C@_0BH@NIHCMEPJ@?$CF?$CK?$FLa?9z?2?9?$FN?$CF1?$FLA?9Z?$FN?$CF?$FLa?9z?$FN@ 0000000180010da8     java_props_md.obj
 0002:00001dc0       ??_C@_02LFNMGJAP@en@       0000000180010dc0     java_props_md.obj
 0002:00001dc4       ??_C@_02PLFPMECB@US@       0000000180010dc4     java_props_md.obj
 0002:00001dc8       ??_C@_02BFDMMJOC@nb@       0000000180010dc8     java_props_md.obj
 0002:00001dcc       ??_C@_02KAJCLHKP@no@       0000000180010dcc     java_props_md.obj
 0002:00001dd0       ??_C@_02NFLNFON@NO@        0000000180010dd0     java_props_md.obj
 0002:00001dd4       ??_C@_02LJIJIGOO@nn@       0000000180010dd4     java_props_md.obj
 0002:00001dd8       ??_C@_02BBMDGADK@NY@       0000000180010dd8     java_props_md.obj
 0002:00001de0       ??_C@_0O@BAKIPCDE@?2kernel32?4dll@ 0000000180010de0     java_props_md.obj
 0002:00001df0       ??_C@_1BM@JEABEHHA@?$AA?2?$AAk?$AAe?$AAr?$AAn?$AAe?$AAl?$AA3?$AA2?$AA?4?$AAd?$AAl?$AAl@ 0000000180010df0     java_props_md.obj
 0002:00001e10       ??_C@_0L@NEBNHFIE@Windows?595@ 0000000180010e10     java_props_md.obj
 0002:00001e20       ??_C@_0L@GBLDALMJ@Windows?598@ 0000000180010e20     java_props_md.obj
 0002:00001e30       ??_C@_0L@DNFOOIFM@Windows?5Me@ 0000000180010e30     java_props_md.obj
 0002:00001e40       ??_C@_0BF@KOJMMOAG@Windows?59X?5?$CIunknown?$CJ@ 0000000180010e40     java_props_md.obj
 0002:00001e58       ??_C@_0L@PJEFFBLH@Windows?5NT@ 0000000180010e58     java_props_md.obj
 0002:00001e68       ??_C@_0N@MEKDBOKB@Windows?52000@ 0000000180010e68     java_props_md.obj
 0002:00001e78       ??_C@_0L@IFICELHB@Windows?5XP@ 0000000180010e78     java_props_md.obj
 0002:00001e88       ??_C@_0N@OPIOENGC@Windows?52003@ 0000000180010e88     java_props_md.obj
 0002:00001e98       ??_C@_0BF@GMBBPJFL@Windows?5NT?5?$CIunknown?$CJ@ 0000000180010e98     java_props_md.obj
 0002:00001eb0       ??_C@_0O@IFKHFILP@Windows?5Vista@ 0000000180010eb0     java_props_md.obj
 0002:00001ec0       ??_C@_09GOHFIPMO@Windows?57@ 0000000180010ec0     java_props_md.obj
 0002:00001ed0       ??_C@_09OJONJDAB@Windows?58@ 0000000180010ed0     java_props_md.obj
 0002:00001ee0       ??_C@_0M@IEJDHGAK@Windows?58?41@ 0000000180010ee0     java_props_md.obj
 0002:00001ef0       ??_C@_0BE@GHBPPLPA@Windows?5Server?52008@ 0000000180010ef0     java_props_md.obj
 0002:00001f08       ??_C@_0BH@ONPOEHKF@Windows?5Server?52008?5R2@ 0000000180010f08     java_props_md.obj
 0002:00001f20       ??_C@_0BE@JMDCHJEN@Windows?5Server?52012@ 0000000180010f20     java_props_md.obj
 0002:00001f38       ??_C@_0BH@GMBCIMKB@Windows?5Server?52012?5R2@ 0000000180010f38     java_props_md.obj
 0002:00001f50       ??_C@_0L@LOGCOBDI@Windows?511@ 0000000180010f50     java_props_md.obj
 0002:00001f60       ??_C@_0L@KHHJNAHJ@Windows?510@ 0000000180010f60     java_props_md.obj
 0002:00001f70       ??_C@_0BE@NBDFFBND@Windows?5Server?52025@ 0000000180010f70     java_props_md.obj
 0002:00001f88       ??_C@_0BE@JOHEMHBE@Windows?5Server?52022@ 0000000180010f88     java_props_md.obj
 0002:00001fa0       ??_C@_0BE@HPMGKAIG@Windows?5Server?52019@ 0000000180010fa0     java_props_md.obj
 0002:00001fb8       ??_C@_0BE@PIFOLMEJ@Windows?5Server?52016@ 0000000180010fb8     java_props_md.obj
 0002:00001fd0       ??_C@_0BC@JFKFADHL@Windows?5?$CIunknown?$CJ@ 0000000180010fd0     java_props_md.obj
 0002:00001fe4       ??_C@_05KBEOJPB@?$CFd?4?$CFd@ 0000000180010fe4     java_props_md.obj
 0002:00001fec       ??_C@_06LADGIEOA@little@   0000000180010fec     java_props_md.obj
 0002:00001ff8       ??_C@_1BC@GGLDBIGJ@?$AAU?$AAS?$AAE?$AAR?$AAN?$AAA?$AAM?$AAE@ 0000000180010ff8     java_props_md.obj
 0002:00002010       ??_C@_1BA@KDMGPDJH@?$AAu?$AAn?$AAk?$AAn?$AAo?$AAw?$AAn@ 0000000180011010     java_props_md.obj
 0002:00002020       ??_C@_17BJPFHBEJ@?$AAC?$AA?3?$AA?2@ 0000000180011020     java_props_md.obj
 0002:00002028       ??_C@_0M@JNHAKOPM@MS950_HKSCS@ 0000000180011028     java_props_md.obj
 0002:00002038       ??_C@_0O@KBEEOPPB@UnicodeLittle@ 0000000180011038     java_props_md.obj
 0002:00002048       ??_C@_01KICIPPFI@?2@       0000000180011048     java_props_md.obj
 0002:0000204c       ??_C@_01ICJEACDI@?$DL@     000000018001104c     java_props_md.obj
 0002:00002050       ??_C@_02PCIJFNDE@?$AN?6@   0000000180011050     java_props_md.obj
 0002:00002058       ??_C@_0BP@GJLHLAKJ@java?1lang?1NullPointerException@ 0000000180011058     jni_util.obj
 0002:00002078       ??_C@_0CJ@ODBKFPOB@java?1lang?1ArrayIndexOutOfBounds@ 0000000180011078     jni_util.obj
 0002:000020a8       ??_C@_0BL@ENCPOIKC@java?1lang?1OutOfMemoryError@ 00000001800110a8     jni_util.obj
 0002:000020c8       ??_C@_0CD@MOHADDFA@java?1lang?1IllegalArgumentExcept@ 00000001800110c8     jni_util.obj
 0002:000020f0       ??_C@_0BI@NBLNIHIB@java?1lang?1InternalError@ 00000001800110f0     jni_util.obj
 0002:00002108       ??_C@_0CB@KCPANAMN@java?1lang?1ClassNotFoundExceptio@ 0000000180011108     jni_util.obj
 0002:00002130       ??_C@_0BE@EBAPEBGJ@java?1io?1IOException@ 0000000180011130     jni_util.obj
 0002:00002144       ??_C@_05DNDNCJEB@?5?$CI?$CFs?$CJ@ 0000000180011144     jni_util.obj
 0002:00002150       ??_C@_0CH@NCPCFFHJ@?$CILjava?1lang?1String?$DL?$CJLjava?1lang?1@ 0000000180011150     jni_util.obj
 0002:00002178       ??_C@_06CMLIEHFC@concat@   0000000180011178     jni_util.obj
 0002:00002180       ??_C@_0BH@GDIHDDN@no?5further?5information@ 0000000180011180     jni_util.obj
 0002:00002198       ??_C@_0CO@NPADHBGE@JNU_CallStaticMethodByName?3?5ill@ 0000000180011198     jni_util.obj
 0002:000021c8       ??_C@_0CJ@MELNKLJP@JNU_CallMethodByNameV?3?5illegal?5@ 00000001800111c8     jni_util.obj
 0002:000021f4       ??_C@_06FALKBLGB@?$DMinit?$DO@ 00000001800111f4     jni_util.obj
 0002:00002200       ??_C@_0CN@KPIMNLJN@NUL?5character?5not?5allowed?5in?5pl@ 0000000180011200     jni_util.obj
 0002:00002230       ??_C@_06FEGJKAJG@8859_1@   0000000180011230     jni_util.obj
 0002:00002238       ??_C@_09KEDHCKDI@ISO8859?91@ 0000000180011238     jni_util.obj
 0002:00002248       ??_C@_09PDECJGAG@ISO8859_1@ 0000000180011248     jni_util.obj
 0002:00002258       ??_C@_0L@GJIJNDEK@ISO?98859?91@ 0000000180011258     jni_util.obj
 0002:00002268       ??_C@_09BGDIBLML@ISO646?9US@ 0000000180011268     jni_util.obj
 0002:00002274       ??_C@_06BFOBJALC@Cp1252@   0000000180011274     jni_util.obj
 0002:00002280       ??_C@_08MIMKAGHL@utf?916le@ 0000000180011280     jni_util.obj
 0002:00002290       ??_C@_0CP@MKKFCJCD@?$CILjava?1lang?1String?$DL?$CJLjava?1nio?1c@ 0000000180011290     jni_util.obj
 0002:000022c0       ??_C@_07ILJBKILD@forName@  00000001800112c0     jni_util.obj
 0002:000022c8       ??_C@_0BJ@ECKJLLIP@java?1nio?1charset?1Charset@ 00000001800112c8     jni_util.obj
 0002:000022e8       ??_C@_0BM@KEODIIBN@platform?5encoding?5undefined@ 00000001800112e8     jni_util.obj
 0002:00002308       ??_C@_0BP@PBJBECGC@?$CILjava?1nio?1charset?1Charset?$DL?$CJ?$FLB@ 0000000180011308     jni_util.obj
 0002:00002328       ??_C@_08LJNJGADH@getBytes@ 0000000180011328     jni_util.obj
 0002:00002338       ??_C@_0CA@JEKLGAML@?$CI?$FLBLjava?1nio?1charset?1Charset?$DL?$CJV@ 0000000180011338     jni_util.obj
 0002:00002358       ??_C@_01HMGJMAIH@B@        0000000180011358     jni_util.obj
 0002:0000235c       ??_C@_05DMGOLBNP@coder@    000000018001135c     jni_util.obj
 0002:00002364       ??_C@_02KCBIMKDL@?$FLB@    0000000180011364     jni_util.obj
 0002:00002368       ??_C@_05MFEJDJP@value@     0000000180011368     jni_util.obj
 0002:00002370       ??_C@_0CC@PDGFIJNH@platform?5encoding?5not?5initializ@ 0000000180011370     jni_util.obj
 0002:00002398       ??_C@_0CG@BPPCDHBK@requested?5array?5size?5exceeds?5VM@ 0000000180011398     jni_util.obj
 0002:000023c0       ??_C@_04HIBGFPH@NULL@      00000001800113c0     jni_util.obj
 0002:000023c8       ??_C@_08JCDFGHAO@toString@ 00000001800113c8     jni_util.obj
 0002:000023d8       ??_C@_0CG@ENHAICHD@JNU_GetFieldByName?3?5illegal?5sig@ 00000001800113d8     jni_util.obj
 0002:00002400       ??_C@_0CG@PKMPNPAI@JNU_SetFieldByName?3?5illegal?5sig@ 0000000180011400     jni_util.obj
 0002:00002428       ??_C@_0CM@FFECHOAH@JNU_GetStaticFieldByName?3?5illeg@ 0000000180011428     jni_util.obj
 0002:00002458       FOLDERID_Profile           0000000180011458     shell32:shguid.obj
 0002:00002478       _pDefaultRawDllMain        0000000180011478     MSVCRT:dll_dllmain.obj
 0002:00002478       _pRawDllMain               0000000180011478     MSVCRT:dll_dllmain.obj
 0002:00002480       _load_config_used          0000000180011480     MSVCRT:loadcfg.obj
 0002:00002680       __volatile_metadata        0000000180011680     <linker-defined>
 0002:000029b8       __rtc_iaa                  00000001800119b8     MSVCRT:initsect.obj
 0002:000029c0       __rtc_izz                  00000001800119c0     MSVCRT:initsect.obj
 0002:000029c8       __rtc_taa                  00000001800119c8     MSVCRT:initsect.obj
 0002:000029d0       __rtc_tzz                  00000001800119d0     MSVCRT:initsect.obj
 0002:000070bc       __IMPORT_DESCRIPTOR_jvm    00000001800160bc     jvm:jvm.dll
 0002:000070d0       __IMPORT_DESCRIPTOR_ADVAPI32 00000001800160d0     advapi32:ADVAPI32.dll
 0002:000070e4       __IMPORT_DESCRIPTOR_ole32  00000001800160e4     ole32:ole32.dll
 0002:000070f8       __IMPORT_DESCRIPTOR_SHELL32 00000001800160f8     shell32:SHELL32.dll
 0002:0000710c       __IMPORT_DESCRIPTOR_VERSION 000000018001610c     version:VERSION.dll
 0002:00007120       __IMPORT_DESCRIPTOR_KERNEL32 0000000180016120     kernel32:KERNEL32.dll
 0002:00007134       __IMPORT_DESCRIPTOR_VCRUNTIME140 0000000180016134     vcruntime:VCRUNTIME140.dll
 0002:00007148       __IMPORT_DESCRIPTOR_api-ms-win-crt-heap-l1-1-0 0000000180016148     ucrt:api-ms-win-crt-heap-l1-1-0.dll
 0002:0000715c       __IMPORT_DESCRIPTOR_api-ms-win-crt-string-l1-1-0 000000018001615c     ucrt:api-ms-win-crt-string-l1-1-0.dll
 0002:00007170       __IMPORT_DESCRIPTOR_api-ms-win-crt-stdio-l1-1-0 0000000180016170     ucrt:api-ms-win-crt-stdio-l1-1-0.dll
 0002:00007184       __IMPORT_DESCRIPTOR_api-ms-win-crt-convert-l1-1-0 0000000180016184     ucrt:api-ms-win-crt-convert-l1-1-0.dll
 0002:00007198       __IMPORT_DESCRIPTOR_api-ms-win-crt-runtime-l1-1-0 0000000180016198     ucrt:api-ms-win-crt-runtime-l1-1-0.dll
 0002:000071ac       __IMPORT_DESCRIPTOR_api-ms-win-crt-filesystem-l1-1-0 00000001800161ac     ucrt:api-ms-win-crt-filesystem-l1-1-0.dll
 0002:000071c0       __IMPORT_DESCRIPTOR_api-ms-win-crt-environment-l1-1-0 00000001800161c0     ucrt:api-ms-win-crt-environment-l1-1-0.dll
 0002:000071d4       __NULL_IMPORT_DESCRIPTOR   00000001800161d4     jvm:jvm.dll
 0003:00000240       monthsType                 0000000180019240     HostLocaleProviderAdapter_md.obj
 0003:00000278       sMonthsType                0000000180019278     HostLocaleProviderAdapter_md.obj
 0003:000002b0       wDaysType                  00000001800192b0     HostLocaleProviderAdapter_md.obj
 0003:000002d0       sWDaysType                 00000001800192d0     HostLocaleProviderAdapter_md.obj
 0003:000002f0       ampmType                   00000001800192f0     HostLocaleProviderAdapter_md.obj
 0003:00000300       fixes                      0000000180019300     HostLocaleProviderAdapter_md.obj
 0003:00000c70       _fltused                   0000000180019c70     MSVCRT:fltused.obj
 0003:00000c80       __security_cookie          0000000180019c80     MSVCRT:gs_cookie.obj
 0003:00000cc0       __security_cookie_complement 0000000180019cc0     MSVCRT:gs_cookie.obj
 0003:00000cd0       __scrt_native_dllmain_reason 0000000180019cd0     MSVCRT:utility.obj
 0003:00000cd8       __isa_inverted             0000000180019cd8     MSVCRT:cpu_disp.obj
 0003:00000ce0       __isa_available            0000000180019ce0     MSVCRT:cpu_disp.obj
 0003:00000ce4       __isa_enabled              0000000180019ce4     MSVCRT:cpu_disp.obj
 0003:00000ce8       __memset_fast_string_threshold 0000000180019ce8     MSVCRT:cpu_disp.obj
 0003:00000cf0       __memset_nt_threshold      0000000180019cf0     MSVCRT:cpu_disp.obj
 0003:00000d00       __scrt_ucrt_dll_is_in_use  0000000180019d00     MSVCRT:ucrt_stubs.obj
 0003:00000d10       initialized                0000000180019d10     HostLocaleProviderAdapter_md.obj
 0003:00001430       ?__type_info_root_node@@3U__type_info_node@@A 000000018001a430     MSVCRT:tncleanup.obj
 0003:00001440       __scrt_current_native_startup_state 000000018001a440     MSVCRT:utility.obj
 0003:00001448       __scrt_native_startup_lock 000000018001a448     MSVCRT:utility.obj
 0003:00001488       __scrt_debugger_hook_flag  000000018001a488     MSVCRT:utility_desktop.obj
 0003:0000148c       __avx10_version            000000018001a48c     MSVCRT:cpu_disp.obj
 0003:00001490       __favor                    000000018001a490     MSVCRT:cpu_disp.obj
 0003:00001498       ?_OptionsStorage@?1??__local_stdio_scanf_options@@9@9 000000018001a498     <common>
 0003:000014a0       raf_fd                     000000018001a4a0     <common>
 0003:000014a8       ?_OptionsStorage@?1??__local_stdio_printf_options@@9@9 000000018001a4a8     <common>
 0003:000014b0       pEnumCalendarInfoExEx      000000018001a4b0     <common>
 0003:000014b8       pGetCalendarInfoEx         000000018001a4b8     <common>
 0003:000014c0       pGetLocaleInfoEx           000000018001a4c0     <common>
 0003:000014c8       fos_fd                     000000018001a4c8     <common>
 0003:000014d0       fis_fd                     000000018001a4d0     <common>
 0003:000014d8       IO_append_fdID             000000018001a4d8     <common>
 0003:000014e0       IO_handle_fdID             000000018001a4e0     <common>
 0003:000014e8       IO_fd_fdID                 000000018001a4e8     <common>
 0003:000014f0       __dyn_tls_init_callback    000000018001a4f0     <common>

 entry point at        0001:0000d400

 Static symbols

 0000:fffe2000       .debug$S                   0000000180000000     java.exp
 0000:fffe2000       .debug$S                   0000000180000000     vcruntime:VCRUNTIME140.dll
 0000:fffe2000       .debug$S                   0000000180000000     vcruntime:VCRUNTIME140.dll
 0000:fffe2000       .debug$S                   0000000180000000     vcruntime:VCRUNTIME140.dll
 0000:fffe2000       .debug$S                   0000000180000000     vcruntime:VCRUNTIME140.dll
 0000:fffe2000       .debug$S                   0000000180000000     vcruntime:VCRUNTIME140.dll
 0000:fffe2000       .debug$S                   0000000180000000     vcruntime:VCRUNTIME140.dll
 0000:fffe2000       .debug$S                   0000000180000000     vcruntime:VCRUNTIME140.dll
 0000:fffe2000       .debug$S                   0000000180000000     vcruntime:VCRUNTIME140.dll
 0000:fffe2000       .debug$S                   0000000180000000     vcruntime:VCRUNTIME140.dll
 0000:fffe2000       .debug$S                   0000000180000000     vcruntime:VCRUNTIME140.dll
 0000:fffe2000       .debug$S                   0000000180000000     ucrt:api-ms-win-crt-convert-l1-1-0.dll
 0000:fffe2000       .debug$S                   0000000180000000     ucrt:api-ms-win-crt-convert-l1-1-0.dll
 0000:fffe2000       .debug$S                   0000000180000000     ucrt:api-ms-win-crt-convert-l1-1-0.dll
 0000:fffe2000       .debug$S                   0000000180000000     ucrt:api-ms-win-crt-environment-l1-1-0.dll
 0000:fffe2000       .debug$S                   0000000180000000     ucrt:api-ms-win-crt-environment-l1-1-0.dll
 0000:fffe2000       .debug$S                   0000000180000000     ucrt:api-ms-win-crt-environment-l1-1-0.dll
 0000:fffe2000       .debug$S                   0000000180000000     ucrt:api-ms-win-crt-filesystem-l1-1-0.dll
 0000:fffe2000       .debug$S                   0000000180000000     ucrt:api-ms-win-crt-filesystem-l1-1-0.dll
 0000:fffe2000       .debug$S                   0000000180000000     ucrt:api-ms-win-crt-heap-l1-1-0.dll
 0000:fffe2000       .debug$S                   0000000180000000     ucrt:api-ms-win-crt-heap-l1-1-0.dll
 0000:fffe2000       .debug$S                   0000000180000000     ucrt:api-ms-win-crt-heap-l1-1-0.dll
 0000:fffe2000       .debug$S                   0000000180000000     ucrt:api-ms-win-crt-runtime-l1-1-0.dll
 0000:fffe2000       .debug$S                   0000000180000000     ucrt:api-ms-win-crt-runtime-l1-1-0.dll
 0000:fffe2000       .debug$S                   0000000180000000     ucrt:api-ms-win-crt-runtime-l1-1-0.dll
 0000:fffe2000       .debug$S                   0000000180000000     ucrt:api-ms-win-crt-runtime-l1-1-0.dll
 0000:fffe2000       .debug$S                   0000000180000000     ucrt:api-ms-win-crt-runtime-l1-1-0.dll
 0000:fffe2000       .debug$S                   0000000180000000     ucrt:api-ms-win-crt-runtime-l1-1-0.dll
 0000:fffe2000       .debug$S                   0000000180000000     ucrt:api-ms-win-crt-runtime-l1-1-0.dll
 0000:fffe2000       .debug$S                   0000000180000000     ucrt:api-ms-win-crt-runtime-l1-1-0.dll
 0000:fffe2000       .debug$S                   0000000180000000     ucrt:api-ms-win-crt-runtime-l1-1-0.dll
 0000:fffe2000       .debug$S                   0000000180000000     ucrt:api-ms-win-crt-runtime-l1-1-0.dll
 0000:fffe2000       .debug$S                   0000000180000000     ucrt:api-ms-win-crt-runtime-l1-1-0.dll
 0000:fffe2000       .debug$S                   0000000180000000     ucrt:api-ms-win-crt-runtime-l1-1-0.dll
 0000:fffe2000       .debug$S                   0000000180000000     ucrt:api-ms-win-crt-runtime-l1-1-0.dll
 0000:fffe2000       .debug$S                   0000000180000000     ucrt:api-ms-win-crt-runtime-l1-1-0.dll
 0000:fffe2000       .debug$S                   0000000180000000     ucrt:api-ms-win-crt-stdio-l1-1-0.dll
 0000:fffe2000       .debug$S                   0000000180000000     ucrt:api-ms-win-crt-stdio-l1-1-0.dll
 0000:fffe2000       .debug$S                   0000000180000000     ucrt:api-ms-win-crt-stdio-l1-1-0.dll
 0000:fffe2000       .debug$S                   0000000180000000     ucrt:api-ms-win-crt-stdio-l1-1-0.dll
 0000:fffe2000       .debug$S                   0000000180000000     ucrt:api-ms-win-crt-stdio-l1-1-0.dll
 0000:fffe2000       .debug$S                   0000000180000000     ucrt:api-ms-win-crt-stdio-l1-1-0.dll
 0000:fffe2000       .debug$S                   0000000180000000     ucrt:api-ms-win-crt-stdio-l1-1-0.dll
 0000:fffe2000       .debug$S                   0000000180000000     ucrt:api-ms-win-crt-stdio-l1-1-0.dll
 0000:fffe2000       .debug$S                   0000000180000000     ucrt:api-ms-win-crt-string-l1-1-0.dll
 0000:fffe2000       .debug$S                   0000000180000000     ucrt:api-ms-win-crt-string-l1-1-0.dll
 0000:fffe2000       .debug$S                   0000000180000000     ucrt:api-ms-win-crt-string-l1-1-0.dll
 0000:fffe2000       .debug$S                   0000000180000000     ucrt:api-ms-win-crt-string-l1-1-0.dll
 0000:fffe2000       .debug$S                   0000000180000000     ucrt:api-ms-win-crt-string-l1-1-0.dll
 0000:fffe2000       .debug$S                   0000000180000000     ucrt:api-ms-win-crt-string-l1-1-0.dll
 0000:fffe2000       .debug$S                   0000000180000000     ucrt:api-ms-win-crt-string-l1-1-0.dll
 0000:fffe2000       .debug$S                   0000000180000000     ucrt:api-ms-win-crt-string-l1-1-0.dll
 0000:fffe2000       .debug$S                   0000000180000000     ucrt:api-ms-win-crt-string-l1-1-0.dll
 0000:fffe2000       .debug$S                   0000000180000000     ucrt:api-ms-win-crt-string-l1-1-0.dll
 0000:fffe2000       .debug$S                   0000000180000000     ucrt:api-ms-win-crt-string-l1-1-0.dll
 0000:fffe2000       .debug$S                   0000000180000000     ucrt:api-ms-win-crt-string-l1-1-0.dll
 0000:fffe2000       .debug$S                   0000000180000000     ucrt:api-ms-win-crt-string-l1-1-0.dll
 0000:fffe2000       .debug$S                   0000000180000000     ucrt:api-ms-win-crt-string-l1-1-0.dll
 0000:fffe2000       .debug$S                   0000000180000000     ucrt:api-ms-win-crt-string-l1-1-0.dll
 0000:fffe2000       .debug$S                   0000000180000000     ucrt:api-ms-win-crt-string-l1-1-0.dll
 0000:fffe2000       .debug$S                   0000000180000000     advapi32:ADVAPI32.dll
 0000:fffe2000       .debug$S                   0000000180000000     advapi32:ADVAPI32.dll
 0000:fffe2000       .debug$S                   0000000180000000     advapi32:ADVAPI32.dll
 0000:fffe2000       .debug$S                   0000000180000000     advapi32:ADVAPI32.dll
 0000:fffe2000       .debug$S                   0000000180000000     advapi32:ADVAPI32.dll
 0000:fffe2000       .debug$S                   0000000180000000     advapi32:ADVAPI32.dll
 0000:fffe2000       .debug$S                   0000000180000000     advapi32:ADVAPI32.dll
 0000:fffe2000       .debug$S                   0000000180000000     advapi32:ADVAPI32.dll
 0000:fffe2000       .debug$S                   0000000180000000     advapi32:ADVAPI32.dll
 0000:fffe2000       .debug$S                   0000000180000000     advapi32:ADVAPI32.dll
 0000:fffe2000       .debug$S                   0000000180000000     advapi32:ADVAPI32.dll
 0000:fffe2000       .debug$S                   0000000180000000     advapi32:ADVAPI32.dll
 0000:fffe2000       .debug$S                   0000000180000000     advapi32:ADVAPI32.dll
 0000:fffe2000       .debug$S                   0000000180000000     advapi32:ADVAPI32.dll
 0000:fffe2000       .debug$S                   0000000180000000     advapi32:ADVAPI32.dll
 0000:fffe2000       .debug$S                   0000000180000000     kernel32:KERNEL32.dll
 0000:fffe2000       .debug$S                   0000000180000000     kernel32:KERNEL32.dll
 0000:fffe2000       .debug$S                   0000000180000000     kernel32:KERNEL32.dll
 0000:fffe2000       .debug$S                   0000000180000000     kernel32:KERNEL32.dll
 0000:fffe2000       .debug$S                   0000000180000000     kernel32:KERNEL32.dll
 0000:fffe2000       .debug$S                   0000000180000000     kernel32:KERNEL32.dll
 0000:fffe2000       .debug$S                   0000000180000000     kernel32:KERNEL32.dll
 0000:fffe2000       .debug$S                   0000000180000000     kernel32:KERNEL32.dll
 0000:fffe2000       .debug$S                   0000000180000000     kernel32:KERNEL32.dll
 0000:fffe2000       .debug$S                   0000000180000000     kernel32:KERNEL32.dll
 0000:fffe2000       .debug$S                   0000000180000000     kernel32:KERNEL32.dll
 0000:fffe2000       .debug$S                   0000000180000000     kernel32:KERNEL32.dll
 0000:fffe2000       .debug$S                   0000000180000000     kernel32:KERNEL32.dll
 0000:fffe2000       .debug$S                   0000000180000000     kernel32:KERNEL32.dll
 0000:fffe2000       .debug$S                   0000000180000000     kernel32:KERNEL32.dll
 0000:fffe2000       .debug$S                   0000000180000000     kernel32:KERNEL32.dll
 0000:fffe2000       .debug$S                   0000000180000000     kernel32:KERNEL32.dll
 0000:fffe2000       .debug$S                   0000000180000000     kernel32:KERNEL32.dll
 0000:fffe2000       .debug$S                   0000000180000000     kernel32:KERNEL32.dll
 0000:fffe2000       .debug$S                   0000000180000000     kernel32:KERNEL32.dll
 0000:fffe2000       .debug$S                   0000000180000000     kernel32:KERNEL32.dll
 0000:fffe2000       .debug$S                   0000000180000000     kernel32:KERNEL32.dll
 0000:fffe2000       .debug$S                   0000000180000000     kernel32:KERNEL32.dll
 0000:fffe2000       .debug$S                   0000000180000000     kernel32:KERNEL32.dll
 0000:fffe2000       .debug$S                   0000000180000000     kernel32:KERNEL32.dll
 0000:fffe2000       .debug$S                   0000000180000000     kernel32:KERNEL32.dll
 0000:fffe2000       .debug$S                   0000000180000000     kernel32:KERNEL32.dll
 0000:fffe2000       .debug$S                   0000000180000000     kernel32:KERNEL32.dll
 0000:fffe2000       .debug$S                   0000000180000000     kernel32:KERNEL32.dll
 0000:fffe2000       .debug$S                   0000000180000000     kernel32:KERNEL32.dll
 0000:fffe2000       .debug$S                   0000000180000000     kernel32:KERNEL32.dll
 0000:fffe2000       .debug$S                   0000000180000000     kernel32:KERNEL32.dll
 0000:fffe2000       .debug$S                   0000000180000000     kernel32:KERNEL32.dll
 0000:fffe2000       .debug$S                   0000000180000000     kernel32:KERNEL32.dll
 0000:fffe2000       .debug$S                   0000000180000000     kernel32:KERNEL32.dll
 0000:fffe2000       .debug$S                   0000000180000000     kernel32:KERNEL32.dll
 0000:fffe2000       .debug$S                   0000000180000000     kernel32:KERNEL32.dll
 0000:fffe2000       .debug$S                   0000000180000000     kernel32:KERNEL32.dll
 0000:fffe2000       .debug$S                   0000000180000000     kernel32:KERNEL32.dll
 0000:fffe2000       .debug$S                   0000000180000000     kernel32:KERNEL32.dll
 0000:fffe2000       .debug$S                   0000000180000000     kernel32:KERNEL32.dll
 0000:fffe2000       .debug$S                   0000000180000000     kernel32:KERNEL32.dll
 0000:fffe2000       .debug$S                   0000000180000000     kernel32:KERNEL32.dll
 0000:fffe2000       .debug$S                   0000000180000000     kernel32:KERNEL32.dll
 0000:fffe2000       .debug$S                   0000000180000000     kernel32:KERNEL32.dll
 0000:fffe2000       .debug$S                   0000000180000000     kernel32:KERNEL32.dll
 0000:fffe2000       .debug$S                   0000000180000000     kernel32:KERNEL32.dll
 0000:fffe2000       .debug$S                   0000000180000000     kernel32:KERNEL32.dll
 0000:fffe2000       .debug$S                   0000000180000000     kernel32:KERNEL32.dll
 0000:fffe2000       .debug$S                   0000000180000000     kernel32:KERNEL32.dll
 0000:fffe2000       .debug$S                   0000000180000000     kernel32:KERNEL32.dll
 0000:fffe2000       .debug$S                   0000000180000000     kernel32:KERNEL32.dll
 0000:fffe2000       .debug$S                   0000000180000000     kernel32:KERNEL32.dll
 0000:fffe2000       .debug$S                   0000000180000000     kernel32:KERNEL32.dll
 0000:fffe2000       .debug$S                   0000000180000000     kernel32:KERNEL32.dll
 0000:fffe2000       .debug$S                   0000000180000000     kernel32:KERNEL32.dll
 0000:fffe2000       .debug$S                   0000000180000000     kernel32:KERNEL32.dll
 0000:fffe2000       .debug$S                   0000000180000000     kernel32:KERNEL32.dll
 0000:fffe2000       .debug$S                   0000000180000000     kernel32:KERNEL32.dll
 0000:fffe2000       .debug$S                   0000000180000000     kernel32:KERNEL32.dll
 0000:fffe2000       .debug$S                   0000000180000000     kernel32:KERNEL32.dll
 0000:fffe2000       .debug$S                   0000000180000000     kernel32:KERNEL32.dll
 0000:fffe2000       .debug$S                   0000000180000000     kernel32:KERNEL32.dll
 0000:fffe2000       .debug$S                   0000000180000000     kernel32:KERNEL32.dll
 0000:fffe2000       .debug$S                   0000000180000000     kernel32:KERNEL32.dll
 0000:fffe2000       .debug$S                   0000000180000000     kernel32:KERNEL32.dll
 0000:fffe2000       .debug$S                   0000000180000000     kernel32:KERNEL32.dll
 0000:fffe2000       .debug$S                   0000000180000000     kernel32:KERNEL32.dll
 0000:fffe2000       .debug$S                   0000000180000000     kernel32:KERNEL32.dll
 0000:fffe2000       .debug$S                   0000000180000000     kernel32:KERNEL32.dll
 0000:fffe2000       .debug$S                   0000000180000000     kernel32:KERNEL32.dll
 0000:fffe2000       .debug$S                   0000000180000000     kernel32:KERNEL32.dll
 0000:fffe2000       .debug$S                   0000000180000000     kernel32:KERNEL32.dll
 0000:fffe2000       .debug$S                   0000000180000000     kernel32:KERNEL32.dll
 0000:fffe2000       .debug$S                   0000000180000000     kernel32:KERNEL32.dll
 0000:fffe2000       .debug$S                   0000000180000000     kernel32:KERNEL32.dll
 0000:fffe2000       .debug$S                   0000000180000000     kernel32:KERNEL32.dll
 0000:fffe2000       .debug$S                   0000000180000000     kernel32:KERNEL32.dll
 0000:fffe2000       .debug$S                   0000000180000000     kernel32:KERNEL32.dll
 0000:fffe2000       .debug$S                   0000000180000000     kernel32:KERNEL32.dll
 0000:fffe2000       .debug$S                   0000000180000000     kernel32:KERNEL32.dll
 0000:fffe2000       .debug$S                   0000000180000000     kernel32:KERNEL32.dll
 0000:fffe2000       .debug$S                   0000000180000000     kernel32:KERNEL32.dll
 0000:fffe2000       .debug$S                   0000000180000000     kernel32:KERNEL32.dll
 0000:fffe2000       .debug$S                   0000000180000000     kernel32:KERNEL32.dll
 0000:fffe2000       .debug$S                   0000000180000000     kernel32:KERNEL32.dll
 0000:fffe2000       .debug$S                   0000000180000000     kernel32:KERNEL32.dll
 0000:fffe2000       .debug$S                   0000000180000000     kernel32:KERNEL32.dll
 0000:fffe2000       .debug$S                   0000000180000000     kernel32:KERNEL32.dll
 0000:fffe2000       .debug$S                   0000000180000000     kernel32:KERNEL32.dll
 0000:fffe2000       .debug$S                   0000000180000000     kernel32:KERNEL32.dll
 0000:fffe2000       .debug$S                   0000000180000000     kernel32:KERNEL32.dll
 0000:fffe2000       .debug$S                   0000000180000000     kernel32:KERNEL32.dll
 0000:fffe2000       .debug$S                   0000000180000000     kernel32:KERNEL32.dll
 0000:fffe2000       .debug$S                   0000000180000000     kernel32:KERNEL32.dll
 0000:fffe2000       .debug$S                   0000000180000000     kernel32:KERNEL32.dll
 0000:fffe2000       .debug$S                   0000000180000000     kernel32:KERNEL32.dll
 0000:fffe2000       .debug$S                   0000000180000000     kernel32:KERNEL32.dll
 0000:fffe2000       .debug$S                   0000000180000000     kernel32:KERNEL32.dll
 0000:fffe2000       .debug$S                   0000000180000000     ole32:ole32.dll
 0000:fffe2000       .debug$S                   0000000180000000     shell32:SHELL32.dll
 0000:fffe2000       .debug$S                   0000000180000000     version:VERSION.dll
 0000:fffe2000       .debug$S                   0000000180000000     version:VERSION.dll
 0000:fffe2000       .debug$S                   0000000180000000     version:VERSION.dll
 0000:fffe2000       .debug$S                   0000000180000000     jvm:jvm.dll
 0000:fffe2000       .debug$S                   0000000180000000     jvm:jvm.dll
 0000:fffe2000       .debug$S                   0000000180000000     jvm:jvm.dll
 0000:fffe2000       .debug$S                   0000000180000000     jvm:jvm.dll
 0000:fffe2000       .debug$S                   0000000180000000     jvm:jvm.dll
 0000:fffe2000       .debug$S                   0000000180000000     jvm:jvm.dll
 0000:fffe2000       .debug$S                   0000000180000000     jvm:jvm.dll
 0000:fffe2000       .debug$S                   0000000180000000     jvm:jvm.dll
 0000:fffe2000       .debug$S                   0000000180000000     jvm:jvm.dll
 0000:fffe2000       .debug$S                   0000000180000000     jvm:jvm.dll
 0000:fffe2000       .debug$S                   0000000180000000     jvm:jvm.dll
 0000:fffe2000       .debug$S                   0000000180000000     jvm:jvm.dll
 0000:fffe2000       .debug$S                   0000000180000000     jvm:jvm.dll
 0000:fffe2000       .debug$S                   0000000180000000     jvm:jvm.dll
 0000:fffe2000       .debug$S                   0000000180000000     jvm:jvm.dll
 0000:fffe2000       .debug$S                   0000000180000000     jvm:jvm.dll
 0000:fffe2000       .debug$S                   0000000180000000     jvm:jvm.dll
 0000:fffe2000       .debug$S                   0000000180000000     jvm:jvm.dll
 0000:fffe2000       .debug$S                   0000000180000000     jvm:jvm.dll
 0000:fffe2000       .debug$S                   0000000180000000     jvm:jvm.dll
 0000:fffe2000       .debug$S                   0000000180000000     jvm:jvm.dll
 0000:fffe2000       .debug$S                   0000000180000000     jvm:jvm.dll
 0000:fffe2000       .debug$S                   0000000180000000     jvm:jvm.dll
 0000:fffe2000       .debug$S                   0000000180000000     jvm:jvm.dll
 0000:fffe2000       .debug$S                   0000000180000000     jvm:jvm.dll
 0000:fffe2000       .debug$S                   0000000180000000     jvm:jvm.dll
 0000:fffe2000       .debug$S                   0000000180000000     jvm:jvm.dll
 0000:fffe2000       .debug$S                   0000000180000000     jvm:jvm.dll
 0000:fffe2000       .debug$S                   0000000180000000     jvm:jvm.dll
 0000:fffe2000       .debug$S                   0000000180000000     jvm:jvm.dll
 0000:fffe2000       .debug$S                   0000000180000000     jvm:jvm.dll
 0000:fffe2000       .debug$S                   0000000180000000     jvm:jvm.dll
 0000:fffe2000       .debug$S                   0000000180000000     jvm:jvm.dll
 0000:fffe2000       .debug$S                   0000000180000000     jvm:jvm.dll
 0000:fffe2000       .debug$S                   0000000180000000     jvm:jvm.dll
 0000:fffe2000       .debug$S                   0000000180000000     jvm:jvm.dll
 0000:fffe2000       .debug$S                   0000000180000000     jvm:jvm.dll
 0000:fffe2000       .debug$S                   0000000180000000     jvm:jvm.dll
 0000:fffe2000       .debug$S                   0000000180000000     jvm:jvm.dll
 0000:fffe2000       .debug$S                   0000000180000000     jvm:jvm.dll
 0000:fffe2000       .debug$S                   0000000180000000     jvm:jvm.dll
 0000:fffe2000       .debug$S                   0000000180000000     jvm:jvm.dll
 0000:fffe2000       .debug$S                   0000000180000000     jvm:jvm.dll
 0000:fffe2000       .debug$S                   0000000180000000     jvm:jvm.dll
 0000:fffe2000       .debug$S                   0000000180000000     jvm:jvm.dll
 0000:fffe2000       .debug$S                   0000000180000000     jvm:jvm.dll
 0000:fffe2000       .debug$S                   0000000180000000     jvm:jvm.dll
 0000:fffe2000       .debug$S                   0000000180000000     jvm:jvm.dll
 0000:fffe2000       .debug$S                   0000000180000000     jvm:jvm.dll
 0000:fffe2000       .debug$S                   0000000180000000     jvm:jvm.dll
 0000:fffe2000       .debug$S                   0000000180000000     jvm:jvm.dll
 0000:fffe2000       .debug$S                   0000000180000000     jvm:jvm.dll
 0000:fffe2000       .debug$S                   0000000180000000     jvm:jvm.dll
 0000:fffe2000       .debug$S                   0000000180000000     jvm:jvm.dll
 0000:fffe2000       .debug$S                   0000000180000000     jvm:jvm.dll
 0000:fffe2000       .debug$S                   0000000180000000     jvm:jvm.dll
 0000:fffe2000       .debug$S                   0000000180000000     jvm:jvm.dll
 0000:fffe2000       .debug$S                   0000000180000000     jvm:jvm.dll
 0000:fffe2000       .debug$S                   0000000180000000     jvm:jvm.dll
 0000:fffe2000       .debug$S                   0000000180000000     jvm:jvm.dll
 0000:fffe2000       .debug$S                   0000000180000000     jvm:jvm.dll
 0000:fffe2000       .debug$S                   0000000180000000     jvm:jvm.dll
 0000:fffe2000       .debug$S                   0000000180000000     jvm:jvm.dll
 0000:fffe2000       .debug$S                   0000000180000000     jvm:jvm.dll
 0000:fffe2000       .debug$S                   0000000180000000     jvm:jvm.dll
 0000:fffe2000       .debug$S                   0000000180000000     jvm:jvm.dll
 0000:fffe2000       .debug$S                   0000000180000000     jvm:jvm.dll
 0000:fffe2000       .debug$S                   0000000180000000     jvm:jvm.dll
 0000:fffe2000       .debug$S                   0000000180000000     jvm:jvm.dll
 0000:fffe2000       .debug$S                   0000000180000000     jvm:jvm.dll
 0000:fffe2000       .debug$S                   0000000180000000     jvm:jvm.dll
 0000:fffe2000       .debug$S                   0000000180000000     jvm:jvm.dll
 0000:fffe2000       .debug$S                   0000000180000000     jvm:jvm.dll
 0000:fffe2000       .debug$S                   0000000180000000     jvm:jvm.dll
 0000:fffe2000       .debug$S                   0000000180000000     jvm:jvm.dll
 0000:fffe2000       .debug$S                   0000000180000000     jvm:jvm.dll
 0000:fffe2000       .debug$S                   0000000180000000     jvm:jvm.dll
 0000:fffe2000       .debug$S                   0000000180000000     jvm:jvm.dll
 0000:fffe2000       .debug$S                   0000000180000000     jvm:jvm.dll
 0000:fffe2000       .debug$S                   0000000180000000     jvm:jvm.dll
 0000:fffe2000       .debug$S                   0000000180000000     jvm:jvm.dll
 0000:fffe2000       .debug$S                   0000000180000000     jvm:jvm.dll
 0000:fffe2000       .debug$S                   0000000180000000     jvm:jvm.dll
 0000:fffe2000       .debug$S                   0000000180000000     jvm:jvm.dll
 0000:fffe2000       .debug$S                   0000000180000000     jvm:jvm.dll
 0000:fffe2000       .debug$S                   0000000180000000     jvm:jvm.dll
 0000:fffe2000       .debug$S                   0000000180000000     jvm:jvm.dll
 0000:fffe2000       .debug$S                   0000000180000000     jvm:jvm.dll
 0000:fffe2000       .debug$S                   0000000180000000     jvm:jvm.dll
 0000:fffe2000       .debug$S                   0000000180000000     jvm:jvm.dll
 0000:fffe2000       .debug$S                   0000000180000000     jvm:jvm.dll
 0000:fffe2000       .debug$S                   0000000180000000     jvm:jvm.dll
 0000:fffe2000       .debug$S                   0000000180000000     jvm:jvm.dll
 0000:fffe2000       .debug$S                   0000000180000000     jvm:jvm.dll
 0000:fffe2000       .debug$S                   0000000180000000     jvm:jvm.dll
 0000:fffe2000       .debug$S                   0000000180000000     jvm:jvm.dll
 0000:fffe2000       .debug$S                   0000000180000000     jvm:jvm.dll
 0000:fffe2000       .debug$S                   0000000180000000     jvm:jvm.dll
 0000:fffe2000       .debug$S                   0000000180000000     jvm:jvm.dll
 0000:fffe2000       .debug$S                   0000000180000000     jvm:jvm.dll
 0000:fffe2000       .debug$S                   0000000180000000     jvm:jvm.dll
 0000:fffe2000       .debug$S                   0000000180000000     jvm:jvm.dll
 0000:fffe2000       .debug$S                   0000000180000000     jvm:jvm.dll
 0000:fffe2000       .debug$S                   0000000180000000     jvm:jvm.dll
 0000:fffe2000       .debug$S                   0000000180000000     jvm:jvm.dll
 0000:fffe2000       .debug$S                   0000000180000000     jvm:jvm.dll
 0000:fffe2000       .debug$S                   0000000180000000     jvm:jvm.dll
 0000:fffe2000       .debug$S                   0000000180000000     jvm:jvm.dll
 0000:fffe2000       .debug$S                   0000000180000000     jvm:jvm.dll
 0000:fffe2000       .debug$S                   0000000180000000     jvm:jvm.dll
 0000:fffe2000       .debug$S                   0000000180000000     jvm:jvm.dll
 0000:fffe2000       .debug$S                   0000000180000000     jvm:jvm.dll
 0000:fffe2000       .debug$S                   0000000180000000     jvm:jvm.dll
 0000:fffe2000       .debug$S                   0000000180000000     jvm:jvm.dll
 0000:fffe2000       .debug$S                   0000000180000000     jvm:jvm.dll
 0000:fffe2000       .debug$S                   0000000180000000     jvm:jvm.dll
 0000:fffe2000       .debug$S                   0000000180000000     jvm:jvm.dll
 0000:fffe2000       .debug$S                   0000000180000000     jvm:jvm.dll
 0000:fffe2000       .debug$S                   0000000180000000     jvm:jvm.dll
 0000:fffe2000       .debug$S                   0000000180000000     jvm:jvm.dll
 0000:fffe2000       .debug$S                   0000000180000000     jvm:jvm.dll
 0000:fffe2000       .debug$S                   0000000180000000     jvm:jvm.dll
 0000:fffe2000       .debug$S                   0000000180000000     jvm:jvm.dll
 0000:fffe2000       .debug$S                   0000000180000000     jvm:jvm.dll
 0000:fffe2000       .debug$S                   0000000180000000     jvm:jvm.dll
 0000:fffe2000       .debug$S                   0000000180000000     jvm:jvm.dll
 0000:fffe2000       .debug$S                   0000000180000000     jvm:jvm.dll
 0000:fffe2000       .debug$S                   0000000180000000     jvm:jvm.dll
 0000:fffe2000       .debug$S                   0000000180000000     jvm:jvm.dll
 0000:fffe2000       .debug$S                   0000000180000000     jvm:jvm.dll
 0000:fffe2000       .debug$S                   0000000180000000     jvm:jvm.dll
 0000:fffe2000       .debug$S                   0000000180000000     jvm:jvm.dll
 0000:fffe2000       .debug$S                   0000000180000000     jvm:jvm.dll
 0000:fffe2000       .debug$S                   0000000180000000     jvm:jvm.dll
 0000:fffe2000       .debug$S                   0000000180000000     jvm:jvm.dll
 0000:fffe2000       .debug$S                   0000000180000000     jvm:jvm.dll
 0000:fffe2000       .debug$S                   0000000180000000     jvm:jvm.dll
 0000:fffe2000       .debug$S                   0000000180000000     jvm:jvm.dll
 0000:fffe2000       .debug$S                   0000000180000000     jvm:jvm.dll
 0000:fffe2000       .debug$S                   0000000180000000     jvm:jvm.dll
 0000:fffe2000       .debug$S                   0000000180000000     jvm:jvm.dll
 0000:fffe2000       .debug$S                   0000000180000000     jvm:jvm.dll
 0000:fffe2000       .debug$S                   0000000180000000     jvm:jvm.dll
 0000:fffe2000       .debug$S                   0000000180000000     jvm:jvm.dll
 0000:fffe2000       .debug$S                   0000000180000000     jvm:jvm.dll
 0000:fffe2000       .debug$S                   0000000180000000     jvm:jvm.dll
 0000:fffe2000       .debug$S                   0000000180000000     jvm:jvm.dll
 0000:fffe2000       .debug$S                   0000000180000000     jvm:jvm.dll
 0000:fffe2000       .debug$S                   0000000180000000     jvm:jvm.dll
 0000:fffe2000       .debug$S                   0000000180000000     jvm:jvm.dll
 0000:fffe2000       .debug$S                   0000000180000000     jvm:jvm.dll
 0000:fffe2000       .debug$S                   0000000180000000     jvm:jvm.dll
 0000:fffe2000       .debug$S                   0000000180000000     jvm:jvm.dll
 0001:00000a6c       getUTF                     0000000180001a6c f   ClassLoader.obj
 0001:000031c0       findJniFunction            00000001800041c0 f   NativeLibraries.obj
 0001:000032a0       initIDs                    00000001800042a0 f   NativeLibraries.obj
 0001:00003c4c       getCmdlineInfo             0000000180004c4c f   ProcessHandleImpl_win.obj
 0001:00003d5c       getStartTime               0000000180004d5c f   ProcessHandleImpl_win.obj
 0001:00003dc4       getStatInfo                0000000180004dc4 f   ProcessHandleImpl_win.obj
 0001:00003edc       procToUser                 0000000180004edc f   ProcessHandleImpl_win.obj
 0001:00004448       initHolder                 0000000180005448 f   ProcessImpl_md.obj
 0001:00004568       processCreate              0000000180005568 f   ProcessImpl_md.obj
 0001:0000486c       releaseHolder              000000018000586c f   ProcessImpl_md.obj
 0001:00004910       win32Error                 0000000180005910 f   ProcessImpl_md.obj
 0001:00004e1c       initIDs                    0000000180005e1c f   RawNativeLibraries.obj
 0001:00005e44       customZoneName             0000000180006e44 f   TimeZone_md.obj
 0001:00006044       getValueInRegistry         0000000180007044 f   TimeZone_md.obj
 0001:0000613c       getWinTimeZone             000000018000713c f   TimeZone_md.obj
 0001:00006620       matchJavaTZ                0000000180007620 f   TimeZone_md.obj
 0001:00007b74       getFileInformation         0000000180008b74 f   WinNTFileSystem_md.obj
 0001:00007d10       getFinalAttributesUnixSocket 0000000180008d10 f   WinNTFileSystem_md.obj
 0001:00007e20       getFinalPath               0000000180008e20 f   WinNTFileSystem_md.obj
 0001:00007fb4       isReservedDeviceNameW      0000000180008fb4 f   WinNTFileSystem_md.obj
 0001:000080dc       removeFileOrDirectory      00000001800090dc f   WinNTFileSystem_md.obj
 0001:000087ec       wcp                        00000001800097ec f   canonicalize_md.obj
 0001:0000889c       next_utf2unicode           000000018000989c f   check_classname.obj
 0001:00008994       skip_over_field_signature  0000000180009994 f   check_classname.obj
 0001:00008a48       skip_over_fieldname        0000000180009a48 f   check_classname.obj
 0001:00009560       handleStdinAvailable       000000018000a560 f   io_util_md.obj
 0001:0000a10c       SetupI18nProps             000000018000b10c f   java_props_md.obj
 0001:0000a300       getConsoleEncoding         000000018000b300 f   java_props_md.obj
 0001:0000a3ac       getEncodingInternal        000000018000b3ac f   java_props_md.obj
 0001:0000bb44       getString646_USChars       000000018000cb44 f   jni_util.obj
 0001:0000bc80       getString8859_1Chars       000000018000cc80 f   jni_util.obj
 0001:0000bdc4       getStringBytes             000000018000cdc4 f   jni_util.obj
 0001:0000bf34       getStringCp1252Chars       000000018000cf34 f   jni_util.obj
 0001:0000c200       getStringPlatformChars0    000000018000d200 f   jni_util.obj
 0001:0000c284       getStringUTF8              000000018000d284 f   jni_util.obj
 0001:0000c46c       newSizedString8859_1       000000018000d46c f   jni_util.obj
 0001:0000c56c       newSizedStringJava         000000018000d56c f   jni_util.obj
 0001:0000c63c       newString646_US            000000018000d63c f   jni_util.obj
 0001:0000c750       newStringCp1252            000000018000d750 f   jni_util.obj
 0001:0000cdc0       $$000000                   000000018000ddc0     MSVCRT:amdsecgs.obj
 0001:0000cfac       capture_current_context    000000018000dfac f   MSVCRT:gs_report.obj
 0001:0000d01c       capture_previous_context   000000018000e01c f   MSVCRT:gs_report.obj
 0001:0000d090       $$000000                   000000018000e090     MSVCRT:chkstk.obj
 0001:0000d0f0       ?dllmain_crt_dispatch@@YAHQEAUHINSTANCE__@@KQEAX@Z 000000018000e0f0 f   MSVCRT:dll_dllmain.obj
 0001:0000d140       ?dllmain_crt_process_attach@@YAHQEAUHINSTANCE__@@QEAX@Z 000000018000e140 f   MSVCRT:dll_dllmain.obj
 0001:0000d258       ?dllmain_crt_process_detach@@YAH_N@Z 000000018000e258 f   MSVCRT:dll_dllmain.obj
 0001:0000d2d8       ?dllmain_dispatch@@YAHQEAUHINSTANCE__@@KQEAX@Z 000000018000e2d8 f   MSVCRT:dll_dllmain.obj
 0001:0000ddb0       $$000000                   000000018000edb0     MSVCRT:guard_dispatch.obj
 0001:0000ddd0       $$000000                   000000018000edd0     MSVCRT:guard_xfg_dispatch.obj
 0001:0000dde6       ?fin$0@?0??dllmain_crt_process_attach@@YAHQEAUHINSTANCE__@@QEAX@Z@4HA 000000018000ede6 f   MSVCRT:dll_dllmain.obj
 0001:0000ddfd       ?fin$0@?0??dllmain_crt_process_detach@@YAH_N@Z@4HA 000000018000edfd f   MSVCRT:dll_dllmain.obj
 0001:0000de16       ?fin$1@?0??dllmain_crt_process_detach@@YAH_N@Z@4HA 000000018000ee16 f   MSVCRT:dll_dllmain.obj
 0001:0000de2a       ?filt$0@?0??dllmain_dispatch@@YAHQEAUHINSTANCE__@@KQEAX@Z@4HA 000000018000ee2a f   MSVCRT:dll_dllmain.obj
 0001:0000de60       __scrt_is_nonwritable_in_current_image$filt$0 000000018000ee60 f   MSVCRT:utility.obj
 0002:00002468       GS_ExceptionPointers       0000000180011468     MSVCRT:gs_report.obj
 0002:000029d8       $unwind$Java_java_lang_reflect_Array_getDouble 00000001800119d8     Array.obj
 0002:000029d8       $unwind$Java_java_lang_reflect_Array_getFloat 00000001800119d8     Array.obj
 0002:000029d8       $unwind$Java_java_lang_reflect_Array_setLong 00000001800119d8     Array.obj
 0002:000029d8       $unwind$Java_java_io_FileInputStream_open0 00000001800119d8     FileInputStream.obj
 0002:000029d8       $unwind$Java_java_io_FileInputStream_readBytes 00000001800119d8     FileInputStream.obj
 0002:000029d8       $unwind$Java_java_io_FileOutputStream_open0 00000001800119d8     FileOutputStream.obj
 0002:000029d8       $unwind$Java_java_io_FileOutputStream_write 00000001800119d8     FileOutputStream.obj
 0002:000029d8       $unwind$Java_sun_util_locale_provider_HostLocaleProviderAdapterImpl_getEras 00000001800119d8     HostLocaleProviderAdapter_md.obj
 0002:000029d8       $unwind$Java_java_lang_Module_defineModule0 00000001800119d8     Module.obj
 0002:000029d8       $unwind$Java_java_io_RandomAccessFile_open0 00000001800119d8     RandomAccessFile.obj
 0002:000029d8       $unwind$Java_java_io_RandomAccessFile_readBytes0 00000001800119d8     RandomAccessFile.obj
 0002:000029d8       $unwind$Java_java_io_RandomAccessFile_write0 00000001800119d8     RandomAccessFile.obj
 0002:000029d8       $unwind$handleRead         00000001800119d8     io_util_md.obj
 0002:000029d8       $unwind$JNU_ToString       00000001800119d8     jni_util.obj
 0002:000029e0       $unwind$Java_java_lang_reflect_Array_setBoolean 00000001800119e0     Array.obj
 0002:000029e0       $unwind$Java_java_lang_reflect_Array_setByte 00000001800119e0     Array.obj
 0002:000029e0       $unwind$Java_java_lang_reflect_Array_setChar 00000001800119e0     Array.obj
 0002:000029e0       $unwind$Java_java_lang_reflect_Array_setFloat 00000001800119e0     Array.obj
 0002:000029e0       $unwind$Java_java_lang_reflect_Array_setInt 00000001800119e0     Array.obj
 0002:000029e0       $unwind$Java_java_lang_reflect_Array_setShort 00000001800119e0     Array.obj
 0002:000029e0       $unwind$Java_java_io_FileOutputStream_writeBytes 00000001800119e0     FileOutputStream.obj
 0002:000029e0       $unwind$Java_java_lang_invoke_LambdaProxyClassArchive_findFromArchive 00000001800119e0     LambdaProxyClassArchive.obj
 0002:000029e0       $unwind$Java_java_io_RandomAccessFile_writeBytes0 00000001800119e0     RandomAccessFile.obj
 0002:000029e8       $unwind$Java_java_lang_Class_forName0 00000001800119e8     Class.obj
 0002:00002a0c       $unwind$Java_java_lang_Class_isAssignableFrom 0000000180011a0c     Class.obj
 0002:00002a0c       $unwind$Java_java_io_FileInputStream_initIDs 0000000180011a0c     FileInputStream.obj
 0002:00002a0c       $unwind$Java_java_io_FileOutputStream_initIDs 0000000180011a0c     FileOutputStream.obj
 0002:00002a0c       $unwind$getCalendarID      0000000180011a0c     HostLocaleProviderAdapter_md.obj
 0002:00002a0c       $unwind$Java_java_lang_Object_getClass 0000000180011a0c     Object.obj
 0002:00002a0c       $unwind$Java_java_lang_ProcessHandleImpl_getCurrentPid0 0000000180011a0c     ProcessHandleImpl_win.obj
 0002:00002a0c       $unwind$Java_java_lang_ProcessImpl_isProcessAlive 0000000180011a0c     ProcessImpl_md.obj
 0002:00002a0c       $unwind$Java_java_io_RandomAccessFile_initIDs 0000000180011a0c     RandomAccessFile.obj
 0002:00002a0c       $unwind$Java_java_lang_Thread_clearInterruptEvent 0000000180011a0c     Thread.obj
 0002:00002a0c       $unwind$Java_sun_io_Win32ErrorMode_setErrorMode 0000000180011a0c     Win32ErrorMode.obj
 0002:00002a0c       $unwind$lastErrorReportable 0000000180011a0c     canonicalize_md.obj
 0002:00002a0c       $unwind$wcp                0000000180011a0c     canonicalize_md.obj
 0002:00002a0c       $unwind$fixClassname       0000000180011a0c     check_classname.obj
 0002:00002a0c       $unwind$handleGetLength    0000000180011a0c     io_util_md.obj
 0002:00002a0c       $unwind$handleLseek        0000000180011a0c     io_util_md.obj
 0002:00002a0c       $unwind$handleSetLength    0000000180011a0c     io_util_md.obj
 0002:00002a0c       $unwind$handleSync         0000000180011a0c     io_util_md.obj
 0002:00002a0c       $unwind$getHomeFromShell32 0000000180011a0c     java_props_md.obj
 0002:00002a0c       $unwind$JNU_GetEnv         0000000180011a0c     jni_util.obj
 0002:00002a0c       $unwind$getStringPlatformChars0 0000000180011a0c     jni_util.obj
 0002:00002a0c       $unwind$__scrt_initialize_default_local_stdio_options 0000000180011a0c     MSVCRT:default_local_stdio_options.obj
 0002:00002a0c       $unwind$?dllmain_crt_dispatch@@YAHQEAUHINSTANCE__@@KQEAX@Z 0000000180011a0c     MSVCRT:dll_dllmain.obj
 0002:00002a0c       $unwind$DllMain            0000000180011a0c     MSVCRT:dll_dllmain_stub.obj
 0002:00002a0c       $unwind$__report_rangecheckfailure 0000000180011a0c     MSVCRT:gs_report.obj
 0002:00002a0c       $unwind$__GSHandlerCheck   0000000180011a0c     MSVCRT:gshandler.obj
 0002:00002a0c       $unwind$__scrt_acquire_startup_lock 0000000180011a0c     MSVCRT:utility.obj
 0002:00002a0c       $unwind$__scrt_dllmain_after_initialize_c 0000000180011a0c     MSVCRT:utility.obj
 0002:00002a0c       $unwind$__scrt_dllmain_before_initialize_c 0000000180011a0c     MSVCRT:utility.obj
 0002:00002a0c       $unwind$__scrt_dllmain_crt_thread_attach 0000000180011a0c     MSVCRT:utility.obj
 0002:00002a0c       $unwind$__scrt_dllmain_crt_thread_detach 0000000180011a0c     MSVCRT:utility.obj
 0002:00002a0c       $unwind$__scrt_dllmain_uninitialize_c 0000000180011a0c     MSVCRT:utility.obj
 0002:00002a0c       $unwind$__scrt_dllmain_uninitialize_critical 0000000180011a0c     MSVCRT:utility.obj
 0002:00002a0c       $unwind$__scrt_initialize_crt 0000000180011a0c     MSVCRT:utility.obj
 0002:00002a14       $unwind$Java_java_lang_Class_getPrimitiveClass 0000000180011a14     Class.obj
 0002:00002a14       $unwind$Java_sun_util_locale_provider_HostLocaleProviderAdapterImpl_getCalendarID 0000000180011a14     HostLocaleProviderAdapter_md.obj
 0002:00002a14       $unwind$getLocaleInfoWrapper 0000000180011a14     HostLocaleProviderAdapter_md.obj
 0002:00002a14       $unwind$Java_jdk_internal_io_JdkConsoleImpl_echo 0000000180011a14     JdkConsoleImpl_md.obj
 0002:00002a14       $unwind$Java_jdk_internal_loader_NativeLibrary_findEntry0 0000000180011a14     NativeLibraries.obj
 0002:00002a14       $unwind$Java_java_io_RandomAccessFile_setLength0 0000000180011a14     RandomAccessFile.obj
 0002:00002a14       $unwind$Java_jdk_internal_loader_RawNativeLibraries_unload0 0000000180011a14     RawNativeLibraries.obj
 0002:00002a14       $unwind$Java_jdk_internal_misc_Signal_findSignal0 0000000180011a14     Signal.obj
 0002:00002a14       $unwind$Java_jdk_internal_util_SystemProps_00024Raw_platformProperties 0000000180011a14     System.obj
 0002:00002a14       $unwind$Java_java_io_WinNTFileSystem_getDriveDirectory 0000000180011a14     WinNTFileSystem_md.obj
 0002:00002a14       $unwind$Java_java_io_WinNTFileSystem_rename0 0000000180011a14     WinNTFileSystem_md.obj
 0002:00002a14       $unwind$verifyClassname    0000000180011a14     check_classname.obj
 0002:00002a14       $unwind$JNU_IsInstanceOfByName 0000000180011a14     jni_util.obj
 0002:00002a14       $unwind$__scrt_dllmain_exception_filter 0000000180011a14     MSVCRT:utility.obj
 0002:00002a28       $unwind$Java_java_lang_ClassLoader_defineClass1 0000000180011a28     ClassLoader.obj
 0002:00002a28       $unwind$Java_java_lang_ClassLoader_defineClass2 0000000180011a28     ClassLoader.obj
 0002:00002a4c       $unwind$Java_java_lang_ClassLoader_defineClass0 0000000180011a4c     ClassLoader.obj
 0002:00002a70       $unwind$Java_java_lang_ClassLoader_findBootstrapClass 0000000180011a70     ClassLoader.obj
 0002:00002a8c       $unwind$getUTF             0000000180011a8c     ClassLoader.obj
 0002:00002aa4       $unwind$Java_java_io_Console_istty 0000000180011aa4     Console_md.obj
 0002:00002aa4       $unwind$Java_java_io_FileDescriptor_sync0 0000000180011aa4     FileDescriptor_md.obj
 0002:00002aa4       $unwind$Java_java_io_FileInputStream_available0 0000000180011aa4     FileInputStream.obj
 0002:00002aa4       $unwind$Java_java_io_FileInputStream_isRegularFile0 0000000180011aa4     FileInputStream.obj
 0002:00002aa4       $unwind$EnumCalendarInfoProc 0000000180011aa4     HostLocaleProviderAdapter_md.obj
 0002:00002aa4       $unwind$Java_sun_util_locale_provider_HostLocaleProviderAdapterImpl_initialize 0000000180011aa4     HostLocaleProviderAdapter_md.obj
 0002:00002aa4       $unwind$Java_java_io_ObjectStreamClass_initNative 0000000180011aa4     ObjectStreamClass.obj
 0002:00002aa4       $unwind$Java_java_lang_ProcessImpl_getExitCodeProcess 0000000180011aa4     ProcessImpl_md.obj
 0002:00002aa4       $unwind$initIDs            0000000180011aa4     RawNativeLibraries.obj
 0002:00002aa4       $unwind$Java_java_lang_Throwable_fillInStackTrace 0000000180011aa4     Throwable.obj
 0002:00002aa4       $unwind$Java_java_io_WinNTFileSystem_initIDs 0000000180011aa4     WinNTFileSystem_md.obj
 0002:00002aa4       $unwind$skip_over_field_signature 0000000180011aa4     check_classname.obj
 0002:00002aa4       $unwind$readSingle         0000000180011aa4     io_util.obj
 0002:00002aa4       $unwind$fileToNTPath       0000000180011aa4     io_util_md.obj
 0002:00002aa4       $unwind$getFD              0000000180011aa4     io_util_md.obj
 0002:00002aa4       $unwind$__raise_securityfailure 0000000180011aa4     MSVCRT:gs_report.obj
 0002:00002aa4       $unwind$__scrt_initialize_onexit_tables 0000000180011aa4     MSVCRT:utility.obj
 0002:00002aa4       $unwind$__scrt_release_startup_lock 0000000180011aa4     MSVCRT:utility.obj
 0002:00002aa4       $unwind$__scrt_uninitialize_crt 0000000180011aa4     MSVCRT:utility.obj
 0002:00002aac       $unwind$Java_java_io_FileDescriptor_initIDs 0000000180011aac     FileDescriptor_md.obj
 0002:00002aac       $unwind$Java_java_io_FileInputStream_length0 0000000180011aac     FileInputStream.obj
 0002:00002aac       $unwind$Java_java_io_FileInputStream_position0 0000000180011aac     FileInputStream.obj
 0002:00002aac       $unwind$initIDs            0000000180011aac     NativeLibraries.obj
 0002:00002aac       $unwind$Java_java_lang_ProcessEnvironment_environmentBlock 0000000180011aac     ProcessEnvironment_md.obj
 0002:00002aac       $unwind$Java_java_lang_ProcessHandleImpl_00024Info_initIDs 0000000180011aac     ProcessHandleImpl_win.obj
 0002:00002aac       $unwind$Java_java_lang_ProcessHandleImpl_isAlive0 0000000180011aac     ProcessHandleImpl_win.obj
 0002:00002aac       $unwind$Java_java_lang_ProcessHandleImpl_waitForProcessExit0 0000000180011aac     ProcessHandleImpl_win.obj
 0002:00002aac       $unwind$releaseHolder      0000000180011aac     ProcessImpl_md.obj
 0002:00002aac       $unwind$Java_java_io_RandomAccessFile_getFilePointer 0000000180011aac     RandomAccessFile.obj
 0002:00002aac       $unwind$Java_java_io_RandomAccessFile_length0 0000000180011aac     RandomAccessFile.obj
 0002:00002aac       $unwind$Java_java_io_RandomAccessFile_seek0 0000000180011aac     RandomAccessFile.obj
 0002:00002aac       $unwind$Java_java_io_WinNTFileSystem_createDirectory0 0000000180011aac     WinNTFileSystem_md.obj
 0002:00002aac       $unwind$Java_java_io_WinNTFileSystem_delete0 0000000180011aac     WinNTFileSystem_md.obj
 0002:00002aac       $unwind$Java_java_io_WinNTFileSystem_getBooleanAttributes0 0000000180011aac     WinNTFileSystem_md.obj
 0002:00002aac       $unwind$writeSingle        0000000180011aac     io_util.obj
 0002:00002aac       $unwind$currentDirLength   0000000180011aac     io_util_md.obj
 0002:00002aac       $unwind$JNU_ClassString    0000000180011aac     jni_util.obj
 0002:00002aac       $unwind$JNU_NewStringPlatform 0000000180011aac     jni_util.obj
 0002:00002aac       $unwind$JNU_ThrowByName    0000000180011aac     jni_util.obj
 0002:00002aac       $unwind$_RTC_Initialize    0000000180011aac     MSVCRT:initsect.obj
 0002:00002aac       $unwind$_RTC_Terminate     0000000180011aac     MSVCRT:initsect.obj
 0002:00002ab8       $unwind$Java_java_io_FileCleanable_cleanupClose0 0000000180011ab8     FileDescriptor_md.obj
 0002:00002ac0       $unwind$Java_java_io_FileInputStream_skip0 0000000180011ac0     FileInputStream.obj
 0002:00002ac0       $unwind$Java_sun_util_locale_provider_HostLocaleProviderAdapterImpl_getNumberPattern 0000000180011ac0     HostLocaleProviderAdapter_md.obj
 0002:00002ac0       $unwind$Java_jdk_internal_loader_RawNativeLibraries_load0 0000000180011ac0     RawNativeLibraries.obj
 0002:00002ac0       $unwind$Java_java_util_TimeZone_getSystemTimeZoneID 0000000180011ac0     TimeZone.obj
 0002:00002ac0       $unwind$Java_java_io_WinNTFileSystem_getFinalPath0 0000000180011ac0     WinNTFileSystem_md.obj
 0002:00002ac0       $unwind$removeFileOrDirectory 0000000180011ac0     WinNTFileSystem_md.obj
 0002:00002ac0       $unwind$fileOpen           0000000180011ac0     io_util_md.obj
 0002:00002ad8       $unwind$Java_sun_util_locale_provider_HostLocaleProviderAdapterImpl_getDefaultLocale 0000000180011ad8     HostLocaleProviderAdapter_md.obj
 0002:00002ad8       $unwind$Java_java_io_ObjectStreamClass_hasStaticInitializer 0000000180011ad8     ObjectStreamClass.obj
 0002:00002ad8       $unwind$Java_java_lang_ProcessHandleImpl_00024Info_info0 0000000180011ad8     ProcessHandleImpl_win.obj
 0002:00002ad8       $unwind$Java_java_lang_ProcessHandleImpl_destroy0 0000000180011ad8     ProcessHandleImpl_win.obj
 0002:00002ad8       $unwind$Java_java_lang_System_setErr0 0000000180011ad8     System.obj
 0002:00002ad8       $unwind$Java_java_lang_System_setIn0 0000000180011ad8     System.obj
 0002:00002ad8       $unwind$Java_java_lang_System_setOut0 0000000180011ad8     System.obj
 0002:00002ad8       $unwind$Java_java_util_TimeZone_getSystemGMTOffsetID 0000000180011ad8     TimeZone.obj
 0002:00002ad8       $unwind$Java_java_io_WinNTFileSystem_checkAccess0 0000000180011ad8     WinNTFileSystem_md.obj
 0002:00002ad8       $unwind$Java_java_io_WinNTFileSystem_setReadOnly0 0000000180011ad8     WinNTFileSystem_md.obj
 0002:00002ad8       $unwind$getPrefixed        0000000180011ad8     canonicalize_md.obj
 0002:00002ad8       $unwind$fileDescriptorClose 0000000180011ad8     io_util_md.obj
 0002:00002ad8       $unwind$GetStringPlatform  0000000180011ad8     java_props_md.obj
 0002:00002ad8       $unwind$getConsoleEncoding 0000000180011ad8     java_props_md.obj
 0002:00002ad8       $unwind$JNU_ThrowByNameWithLastError 0000000180011ad8     jni_util.obj
 0002:00002ad8       $unwind$_DllMainCRTStartup 0000000180011ad8     MSVCRT:dll_dllmain.obj
 0002:00002ae8       $unwind$Java_sun_util_locale_provider_HostLocaleProviderAdapterImpl_getDateTimePattern 0000000180011ae8     HostLocaleProviderAdapter_md.obj
 0002:00002b08       $unwind$Java_sun_util_locale_provider_HostLocaleProviderAdapterImpl_getAmPmStrings 0000000180011b08     HostLocaleProviderAdapter_md.obj
 0002:00002b08       $unwind$Java_sun_util_locale_provider_HostLocaleProviderAdapterImpl_getMonths 0000000180011b08     HostLocaleProviderAdapter_md.obj
 0002:00002b08       $unwind$Java_sun_util_locale_provider_HostLocaleProviderAdapterImpl_getShortMonths 0000000180011b08     HostLocaleProviderAdapter_md.obj
 0002:00002b08       $unwind$Java_sun_util_locale_provider_HostLocaleProviderAdapterImpl_getShortWeekdays 0000000180011b08     HostLocaleProviderAdapter_md.obj
 0002:00002b08       $unwind$Java_sun_util_locale_provider_HostLocaleProviderAdapterImpl_getWeekdays 0000000180011b08     HostLocaleProviderAdapter_md.obj
 0002:00002b10       $unwind$Java_sun_util_locale_provider_HostLocaleProviderAdapterImpl_getCalendarDataValue 0000000180011b10     HostLocaleProviderAdapter_md.obj
 0002:00002b10       $unwind$Java_sun_util_locale_provider_HostLocaleProviderAdapterImpl_isNativeDigit 0000000180011b10     HostLocaleProviderAdapter_md.obj
 0002:00002b10       $unwind$JNU_GetStaticFieldByName 0000000180011b10     jni_util.obj
 0002:00002b24       $unwind$Java_sun_util_locale_provider_HostLocaleProviderAdapterImpl_getCurrencySymbol 0000000180011b24     HostLocaleProviderAdapter_md.obj
 0002:00002b24       $unwind$Java_sun_util_locale_provider_HostLocaleProviderAdapterImpl_getDecimalSeparator 0000000180011b24     HostLocaleProviderAdapter_md.obj
 0002:00002b24       $unwind$Java_sun_util_locale_provider_HostLocaleProviderAdapterImpl_getGroupingSeparator 0000000180011b24     HostLocaleProviderAdapter_md.obj
 0002:00002b24       $unwind$Java_sun_util_locale_provider_HostLocaleProviderAdapterImpl_getInfinity 0000000180011b24     HostLocaleProviderAdapter_md.obj
 0002:00002b24       $unwind$Java_sun_util_locale_provider_HostLocaleProviderAdapterImpl_getInternationalCurrencySymbol 0000000180011b24     HostLocaleProviderAdapter_md.obj
 0002:00002b24       $unwind$Java_sun_util_locale_provider_HostLocaleProviderAdapterImpl_getMinusSign 0000000180011b24     HostLocaleProviderAdapter_md.obj
 0002:00002b24       $unwind$Java_sun_util_locale_provider_HostLocaleProviderAdapterImpl_getMonetaryDecimalSeparator 0000000180011b24     HostLocaleProviderAdapter_md.obj
 0002:00002b24       $unwind$Java_sun_util_locale_provider_HostLocaleProviderAdapterImpl_getNaN 0000000180011b24     HostLocaleProviderAdapter_md.obj
 0002:00002b24       $unwind$Java_sun_util_locale_provider_HostLocaleProviderAdapterImpl_getPerMill 0000000180011b24     HostLocaleProviderAdapter_md.obj
 0002:00002b24       $unwind$Java_sun_util_locale_provider_HostLocaleProviderAdapterImpl_getPercent 0000000180011b24     HostLocaleProviderAdapter_md.obj
 0002:00002b24       $unwind$Java_sun_util_locale_provider_HostLocaleProviderAdapterImpl_getZeroDigit 0000000180011b24     HostLocaleProviderAdapter_md.obj
 0002:00002b44       $unwind$Java_sun_util_locale_provider_HostLocaleProviderAdapterImpl_getCalendarDisplayStrings 0000000180011b44     HostLocaleProviderAdapter_md.obj
 0002:00002b44       $unwind$Java_java_io_WinNTFileSystem_setLastModifiedTime0 0000000180011b44     WinNTFileSystem_md.obj
 0002:00002b58       $unwind$Java_sun_util_locale_provider_HostLocaleProviderAdapterImpl_getDisplayString 0000000180011b58     HostLocaleProviderAdapter_md.obj
 0002:00002b74       $unwind$getCalendarInfoWrapper 0000000180011b74     HostLocaleProviderAdapter_md.obj
 0002:00002b74       $unwind$winFileHandleOpen  0000000180011b74     io_util_md.obj
 0002:00002b88       $unwind$replaceCalendarArrayElems 0000000180011b88     HostLocaleProviderAdapter_md.obj
 0002:00002ba8       $unwind$getNumberPattern   0000000180011ba8     HostLocaleProviderAdapter_md.obj
 0002:00002bc4       $unwind$getNumberPart      0000000180011bc4     HostLocaleProviderAdapter_md.obj
 0002:00002be4       $unwind$getFixPart         0000000180011be4     HostLocaleProviderAdapter_md.obj
 0002:00002bf8       $unwind$enumCalendarInfoWrapper 0000000180011bf8     HostLocaleProviderAdapter_md.obj
 0002:00002c0c       $unwind$getErasImpl        0000000180011c0c     HostLocaleProviderAdapter_md.obj
 0002:00002c30       $unwind$Java_java_lang_invoke_LambdaProxyClassArchive_addToArchive 0000000180011c30     LambdaProxyClassArchive.obj
 0002:00002c30       $unwind$getStartTime       0000000180011c30     ProcessHandleImpl_win.obj
 0002:00002c38       $unwind$Java_jdk_internal_loader_NativeLibraries_load 0000000180011c38     NativeLibraries.obj
 0002:00002c5c       $unwind$Java_jdk_internal_loader_NativeLibraries_unload 0000000180011c5c     NativeLibraries.obj
 0002:00002c5c       $unwind$getStringBytes     0000000180011c5c     jni_util.obj
 0002:00002c5c       $unwind$newSizedStringJava 0000000180011c5c     jni_util.obj
 0002:00002c74       $unwind$Java_jdk_internal_loader_NativeLibraries_findBuiltinLib 0000000180011c74     NativeLibraries.obj
 0002:00002c74       $unwind$JNU_CallMethodByNameV 0000000180011c74     jni_util.obj
 0002:00002c74       $unwind$getString646_USChars 0000000180011c74     jni_util.obj
 0002:00002c74       $unwind$getString8859_1Chars 0000000180011c74     jni_util.obj
 0002:00002c74       $unwind$getStringUTF8      0000000180011c74     jni_util.obj
 0002:00002c90       $unwind$findJniFunction    0000000180011c90     NativeLibraries.obj
 0002:00002c90       $unwind$prefixAbpath       0000000180011c90     io_util_md.obj
 0002:00002c90       $unwind$JNU_CopyObjectArray 0000000180011c90     jni_util.obj
 0002:00002ca8       $unwind$Java_java_lang_ProcessHandleImpl_parent0 0000000180011ca8     ProcessHandleImpl_win.obj
 0002:00002cc8       $unwind$Java_java_lang_ProcessHandleImpl_getProcessPids0 0000000180011cc8     ProcessHandleImpl_win.obj
 0002:00002cec       $unwind$getStatInfo        0000000180011cec     ProcessHandleImpl_win.obj
 0002:00002d00       $unwind$getCmdlineInfo     0000000180011d00     ProcessHandleImpl_win.obj
 0002:00002d1c       $unwind$procToUser         0000000180011d1c     ProcessHandleImpl_win.obj
 0002:00002d38       $unwind$swprintf           0000000180011d38     ProcessImpl_md.obj
 0002:00002d38       $unwind$snprintf           0000000180011d38     TimeZone_md.obj
 0002:00002d48       $unwind$Java_java_lang_ProcessImpl_waitForInterruptibly 0000000180011d48     ProcessImpl_md.obj
 0002:00002d48       $unwind$customZoneName     0000000180011d48     TimeZone_md.obj
 0002:00002d48       $unwind$handleWrite        0000000180011d48     io_util_md.obj
 0002:00002d50       $unwind$Java_java_lang_ProcessImpl_waitForTimeoutInterruptibly 0000000180011d50     ProcessImpl_md.obj
 0002:00002d5c       $unwind$Java_java_lang_ProcessImpl_create 0000000180011d5c     ProcessImpl_md.obj
 0002:00002d74       $unwind$Java_java_lang_ProcessImpl_openForAtomicAppend 0000000180011d74     ProcessImpl_md.obj
 0002:00002d74       $unwind$Java_java_io_WinNTFileSystem_createFileExclusively0 0000000180011d74     WinNTFileSystem_md.obj
 0002:00002d74       $unwind$Java_java_io_WinNTFileSystem_getLastModifiedTime0 0000000180011d74     WinNTFileSystem_md.obj
 0002:00002d84       $unwind$os_error_message   0000000180011d84     ProcessImpl_md.obj
 0002:00002d90       $unwind$win32Error         0000000180011d90     ProcessImpl_md.obj
 0002:00002dac       $unwind$initHolder         0000000180011dac     ProcessImpl_md.obj
 0002:00002dac       $unwind$Java_java_io_WinNTFileSystem_setPermission0 0000000180011dac     WinNTFileSystem_md.obj
 0002:00002dc0       $unwind$processCreate      0000000180011dc0     ProcessImpl_md.obj
 0002:00002de4       $unwind$Java_java_lang_System_mapLibraryName 0000000180011de4     System.obj
 0002:00002e08       $unwind$findJavaTZ_md      0000000180011e08     TimeZone_md.obj
 0002:00002e20       $unwind$getGMTOffsetID     0000000180011e20     TimeZone_md.obj
 0002:00002e3c       $unwind$getValueInRegistry 0000000180011e3c     TimeZone_md.obj
 0002:00002e5c       $unwind$getWinTimeZone     0000000180011e5c     TimeZone_md.obj
 0002:00002e80       $unwind$matchJavaTZ        0000000180011e80     TimeZone_md.obj
 0002:00002ea0       $unwind$Java_sun_security_provider_NativeSeedGenerator_nativeGenerateSeed 0000000180011ea0     WinCAPISeedGenerator.obj
 0002:00002eb4       $unwind$Java_java_io_WinNTFileSystem_getNameMax0 0000000180011eb4     WinNTFileSystem_md.obj
 0002:00002eb4       $unwind$getFinalPath       0000000180011eb4     WinNTFileSystem_md.obj
 0002:00002ec8       $unwind$getFileInformation 0000000180011ec8     WinNTFileSystem_md.obj
 0002:00002ed8       $unwind$getFinalAttributesUnixSocket 0000000180011ed8     WinNTFileSystem_md.obj
 0002:00002ef0       $unwind$getFinalAttributesIfReparsePoint 0000000180011ef0     WinNTFileSystem_md.obj
 0002:00002f00       $unwind$getFinalAttributes 0000000180011f00     WinNTFileSystem_md.obj
 0002:00002f1c       $unwind$Java_java_io_WinNTFileSystem_canonicalize0 0000000180011f1c     WinNTFileSystem_md.obj
 0002:00002f3c       $unwind$Java_java_io_WinNTFileSystem_canonicalizeWithPrefix0 0000000180011f3c     WinNTFileSystem_md.obj
 0002:00002f60       $unwind$isReservedDeviceNameW 0000000180011f60     WinNTFileSystem_md.obj
 0002:00002f70       $unwind$Java_java_io_WinNTFileSystem_getLength0 0000000180011f70     WinNTFileSystem_md.obj
 0002:00002f90       $unwind$Java_java_io_WinNTFileSystem_list0 0000000180011f90     WinNTFileSystem_md.obj
 0002:00002fb4       $unwind$Java_java_io_WinNTFileSystem_getSpace0 0000000180011fb4     WinNTFileSystem_md.obj
 0002:00002fd0       $unwind$wcanonicalize      0000000180011fd0     canonicalize_md.obj
 0002:00002ff4       $unwind$wcanonicalizeWithPrefix 0000000180011ff4     canonicalize_md.obj
 0002:00003010       $unwind$JDK_Canonicalize   0000000180012010     canonicalize_md.obj
 0002:0000302c       $unwind$verifyFixClassname 000000018001202c     check_classname.obj
 0002:00003038       $unwind$skip_over_fieldname 0000000180012038     check_classname.obj
 0002:0000304c       $unwind$next_utf2unicode   000000018001204c     check_classname.obj
 0002:00003058       $unwind$readBytes          0000000180012058     io_util.obj
 0002:00003058       $unwind$writeBytes         0000000180012058     io_util.obj
 0002:00003078       $unwind$throwFileNotFoundException 0000000180012078     io_util.obj
 0002:00003088       $unwind$pathToNTPath       0000000180012088     io_util_md.obj
 0002:000030a0       $unwind$currentDir         00000001800120a0     io_util_md.obj
 0002:000030b0       $unwind$handleAvailable    00000001800120b0     io_util_md.obj
 0002:000030c0       $unwind$handleAppend       00000001800120c0     io_util_md.obj
 0002:000030c8       $unwind$handleStdinAvailable 00000001800120c8     io_util_md.obj
 0002:000030dc       $unwind$sscanf             00000001800120dc     java_props_md.obj
 0002:000030e8       $unwind$getJavaIDFromLangID 00000001800120e8     java_props_md.obj
 0002:00003104       $unwind$GetJavaProperties  0000000180012104     java_props_md.obj
 0002:0000312c       $unwind$SetupI18nProps     000000018001212c     java_props_md.obj
 0002:00003148       $unwind$getEncodingInternal 0000000180012148     java_props_md.obj
 0002:00003164       $unwind$JDK_LoadSystemLibrary 0000000180012164     jdk_util_md.obj
 0002:0000317c       $unwind$jio_snprintf       000000018001217c     jio.obj
 0002:00003184       $unwind$jio_fprintf        0000000180012184     jio.obj
 0002:0000318c       $unwind$JNU_ThrowByNameWithMessageAndLastError 000000018001218c     jni_util.obj
 0002:000031a8       $unwind$JNU_CallStaticMethodByName 00000001800121a8     jni_util.obj
 0002:000031b8       $unwind$JNU_CallMethodByName 00000001800121b8     jni_util.obj
 0002:000031c0       $unwind$JNU_NewObjectByName 00000001800121c0     jni_util.obj
 0002:000031d0       $unwind$JNU_GetFieldByName 00000001800121d0     jni_util.obj
 0002:000031e8       $unwind$JNU_SetFieldByName 00000001800121e8     jni_util.obj
 0002:000031f8       $unwind$InitializeEncoding 00000001800121f8     jni_util.obj
 0002:0000320c       $unwind$newSizedString8859_1 000000018001220c     jni_util.obj
 0002:0000322c       $unwind$newString646_US    000000018001222c     jni_util.obj
 0002:0000322c       $unwind$newStringCp1252    000000018001222c     jni_util.obj
 0002:0000324c       $unwind$getStringCp1252Chars 000000018001224c     jni_util.obj
 0002:00003268       $unwind$getLastErrorString 0000000180012268     jni_util_md.obj
 0002:00003280       $unwind$__GSHandlerCheckCommon 0000000180012280     MSVCRT:gshandler.obj
 0002:00003288       $xdatasym                  0000000180012288     MSVCRT:amdsecgs.obj
 0002:0000328c       $unwind$__report_securityfailure 000000018001228c     MSVCRT:gs_report.obj
 0002:00003294       $unwind$__report_gsfailure 0000000180012294     MSVCRT:gs_report.obj
 0002:0000329c       $unwind$capture_current_context 000000018001229c     MSVCRT:gs_report.obj
 0002:000032a8       $unwind$capture_previous_context 00000001800122a8     MSVCRT:gs_report.obj
 0002:000032b8       $xdatasym                  00000001800122b8     MSVCRT:chkstk.obj
 0002:000032c0       $unwind$?dllmain_crt_process_attach@@YAHQEAUHINSTANCE__@@QEAX@Z 00000001800122c0     MSVCRT:dll_dllmain.obj
 0002:000032fc       $unwind$?fin$0@?0??dllmain_crt_process_attach@@YAHQEAUHINSTANCE__@@QEAX@Z@4HA 00000001800122fc     MSVCRT:dll_dllmain.obj
 0002:000032fc       $unwind$?fin$0@?0??dllmain_crt_process_detach@@YAH_N@Z@4HA 00000001800122fc     MSVCRT:dll_dllmain.obj
 0002:000032fc       $unwind$?fin$1@?0??dllmain_crt_process_detach@@YAH_N@Z@4HA 00000001800122fc     MSVCRT:dll_dllmain.obj
 0002:00003304       $unwind$?dllmain_crt_process_detach@@YAH_N@Z 0000000180012304     MSVCRT:dll_dllmain.obj
 0002:00003358       $unwind$?dllmain_dispatch@@YAHQEAUHINSTANCE__@@KQEAX@Z 0000000180012358     MSVCRT:dll_dllmain.obj
 0002:00003380       $unwind$?filt$0@?0??dllmain_dispatch@@YAHQEAUHINSTANCE__@@KQEAX@Z@4HA 0000000180012380     MSVCRT:dll_dllmain.obj
 0002:00003388       $unwind$__security_init_cookie 0000000180012388     MSVCRT:gs_support.obj
 0002:00003394       $unwind$__scrt_is_nonwritable_in_current_image 0000000180012394     MSVCRT:utility.obj
 0002:000033b4       $unwind$__scrt_is_nonwritable_in_current_image$filt$0 00000001800123b4     MSVCRT:utility.obj
 0002:000033bc       $unwind$__scrt_fastfail    00000001800123bc     MSVCRT:utility_desktop.obj
 0002:000033cc       $unwind$__isa_available_init 00000001800123cc     MSVCRT:cpu_disp.obj
 0002:000033e0       $xdatasym                  00000001800123e0     MSVCRT:guard_dispatch.obj
 0002:000033e8       $xdatasym                  00000001800123e8     MSVCRT:guard_xfg_dispatch.obj
 0002:000033f0       .edata                     00000001800123f0     java.exp
 0002:00003418       rgpv                       0000000180012418     java.exp
 0002:00003890       rgszName                   0000000180012890     java.exp
 0002:00003d08       rgwOrd                     0000000180012d08     java.exp
 0002:00003f44       szName                     0000000180012f44     java.exp
 0002:00003f4d       $N00001                    0000000180012f4d     java.exp
 0002:00003f64       $N00002                    0000000180012f64     java.exp
 0002:00003f81       $N00003                    0000000180012f81     java.exp
 0002:00003f94       $N00004                    0000000180012f94     java.exp
 0002:00003fa5       $N00005                    0000000180012fa5     java.exp
 0002:00003fbb       $N00006                    0000000180012fbb     java.exp
 0002:00003fc6       $N00007                    0000000180012fc6     java.exp
 0002:00003fdb       $N00008                    0000000180012fdb     java.exp
 0002:00003ff1       $N00009                    0000000180012ff1     java.exp
 0002:0000400c       $N00010                    000000018001300c     java.exp
 0002:0000401c       $N00011                    000000018001301c     java.exp
 0002:00004030       $N00012                    0000000180013030     java.exp
 0002:0000403b       $N00013                    000000018001303b     java.exp
 0002:0000404e       $N00014                    000000018001304e     java.exp
 0002:00004067       $N00015                    0000000180013067     java.exp
 0002:00004082       $N00016                    0000000180013082     java.exp
 0002:000040a3       $N00017                    00000001800130a3     java.exp
 0002:000040ba       $N00018                    00000001800130ba     java.exp
 0002:000040ce       $N00019                    00000001800130ce     java.exp
 0002:000040e4       $N00020                    00000001800130e4     java.exp
 0002:00004103       $N00021                    0000000180013103     java.exp
 0002:00004116       $N00022                    0000000180013116     java.exp
 0002:0000413e       $N00023                    000000018001313e     java.exp
 0002:0000414e       $N00024                    000000018001314e     java.exp
 0002:0000416b       $N00025                    000000018001316b     java.exp
 0002:00004192       $N00026                    0000000180013192     java.exp
 0002:000041b2       $N00027                    00000001800131b2     java.exp
 0002:000041c7       $N00028                    00000001800131c7     java.exp
 0002:000041e9       $N00029                    00000001800131e9     java.exp
 0002:00004215       $N00030                    0000000180013215     java.exp
 0002:00004237       $N00031                    0000000180013237     java.exp
 0002:0000424e       $N00032                    000000018001324e     java.exp
 0002:0000426c       $N00033                    000000018001326c     java.exp
 0002:00004286       $N00034                    0000000180013286     java.exp
 0002:00004293       $N00035                    0000000180013293     java.exp
 0002:000042ae       $N00036                    00000001800132ae     java.exp
 0002:000042d7       $N00037                    00000001800132d7     java.exp
 0002:000042fa       $N00038                    00000001800132fa     java.exp
 0002:00004320       $N00039                    0000000180013320     java.exp
 0002:00004346       $N00040                    0000000180013346     java.exp
 0002:0000436a       $N00041                    000000018001336a     java.exp
 0002:0000438c       $N00042                    000000018001338c     java.exp
 0002:000043b4       $N00043                    00000001800133b4     java.exp
 0002:000043d9       $N00044                    00000001800133d9     java.exp
 0002:00004405       $N00045                    0000000180013405     java.exp
 0002:0000442a       $N00046                    000000018001342a     java.exp
 0002:0000444d       $N00047                    000000018001344d     java.exp
 0002:00004474       $N00048                    0000000180013474     java.exp
 0002:00004497       $N00049                    0000000180013497     java.exp
 0002:000044be       $N00050                    00000001800134be     java.exp
 0002:000044e1       $N00051                    00000001800134e1     java.exp
 0002:00004507       $N00052                    0000000180013507     java.exp
 0002:0000452b       $N00053                    000000018001352b     java.exp
 0002:0000454f       $N00054                    000000018001354f     java.exp
 0002:00004578       $N00055                    0000000180013578     java.exp
 0002:000045ac       $N00056                    00000001800135ac     java.exp
 0002:000045d6       $N00057                    00000001800135d6     java.exp
 0002:00004603       $N00058                    0000000180013603     java.exp
 0002:00004629       $N00059                    0000000180013629     java.exp
 0002:0000464f       $N00060                    000000018001364f     java.exp
 0002:00004673       $N00061                    0000000180013673     java.exp
 0002:00004697       $N00062                    0000000180013697     java.exp
 0002:000046c0       $N00063                    00000001800136c0     java.exp
 0002:000046e4       $N00064                    00000001800136e4     java.exp
 0002:0000470d       $N00065                    000000018001370d     java.exp
 0002:00004732       $N00066                    0000000180013732     java.exp
 0002:0000475c       $N00067                    000000018001375c     java.exp
 0002:00004787       $N00068                    0000000180013787     java.exp
 0002:000047bc       $N00069                    00000001800137bc     java.exp
 0002:000047e6       $N00070                    00000001800137e6     java.exp
 0002:00004814       $N00071                    0000000180013814     java.exp
 0002:00004848       $N00072                    0000000180013848     java.exp
 0002:0000486d       $N00073                    000000018001386d     java.exp
 0002:000048a0       $N00074                    00000001800138a0     java.exp
 0002:000048cf       $N00075                    00000001800138cf     java.exp
 0002:000048fa       $N00076                    00000001800138fa     java.exp
 0002:0000492c       $N00077                    000000018001392c     java.exp
 0002:00004954       $N00078                    0000000180013954     java.exp
 0002:0000497d       $N00079                    000000018001397d     java.exp
 0002:000049a4       $N00080                    00000001800139a4     java.exp
 0002:000049c9       $N00081                    00000001800139c9     java.exp
 0002:000049ec       $N00082                    00000001800139ec     java.exp
 0002:00004a14       $N00083                    0000000180013a14     java.exp
 0002:00004a39       $N00084                    0000000180013a39     java.exp
 0002:00004a6b       $N00085                    0000000180013a6b     java.exp
 0002:00004a97       $N00086                    0000000180013a97     java.exp
 0002:00004ac1       $N00087                    0000000180013ac1     java.exp
 0002:00004ae9       $N00088                    0000000180013ae9     java.exp
 0002:00004b11       $N00089                    0000000180013b11     java.exp
 0002:00004b39       $N00090                    0000000180013b39     java.exp
 0002:00004b67       $N00091                    0000000180013b67     java.exp
 0002:00004b93       $N00092                    0000000180013b93     java.exp
 0002:00004bbe       $N00093                    0000000180013bbe     java.exp
 0002:00004bdc       $N00094                    0000000180013bdc     java.exp
 0002:00004c03       $N00095                    0000000180013c03     java.exp
 0002:00004c29       $N00096                    0000000180013c29     java.exp
 0002:00004c49       $N00097                    0000000180013c49     java.exp
 0002:00004c6e       $N00098                    0000000180013c6e     java.exp
 0002:00004c98       $N00099                    0000000180013c98     java.exp
 0002:00004cbf       $N00100                    0000000180013cbf     java.exp
 0002:00004ce6       $N00101                    0000000180013ce6     java.exp
 0002:00004d0a       $N00102                    0000000180013d0a     java.exp
 0002:00004d2c       $N00103                    0000000180013d2c     java.exp
 0002:00004d53       $N00104                    0000000180013d53     java.exp
 0002:00004d81       $N00105                    0000000180013d81     java.exp
 0002:00004da1       $N00106                    0000000180013da1     java.exp
 0002:00004dc5       $N00107                    0000000180013dc5     java.exp
 0002:00004dff       $N00108                    0000000180013dff     java.exp
 0002:00004e1e       $N00109                    0000000180013e1e     java.exp
 0002:00004e51       $N00110                    0000000180013e51     java.exp
 0002:00004e82       $N00111                    0000000180013e82     java.exp
 0002:00004eb5       $N00112                    0000000180013eb5     java.exp
 0002:00004edf       $N00113                    0000000180013edf     java.exp
 0002:00004f0f       $N00114                    0000000180013f0f     java.exp
 0002:00004f40       $N00115                    0000000180013f40     java.exp
 0002:00004f6c       $N00116                    0000000180013f6c     java.exp
 0002:00004f96       $N00117                    0000000180013f96     java.exp
 0002:00004fbf       $N00118                    0000000180013fbf     java.exp
 0002:00004ff4       $N00119                    0000000180013ff4     java.exp
 0002:0000501b       $N00120                    000000018001401b     java.exp
 0002:0000503d       $N00121                    000000018001403d     java.exp
 0002:0000506b       $N00122                    000000018001406b     java.exp
 0002:00005094       $N00123                    0000000180014094     java.exp
 0002:000050be       $N00124                    00000001800140be     java.exp
 0002:000050e8       $N00125                    00000001800140e8     java.exp
 0002:00005117       $N00126                    0000000180014117     java.exp
 0002:00005143       $N00127                    0000000180014143     java.exp
 0002:00005173       $N00128                    0000000180014173     java.exp
 0002:000051aa       $N00129                    00000001800141aa     java.exp
 0002:000051d5       $N00130                    00000001800141d5     java.exp
 0002:000051f7       $N00131                    00000001800141f7     java.exp
 0002:00005211       $N00132                    0000000180014211     java.exp
 0002:00005232       $N00133                    0000000180014232     java.exp
 0002:00005255       $N00134                    0000000180014255     java.exp
 0002:00005278       $N00135                    0000000180014278     java.exp
 0002:00005296       $N00136                    0000000180014296     java.exp
 0002:000052c9       $N00137                    00000001800142c9     java.exp
 0002:00005312       $N00138                    0000000180014312     java.exp
 0002:0000535e       $N00139                    000000018001435e     java.exp
 0002:000053a9       $N00140                    00000001800143a9     java.exp
 0002:000053df       $N00141                    00000001800143df     java.exp
 0002:00005416       $N00142                    0000000180014416     java.exp
 0002:0000544e       $N00143                    000000018001444e     java.exp
 0002:0000546b       $N00144                    000000018001446b     java.exp
 0002:00005492       $N00145                    0000000180014492     java.exp
 0002:000054b7       $N00146                    00000001800144b7     java.exp
 0002:000054dd       $N00147                    00000001800144dd     java.exp
 0002:000054fb       $N00148                    00000001800144fb     java.exp
 0002:00005518       $N00149                    0000000180014518     java.exp
 0002:00005536       $N00150                    0000000180014536     java.exp
 0002:00005560       $N00151                    0000000180014560     java.exp
 0002:00005586       $N00152                    0000000180014586     java.exp
 0002:000055b0       $N00153                    00000001800145b0     java.exp
 0002:000055dd       $N00154                    00000001800145dd     java.exp
 0002:00005618       $N00155                    0000000180014618     java.exp
 0002:00005656       $N00156                    0000000180014656     java.exp
 0002:00005689       $N00157                    0000000180014689     java.exp
 0002:000056b5       $N00158                    00000001800146b5     java.exp
 0002:000056e0       $N00159                    00000001800146e0     java.exp
 0002:0000570e       $N00160                    000000018001470e     java.exp
 0002:00005732       $N00161                    0000000180014732     java.exp
 0002:0000576f       $N00162                    000000018001476f     java.exp
 0002:000057a4       $N00163                    00000001800147a4     java.exp
 0002:000057cb       $N00164                    00000001800147cb     java.exp
 0002:00005804       $N00165                    0000000180014804     java.exp
 0002:00005825       $N00166                    0000000180014825     java.exp
 0002:0000584d       $N00167                    000000018001484d     java.exp
 0002:00005872       $N00168                    0000000180014872     java.exp
 0002:00005897       $N00169                    0000000180014897     java.exp
 0002:000058be       $N00170                    00000001800148be     java.exp
 0002:000058e4       $N00171                    00000001800148e4     java.exp
 0002:00005908       $N00172                    0000000180014908     java.exp
 0002:0000592f       $N00173                    000000018001492f     java.exp
 0002:00005954       $N00174                    0000000180014954     java.exp
 0002:0000597a       $N00175                    000000018001497a     java.exp
 0002:000059a5       $N00176                    00000001800149a5     java.exp
 0002:000059cb       $N00177                    00000001800149cb     java.exp
 0002:000059ec       $N00178                    00000001800149ec     java.exp
 0002:00005a14       $N00179                    0000000180014a14     java.exp
 0002:00005a39       $N00180                    0000000180014a39     java.exp
 0002:00005a5e       $N00181                    0000000180014a5e     java.exp
 0002:00005a85       $N00182                    0000000180014a85     java.exp
 0002:00005aab       $N00183                    0000000180014aab     java.exp
 0002:00005acf       $N00184                    0000000180014acf     java.exp
 0002:00005af4       $N00185                    0000000180014af4     java.exp
 0002:00005b1a       $N00186                    0000000180014b1a     java.exp
 0002:00005b4b       $N00187                    0000000180014b4b     java.exp
 0002:00005b85       $N00188                    0000000180014b85     java.exp
 0002:00005bba       $N00189                    0000000180014bba     java.exp
 0002:00005be7       $N00190                    0000000180014be7     java.exp
 0002:00005c13       $N00191                    0000000180014c13     java.exp
 0002:00005c3c       $N00192                    0000000180014c3c     java.exp
 0002:00005c79       $N00193                    0000000180014c79     java.exp
 0002:00005cb3       $N00194                    0000000180014cb3     java.exp
 0002:00005cf3       $N00195                    0000000180014cf3     java.exp
 0002:00005d2b       $N00196                    0000000180014d2b     java.exp
 0002:00005d59       $N00197                    0000000180014d59     java.exp
 0002:00005d89       $N00198                    0000000180014d89     java.exp
 0002:00005dbb       $N00199                    0000000180014dbb     java.exp
 0002:00005ded       $N00200                    0000000180014ded     java.exp
 0002:00005e21       $N00201                    0000000180014e21     java.exp
 0002:00005e52       $N00202                    0000000180014e52     java.exp
 0002:00005e7b       $N00203                    0000000180014e7b     java.exp
 0002:00005ea9       $N00204                    0000000180014ea9     java.exp
 0002:00005ed7       $N00205                    0000000180014ed7     java.exp
 0002:00005f0a       $N00206                    0000000180014f0a     java.exp
 0002:00005f3b       $N00207                    0000000180014f3b     java.exp
 0002:00005f6b       $N00208                    0000000180014f6b     java.exp
 0002:00005f9d       $N00209                    0000000180014f9d     java.exp
 0002:00005fd5       $N00210                    0000000180014fd5     java.exp
 0002:00005fff       $N00211                    0000000180014fff     java.exp
 0002:00006025       $N00212                    0000000180015025     java.exp
 0002:0000604a       $N00213                    000000018001504a     java.exp
 0002:00006078       $N00214                    0000000180015078     java.exp
 0002:0000609a       $N00215                    000000018001509a     java.exp
 0002:000060bc       $N00216                    00000001800150bc     java.exp
 0002:000060dd       $N00217                    00000001800150dd     java.exp
 0002:000060fe       $N00218                    00000001800150fe     java.exp
 0002:00006123       $N00219                    0000000180015123     java.exp
 0002:00006156       $N00220                    0000000180015156     java.exp
 0002:00006189       $N00221                    0000000180015189     java.exp
 0002:000061c4       $N00222                    00000001800151c4     java.exp
 0002:000061ff       $N00223                    00000001800151ff     java.exp
 0002:00006233       $N00224                    0000000180015233     java.exp
 0002:00006266       $N00225                    0000000180015266     java.exp
 0002:000062a1       $N00226                    00000001800152a1     java.exp
 0002:000062d4       $N00227                    00000001800152d4     java.exp
 0002:00006305       $N00228                    0000000180015305     java.exp
 0002:00006337       $N00229                    0000000180015337     java.exp
 0002:00006372       $N00230                    0000000180015372     java.exp
 0002:000063a6       $N00231                    00000001800153a6     java.exp
 0002:000063e2       $N00232                    00000001800153e2     java.exp
 0002:00006423       $N00233                    0000000180015423     java.exp
 0002:00006463       $N00234                    0000000180015463     java.exp
 0002:00006493       $N00235                    0000000180015493     java.exp
 0002:000064c7       $N00236                    00000001800154c7     java.exp
 0002:000064f8       $N00237                    00000001800154f8     java.exp
 0002:0000652a       $N00238                    000000018001552a     java.exp
 0002:00006585       $N00239                    0000000180015585     java.exp
 0002:000065d6       $N00240                    00000001800155d6     java.exp
 0002:00006608       $N00241                    0000000180015608     java.exp
 0002:0000663c       $N00242                    000000018001563c     java.exp
 0002:00006675       $N00243                    0000000180015675     java.exp
 0002:000066b4       $N00244                    00000001800156b4     java.exp
 0002:000066ed       $N00245                    00000001800156ed     java.exp
 0002:00006723       $N00246                    0000000180015723     java.exp
 0002:00006755       $N00247                    0000000180015755     java.exp
 0002:0000678c       $N00248                    000000018001578c     java.exp
 0002:000067b7       $N00249                    00000001800157b7     java.exp
 0002:000067ee       $N00250                    00000001800157ee     java.exp
 0002:00006821       $N00251                    0000000180015821     java.exp
 0002:00006849       $N00252                    0000000180015849     java.exp
 0002:0000688b       $N00253                    000000018001588b     java.exp
 0002:000068d6       $N00254                    00000001800158d6     java.exp
 0002:00006927       $N00255                    0000000180015927     java.exp
 0002:0000697d       $N00256                    000000018001597d     java.exp
 0002:000069c7       $N00257                    00000001800159c7     java.exp
 0002:00006a15       $N00258                    0000000180015a15     java.exp
 0002:00006a64       $N00259                    0000000180015a64     java.exp
 0002:00006ab4       $N00260                    0000000180015ab4     java.exp
 0002:00006b01       $N00261                    0000000180015b01     java.exp
 0002:00006b4e       $N00262                    0000000180015b4e     java.exp
 0002:00006b92       $N00263                    0000000180015b92     java.exp
 0002:00006be3       $N00264                    0000000180015be3     java.exp
 0002:00006c2b       $N00265                    0000000180015c2b     java.exp
 0002:00006c86       $N00266                    0000000180015c86     java.exp
 0002:00006ccf       $N00267                    0000000180015ccf     java.exp
 0002:00006d27       $N00268                    0000000180015d27     java.exp
 0002:00006d6d       $N00269                    0000000180015d6d     java.exp
 0002:00006db0       $N00270                    0000000180015db0     java.exp
 0002:00006dfd       $N00271                    0000000180015dfd     java.exp
 0002:00006e44       $N00272                    0000000180015e44     java.exp
 0002:00006e8b       $N00273                    0000000180015e8b     java.exp
 0002:00006ed6       $N00274                    0000000180015ed6     java.exp
 0002:00006f23       $N00275                    0000000180015f23     java.exp
 0002:00006f6b       $N00276                    0000000180015f6b     java.exp
 0002:00006fb4       $N00277                    0000000180015fb4     java.exp
 0002:00006ffb       $N00278                    0000000180015ffb     java.exp
 0002:00007045       $N00279                    0000000180016045     java.exp
 0002:0000705b       $N00280                    000000018001605b     java.exp
 0002:0000706a       $N00281                    000000018001606a     java.exp
 0002:0000707e       $N00282                    000000018001607e     java.exp
 0002:0000708a       $N00283                    000000018001608a     java.exp
 0002:00007096       $N00284                    0000000180016096     java.exp
 0002:000070a1       $N00285                    00000001800160a1     java.exp
 0002:000070ad       $N00286                    00000001800160ad     java.exp
 0002:00008c28       .idata$6                   0000000180017c28     jvm:jvm.dll
 0002:00008d52       .idata$6                   0000000180017d52     advapi32:ADVAPI32.dll
 0002:00008d70       .idata$6                   0000000180017d70     ole32:ole32.dll
 0002:00008d92       .idata$6                   0000000180017d92     shell32:SHELL32.dll
 0002:00008de0       .idata$6                   0000000180017de0     version:VERSION.dll
 0002:00009596       .idata$6                   0000000180018596     kernel32:KERNEL32.dll
 0002:00009618       .idata$6                   0000000180018618     vcruntime:VCRUNTIME140.dll
 0002:0000988c       .idata$6                   000000018001888c     ucrt:api-ms-win-crt-heap-l1-1-0.dll
 0002:000098ac       .idata$6                   00000001800188ac     ucrt:api-ms-win-crt-string-l1-1-0.dll
 0002:000098ce       .idata$6                   00000001800188ce     ucrt:api-ms-win-crt-stdio-l1-1-0.dll
 0002:000098ee       .idata$6                   00000001800188ee     ucrt:api-ms-win-crt-convert-l1-1-0.dll
 0002:00009910       .idata$6                   0000000180018910     ucrt:api-ms-win-crt-runtime-l1-1-0.dll
 0002:00009932       .idata$6                   0000000180018932     ucrt:api-ms-win-crt-filesystem-l1-1-0.dll
 0002:00009958       .idata$6                   0000000180018958     ucrt:api-ms-win-crt-environment-l1-1-0.dll
 0003:00000000       methods                    0000000180019000     Class.obj
 0003:00000228       methods                    0000000180019228     ClassLoader.obj
 0003:00000900       methods                    0000000180019900     System.obj
 0003:00000950       methods                    0000000180019950     Thread.obj
 0003:00000b00       keyNames                   0000000180019b00     TimeZone_md.obj
 0003:00000b20       methods                    0000000180019b20     VM.obj
 0003:00000b40       methods                    0000000180019b40     VirtualThread.obj
 0003:00000be8       MAX_INPUT_EVENTS           0000000180019be8     io_util_md.obj
 0003:00000bec       ?curDirLenCached@?4??currentDirLength@@9@9 0000000180019bec     io_util_md.obj
 0003:00000bf0       cp1252c1chars              0000000180019bf0     jni_util.obj
 0003:00000d18       handleID                   0000000180019d18     NativeLibraries.obj
 0003:00000d20       jniVersionID               0000000180019d20     NativeLibraries.obj
 0003:00000d28       procHandle                 0000000180019d28     NativeLibraries.obj
 0003:00000d30       noSuchMethodErrCl          0000000180019d30     ObjectStreamClass.obj
 0003:00000d38       ProcessHandleImpl_Info_commandID 0000000180019d38     ProcessHandleImpl_win.obj
 0003:00000d40       ProcessHandleImpl_Info_commandLineID 0000000180019d40     ProcessHandleImpl_win.obj
 0003:00000d48       ProcessHandleImpl_Info_argumentsID 0000000180019d48     ProcessHandleImpl_win.obj
 0003:00000d50       ProcessHandleImpl_Info_totalTimeID 0000000180019d50     ProcessHandleImpl_win.obj
 0003:00000d58       ProcessHandleImpl_Info_startTimeID 0000000180019d58     ProcessHandleImpl_win.obj
 0003:00000d60       ProcessHandleImpl_Info_userID 0000000180019d60     ProcessHandleImpl_win.obj
 0003:00000d68       handleID                   0000000180019d68     RawNativeLibraries.obj
 0003:00000d70       ids                        0000000180019d70     WinNTFileSystem_md.obj
 0003:00000d80       ?u_path@?1??getHomeFromShell32@@9@9 0000000180019d80     java_props_md.obj
 0003:00000d90       ?sprops@?1??GetJavaProperties@@9@9 0000000180019d90     java_props_md.obj
 0003:00000e70       fastEncoding               0000000180019e70     jni_util.obj
 0003:00000e78       jnuCharset                 0000000180019e78     jni_util.obj
 0003:00000e80       String_init_ID             0000000180019e80     jni_util.obj
 0003:00000e88       String_getBytes_ID         0000000180019e88     jni_util.obj
 0003:00000e90       String_coder_ID            0000000180019e90     jni_util.obj
 0003:00000e98       String_value_ID            0000000180019e98     jni_util.obj
 0003:00000ea0       ?cls@?1??JNU_ClassString@@9@9 0000000180019ea0     jni_util.obj
 0003:00000eb0       GS_ExceptionRecord         0000000180019eb0     MSVCRT:gs_report.obj
 0003:00000f50       GS_ContextRecord           0000000180019f50     MSVCRT:gs_report.obj
 0003:00001420       ?__proc_attached@@3HA      000000018001a420     MSVCRT:dll_dllmain.obj
 0003:00001450       ?is_initialized_as_dll@@3_NA 000000018001a450     MSVCRT:utility.obj
 0003:00001451       ?module_local_atexit_table_initialized@@3_NA 000000018001a451     MSVCRT:utility.obj
 0003:00001458       ?module_local_atexit_table@@3U_onexit_table_t@@A 000000018001a458     MSVCRT:utility.obj
 0003:00001470       ?module_local_at_quick_exit_table@@3U_onexit_table_t@@A 000000018001a470     MSVCRT:utility.obj
 0005:00000060       $R000000                   000000018001c060     java.dll.res
